:020000040000fa
:08000000000c040000000000e8
:020000040000fa
:10180000ef2d210040772400000188000000000037
:10181000050007000c000700b229020000000000cc
:101820000040da000000fe004440a90040982c006f
:101830000000e0000300320010002000a00188003a
:101840004440a80000000600c02f2f000100200027
:101850001600370062004000e080480091018800d7
:101860009001ba0062004000e080480091018800c9
:101870009002ba0062004000e08048000002eb00e5
:101880006028e10005003a008301e9000700330009
:10189000038009000059eb00040037006128e100d3
:1018a000010032000082eb00050007009101880072
:1018b0001001ba000200e000e6ff3a000000050057
:1018c000910188008002780062004000e0804800ba
:1018d0003559ba008301e900080032002559ba00e1
:1018e0008301e900050032000400e000f4ff32004b
:1018f00015d9ba008301e900f1ff3a0000000600a3
:101900001017040000000000401704000000000051
:101910006e17040000000000901704000000000093
:10192000a617040000000000ce170400000000000d
:10193000f4170400000000002e180400000000004e
:101940006c18040000000000b8180400000000003b
:101950002a1a040000000000b61a0400000000006b
:10196000841c040000000000a61c0400000000000d
:10197000941d040000000000aa1d040000000000e7
:10198000c01d040000000000201e04000000000034
:101990003c1e040000000000621e04000000000065
:1019a000841e0400000000005445040000000000f4
:1019b0000e83040000000000b84604000000000090
:1019c0001e15040000000000e247040000000000b3
:1019d00034480400000000008848040000000000b3
:1019e000f861040000000000b2480400000000009c
:1019f000d448040000000000b649040000000000c4
:101a0000d475040000000000224a04000000000019
:101a10000c4b040000000000044c04000000000017
:101a2000d483040000000000745004000000000093
:101a3000c284040000000000e05d0400000000001b
:101a4000345e040000000000745e0400000000002a
:101a500058600400000000007c60040000000000ea
:101a6000d8600400000000003c8504000000000075
:101a70004a610400000000008a85040000000000a4
:101a8000b2610400000000001486040000000000a1
:101a90003e620400000000002e640400000000000c
:101aa000d0860400000000009064040000000000e4
:101ab000f2650400000000001e8704000000000022
:101ac0009c6604000000000066870400000000001f
:101ad000c068040000000000ce690400000000009f
:101ae0003288040000000000426a04000000000088
:101af000a46a040000000000be6b040000000000a7
:101b0000e06d040000000000908804000000000068
:101b1000666e040000000000c06e040000000000bb
:101b2000066f040000000000626f04000000000067
:101b3000c06f0400000000006e7004000000000090
:101b4000d8880400000000001e710400000000009e
:101b5000967204000000000096740400000000006b
:101b600078750400000000008415040000000000e7
:101b70007a29040000000000441504000000000061
:101b80006222040000000000c628040000000000db
:101b90006415040000000000281604000000000086
:101ba0003e29040000000000201504000000000091
:101bb0002629040000000000322904000000000073
:101bc000dc28040000000000702704000000000072
:101bd0001416040000000000582204000000000059
:101be0000216040000000000fa28040000000000b3
:101bf0009e22040000000000822204000000000079
:101c0000c0220400000000000e23040000000000b9
:101c1000a827040000000000f622040000000000d5
:101c2000d0150400000000002c2304000000000078
:101c3000ba24040000000000482404000000000052
:101c40005a23040000000000a22404000000000049
:101c50000824040000000000ca2404000000000062
:101c60009a230400000000003a160400000000005f
:101c70002c28040000000000f627040000000000eb
:101c80000428040000000000e62704000000000013
:101c900098240400000000009427040000000000c5
:101ca0009c290400000000009a15040000000000b8
:101cb000ac15040000000000d21804000000000071
:101cc00018190400000000002a1904000000000098
:101cd000061904000000000056190400000000006e
:101ce000441604000000000072160400000000000a
:101cf000de1604000000000060190400000000006f
:101d0000a6160400000000006a190400000000008c
:101d1000cc19040000000000741904000000000049
:101d20007e19040000000000041a040000000000f6
:101d3000161a040000000000d21a0400000000007f
:101d4000921a040000000000661a0400000000005f
:101d5000161b040000000000a41a0400000000008c
:101d60007c1a040000000000f61a040000000000c5
:101d7000e01a0400000000000c1b0400000000003a
:101d8000561b040000000000da1b040000000000e5
:101d9000601b040000000000a01b04000000000005
:101da000261b040000000000141c040000000000ba
:101db000401c04000000000088280400000000000f
:101dc0009428040000000000a02804000000000087
:101dd0005e1c040000000000701c040000000000f5
:101de000d01c040000000000de1c04000000000005
:101df000221d040000000000041d0400000000007b
:101e0000881d0400000000007c1d0400000000008c
:101e10006628040000000000421d040000000000cd
:101e2000541d040000000000681d040000000000b4
:101e30008818040000000000e01804000000000002
:101e4000f2180400000000009e1e040000000000c4
:101e5000ac1e040000000000ce1e040000000000c4
:101e6000f01e040000000000921f040000000000ab
:101e7000401f040000000000e21f040000000000fa
:101e80003220040000000000fa20040000000000de
:101e9000082104000000000072210400000000007e
:101ea000e2200400000000003c21040000000000cb
:101eb0009221040000000000b22104000000000094
:101ec000ec210400000000000622040000000000d5
:101ed00024220400000000002c2204000000000066
:101ee0003e2204000000000054290400000000000d
:101ef000c015040000000000682904000000000074
:101f0000020007000400be00000006006022b800c6
:101f1000060220000000d0008180d2000482d2009e
:101f20008582d2000000a0000202520083825a0083
:101f300003003b000202420083824a000000a1002d
:101f40000603e900f3ff3a0000000600839f6800e3
:101f50000100e00002003d0060001000e080180079
:101f60000300e00002003d0060011100e081190063
:101f7000e6ff07004f00e00002003b006000100099
:101f8000e080180000000600811f78000100e000da
:101f900002003d0060001000e08018000300e00037
:101fa00002003d0060011100e0811900d4ff07002c
:101fb0004f00e00002003b0060001000e0801800cd
:101fc0000000060023c2bf000008a300fdff32008e
:101fd00060022000303a88008000eb00213a88003f
:101fe000511688004600200086168800b116880029
:101ff0000080e800101788000020220040178800a9
:102000003116880090ff29006016880000802f009c
:102010009016880070fd2f00f016880000df200069
:102020002017880080d023001008880000022800b4
:10203000200888000ea1ef009008880030002000e2
:10204000700a880021138800e00320001013880024
:10205000050028000513880030102000401188007a
:10206000c0118800051188008511880000402200f9
:10207000101188009011880010002400601c880056
:1020800014042000b41c880013022000731c880074
:1020900082262000a21c880010002600001c880058
:1020a000541c8800131c8800421c8800013a8800d8
:1020b0002602880011048800210488003104880069
:1020c00041048800510488006104880040442400d1
:1020d00020058800300588004005880050058800ec
:1020e00060058800700588008005880090058800dc
:1020f000a0058800b0058800c0058800d0058800cc
:10210000e0058800f00588000006880010068800b9
:10211000200688003006880080812500a004880001
:1021200000002c00b004880030042000c0048800a7
:10213000d104880060002000e004880011028800bb
:10214000050488000000060000027800e2cf50007d
:1021500086003a000003780090027800858f5100d5
:1021600060003600e06b80000028a30039003200d8
:10217000eb8f420009003600030a7800e06b800014
:102180000020a100e06b8800d022a80011c0b3009d
:1021900090d720000148780097003700e0d8200051
:1021a0009080fb00f0d8200061407800ed4f500097
:1021b0001c003a00402d210010407800ec4f5000e8
:1021c00008003a00602d21001004e00002003200f7
:1021d0006a8a42001400370080252000008a4200ed
:1021e00011003700f34f50000c003a004027210047
:1021f000006890000004e00008003200702d21000b
:102200001004e000020032006a8a42000600370033
:1022100081252000018a4200030037006a8b4200ba
:10222000010037006a8a4200968f510072003e001a
:10223000030b7800e06b80000020a100e06b8800b9
:10224000d022a80011c0b30090d720000148780028
:1022500069003700e0d820009080fb00f0d8200013
:1022600061407800ed4f50001c003a00402d2100e5
:1022700010407800ec4f500008003a00602d21001b
:102280001004e00002003200050ae8005a0037009e
:10229000c0032000008a420057003700f34f50006f
:1022a0000c003a0040272100006890000004e00084
:1022b00008003200702d21001004e00002003200fe
:1022c000050ae8004c003700c1032000018a4200e3
:1022d00049003700050be80047003700050ae80011
:1022e00045003700e0d820009080fb00f0d82000a7
:1022f00061407800ed4f50001a003a00402d210057
:1023000031c1b30090cf10000e003a0041272100e8
:10231000016890000004e000050032000040eb007e
:1023200080689800c0948000000ae9000600370029
:1023300011c0b3004027210001689800000aeb009b
:1023400001003700020a7800402d2100b1c0b3001f
:1023500090cf100028003a00c0082000000b780041
:1023600025003700020a78002300370090407800eb
:102370000180fb00830f50001e003100e06b8000e5
:102380000028a30019003200ebcf400009003600fe
:10239000034a7800e06b80000020a100e06b880019
:1023a000d022a80011c0b30090d7200001487800c7
:1023b000110037006ac04000004a78000080fb002e
:1023c000808f51000c003e00034a7800e06b8000d3
:1023d0000020a100e06b8800d022a80011c0b3004b
:1023e00090d720000148780003003700014ae80038
:1023f00001003700024a780000000600e2cf5000da
:102400009f003a008002780010027800848f51000b
:102410000200310003087800bd003700840f51002e
:102420007a003100e06b80000028a3004d003200ec
:10243000e90f520009003e00820a7800e06b80003c
:102440000020a100e06b8800d022a80011c0b300da
:1024500090d7200001487800ad003700e0d8200078
:102460009080fb00f0d8200061407800ed4f5000d4
:1024700030003a00402d210010407800ec4f500011
:1024800012003a00602d21001004e000020032002a
:10249000ea0a52000200370080da2f00800a420068
:1024a000958f510024003100820a7800e06b800093
:1024b0000020a100e06b8800d022a80011c0b3006a
:1024c00090d72000014878001b003700f34f5000e0
:1024d00016003a0040272100006890000004e00048
:1024e00012003200702d21001004e00002003200c2
:1024f000ea0a52000200370080da2f00800a420008
:10250000958f51000c003100820a7800e06b80004a
:102510000020a100e06b8800d022a80011c0b30009
:1025200090d720000148780003003700ea0a5200e3
:1025300001003700ea0a5200950f5100740039007b
:10254000820a7800e06b80000020a100e06b880028
:10255000d022a80011c0b30090d720000148780015
:102560006b003700e0d820009080fb00f0d82000fe
:1025700061407800ed4f500022003a00402d2100cc
:1025800010407800ec4f50000b003a00602d210005
:102590001004e00002003200840ae9000200370063
:1025a00040fc2f00800a4200958f510058003100f6
:1025b000820a780056003700f34f50000f003a00af
:1025c00040272100006890000004e0000b0032006a
:1025d000702d21001004e00002003200840ae9009e
:1025e0000200370040fc2f00800a4200958f510006
:1025f00047003100820a780045003700840ae9006c
:1026000043003700840ae90041003700e0d8200089
:102610009080fb00f0d8200061407800ed4f500022
:1026200015003a00402d210031c1b30090cf1000b9
:102630000f003a0041272100016890000004e000eb
:10264000050032000040eb00806898004094800054
:10265000800a78002e00370011c0b3004027210007
:102660000168980061948000810a78002800370092
:10267000830a780026003700830a78002400370098
:1026800000027800904078000180fb00820f50002b
:102690001e003600e06b80000028a3001900320005
:1026a000e9cf500009003e00024a7800e06b80004c
:1026b0000020a100e06b8800d022a80011c0b30068
:1026c00090d7200001487800110037006ac0500000
:1026d000004a78000080fb00800f51000c0036009b
:1026e000024a7800e06b80000020a100e06b8800c7
:1026f000d022a80011c0b30090d720000148780074
:1027000003003700014ae90001003700034a78005e
:1027100000000600402d210010427800f44f5200c6
:1027200062003e000480fb0000004000c1e628007b
:102730006081780041e92800e08178000404e0002d
:1027400008003a00e193800040272100908f10009c
:1027500050003100818f51004e0036008101780019
:102760004c003700e24f520006003a00019480000e
:10277000c0938000810f5000460031008101780035
:1027800044003700e44f520008003a0021948000d2
:10279000e0938000810f50003e003100818f510096
:1027a0003c003600810178003a003700e84f5200c3
:1027b00006003a004194800020948000810f500070
:1027c000340031008101780032003700ed4f5200b3
:1027d00006003a004194800070948000810f500000
:1027e0002c003100810178002a003700f04f5200a0
:1027f00006003a0071948000a0948000810f500080
:10280000240031008101780022003700eb4f520094
:1028100006003a00f0252100c1c0b30090cf10009f
:102820001c003600430620001a003700f24f520009
:1028300009003a0043948000219480000101e900de
:10284000c09480000000e800808f50001100360026
:10285000c29488000f003700f34f52000d003a0079
:1028600040272100006890000004e00003003200cf
:10287000639480000001eb0006003700c2948000e2
:1028800043948000d0948000800f510001003600f6
:10289000d29488000480fb00000040004127210002
:1028a0000100400021c0b30027fe07000000060021
:1028b000402d210010427800f34f52005e003e0090
:1028c0000480fb0000004000c1e628006081780021
:1028d00041e92800e0817800e44f520006003a0008
:1028e000a1938000e0938000810f50004c003600df
:1028f000010178004a003700e64f520006003a0016
:10290000c193800000948000810f50004400360085
:102910000101780042003700e84f520006003a00fb
:10292000e193800020948000810f50003c0036002d
:10293000010178003a003700ea4f52000e003a00d9
:102940002594800071948000818f5200050036002c
:1029500040948000808f52003100310005017800e2
:102960002f00370040948000808f50002c003100f1
:10297000010178002a003700ed4f520006003a00ae
:10298000a194800070948000810f500024003600d4
:102990000101780022003700eb4f520006003a0098
:1029a000f0252100c1c0b30090cf10001c003600fc
:1029b000430620001a003700f24f520009003a0087
:1029c00043948000219480000101e900c0948000bc
:1029d0000000e800808f500011003600c29488008b
:1029e0000f003700f34f52000d003a00402721003e
:1029f000006890000004e00003003200639480004f
:102a00000001eb0006003700c29480004394800070
:102a1000d0948000800f510001003600d2948800cd
:102a20000480fb000000400041272100010040001d
:102a300021c0b30071fe0700000006000000060080
:102a4000f06b80000010a000f06b8800006c80002c
:102a50000060a100006c88008040eb00c0d920001d
:102a600001487800302d210001487800e0d820008e
:102a70001048e90000000600f0ff2c000c3e0200a8
:102a80000000000000000600206c80000040a00054
:102a9000206c8800116c8000f0f92f0080806000ad
:102aa000116c8800d02621001080fb0067006000b8
:102ab000e40f500003003a00010078000060a0001d
:102ac000106c88000000060002022000206c8000cc
:102ad00002007000206c8800116c8000f0f92f005b
:102ae00080806000116c8800d02621001080fb00df
:102af00067006000e30f500002003a00028070009f
:102b0000106c880000000600f06b80000010a00030
:102b1000f06b8800e1d820001140e8008048780080
:102b20000080fb0042c1b300f1d8200002f0780021
:102b300000000600b1d9200011407800e84f500095
:102b400002003e008048e80002003700b0d92000b3
:102b50000048eb0000000600b1d9200011407800c9
:102b60000004e000020032008048e9000300370062
:102b700091c0b300b0d920000148780000000600e1
:102b8000e1d820001140e800804878000080fb0078
:102b900092c0b300f1d8200002f0780000000600d7
:102ba000f06b80000010a000f06b8800e1d82000de
:102bb0001140e800804878000080fb00d2c0b300dc
:102bc000f1d8200002f07800006c80000060a100c5
:102bd000006c880081de200031409000b2c0b3005c
:102be0000440bc00414090000080fb000001410017
:102bf0008208780002407800088a02000000000085
:102c000000000600012d210011407800e84f50001f
:102c100002003e008048e80002003700002d21003d
:102c20000048eb0000000600012d21001140780053
:102c30000004e000020032008048e9000300370091
:102c400091c0b300002d210001487800000006006b
:102c5000f06b80000010a000f06b8800102d2100a8
:102c60000048eb0011c0b300c0d920000148780033
:102c700000000600006c800000d8a30001003a00ac
:102c8000f3ff070000000600c0da20009040780043
:102c9000e4cf500012003e00006c80000068a300ea
:102ca0000f0032000182fb0060ec280064407800d5
:102cb0008081fb0055da200063c17a0010ec280007
:102cc000e44078000240e90080f17a00814f510031
:102cd00003003a00c0eb28006442780084f17a00d7
:102ce00000000600c0da200090407800e4cf5000d9
:102cf00015003e00006c80000068a3001200320046
:102d00008181fb0060ec2800634078000081fb00bb
:102d100054da2000e2407a008140e80001717a0034
:102d20008180fb00c0eb2800634078000080fb003e
:102d30000000e800808f500003003a0010ec2800eb
:102d4000e341780003717a0000000600006c800007
:102d50000068a30018003200c1da2000114078009a
:102d60000004e000020032008048e9000300370060
:102d700041c0b300c0da200001487800c0da20006a
:102d80001081fb0060ec2800624078000080fb00ae
:102d900051da2000010040003096880011c0b300d5
:102da000802c210001487800c0eb280062407800a8
:102db0000080fb005096880000000600006c800038
:102dc0000068a30015003200c1da20001140e800bd
:102dd00080487800e44f5000010036008048eb0046
:102de000c0da20001081fb0060ec2800624078000f
:102df0000080fb0051da200001004000309688007e
:102e000011c0b300802c210001487800c0eb2800dd
:102e1000624078000080fb005096880000000600a9
:102e2000f06b80000010a000f06b8800006c800048
:102e30000060a000006c8800e1d820001140e8008c
:102e4000804878000080fb0052c1b300f1d8200018
:102e500002f07800206c80000070a000206c8800d8
:102e6000c0dd20003096880021c0b300802c2100f6
:102e700001487800001920005096880000000600e4
:102e8000f06b80000010a000f06b8800e1d82000fb
:102e90001140e800804878000080fb0062c1b30068
:102ea000f1d8200002f07800c0da20000048eb00e2
:102eb000006c80000060a000006c880070da2000c8
:102ec0003096880011c0b300802c210001487800a2
:102ed000700120005096880000000600f06b800012
:102ee0000010a000f06b8800006c80000080a10042
:102ef000006c8800206c80000090a000206c88008e
:102f0000e1d820001140e800804878000080fb00f4
:102f100072c1b300f1d8200002f078000000060072
:102f2000f06b80000010a000f06b8800e1d820005a
:102f30001140e800804878000080fb0082c1b300a7
:102f4000f1d8200002f0780000000600f06b80004d
:102f50000010a000f06b8800e1d820001140e800cc
:102f6000804878000080fb00b2c1b300f1d8200097
:102f700002f07800006c80000090a100006c8800d6
:102f8000006c800000e0a100006c8800006c8000f4
:102f900000a0a100006c880000000600502621005f
:102fa0000048eb00f06b80000010a000f06b880080
:102fb000e1d820001140e800804878000080fb0044
:102fc000c2c1b300f1d8200002f07800006c80008c
:102fd0000090a100006c8800306c80000030a000e0
:102fe000306c880000000600f06b80000010a0002c
:102ff000f06b8800e1d820001140e800804878009c
:103000000080fb00d2c1b300f1d8200002f07800ac
:10301000006c80000060a000006c880081de200051
:10302000514090000004e00002003a0010c0b300dc
:10303000d040980011c0b30080de200061409800ad
:10304000d0de200030968800802c210001487800d6
:10305000300620005096880000000600d0122000a4
:10306000406f8800d0c2b300088a02000000000050
:103070008041eb0002003700eacf5100050032002a
:103080000380fb000000400042272100c1ec280023
:10309000613178008341e800f3cf5100f6ff36003c
:1030a0008040eb004027210001689800f06b800011
:1030b0000010a000f06b8800e1d820001140e8006b
:1030c000804878000080fb00e2c1b300f1d8200006
:1030d00002f0780000000600f06b80000010a000f5
:1030e000f06b8800e1d820001140e80080487800ab
:1030f0000080fb0022c2b300f1d8200002f078006b
:10310000a1d9200090d920001148780000000600c5
:10311000d3d92000134178008280fb00a0e328006f
:10312000e1407800d0da200090cf50000d003a0046
:103130000240e80080497800e54f50000b003a005b
:10314000f06b80000010a000f06b8800e0d8200039
:103150001081fb0041c2b300f0d82000017178005b
:1031600002003700d0d920000048eb000000060024
:10317000d0d920000048eb00f06b80000010a000c8
:10318000f06b8800e1d820001140e800804878000a
:103190000080fb0032c2b300f1d8200002f07800ba
:1031a00000000600b0d920001080fb0000004000a5
:1031b00041ef280060807800000001000000060058
:1031c000e1d9200011407800e54f500002003e0098
:1031d0008048e80002003700e0d920000048eb00fa
:1031e00000000600e1d92000114078000004e00052
:1031f000020032008048e9000300370061c0b300dc
:10320000e0d920000148780000000600006c800032
:103210000068a30005003200031920000001eb0044
:1032200021c0b300c0dd2000c7fb0700000006007e
:10323000006c80000068a300050032000319200024
:103240000001eb0021c0b300c0dd20006bfc0700d3
:1032500000000600302d21000048eb00f06b8000dc
:103260000010a000f06b8800e0d820001081fb0067
:1032700061c0b300f0d820000171780000000600a2
:10328000302d21000048eb00f06b80000010a00002
:10329000f06b8800e0d820001081fb0071c0b30003
:1032a000f0d820000171780000000600f4ff07004c
:1032b000206c80000080a000206c880000000600c8
:1032c000efff0700206c80000030a000206c880019
:1032d00000000600006c80000088a30001003a0096
:1032e000e9fd070000000600006c80000088a300d4
:1032f00001003a00f4fd070000000600006c8000a9
:103300000088a30011003200006c80000098a30028
:1033100004003a005026210061c0b30090cf100095
:103320001c003600006c80000090a100006c88003a
:10333000c3fd0700902621000048eb00206c8000b0
:103340000010a000206c880012003700006c800084
:103350000080a000006c8800f06b80000010a000ce
:10336000f06b88008040eb00502621000148780077
:103370000000eb009095880050938800a09588008d
:10338000c026210001487800206c800000b0a00019
:10339000206c880000000600006c80000088a300fc
:1033a00017003200c02b21001004e00004003a0096
:1033b0005026210061c0b30090cf100005003600f8
:1033c0009ffd0700206c80000010a000206c88008a
:1033d0000c003700006c80000098a300040032004d
:1033e000006c80000090a100006c88000500370090
:1033f000006c80000090a000006c88000100370085
:103400008ffd070000000600f1d920001104e00044
:1034100003003a0010c0b300804878000200370073
:10342000f0d920000048eb0000000600f1d9200090
:10343000114078000004e000020032008048e900fa
:103440000300370011c0b300f0d920000148780014
:1034500000000600f06b80000010a000f06b8800f8
:10346000006c80000060a000006c8800006c800090
:103470000090a100006c8800502621000048eb005d
:10348000e1d820001140e800804878000080fb006f
:1034900092c1b300f1d8200002f07800206c8000c7
:1034a0000120220001007000206c880000dd200057
:1034b0003096880011c0b300802c210001487800ac
:1034c000600920005096880000000600006c800013
:1034d0000098a30004003200006c80000090a1005e
:1034e000006c880003003700006c80000090a00092
:1034f000006c880000000600006c80000098a300ab
:10350000070032004efd0700206c80000010a00074
:10351000206c8800006c80000090a100006c880086
:1035200000000600630920002203200011c0b30040
:1035300000dd2000b1fb0700206c800000a0a0008f
:10354000206c880000000600630920002203200090
:1035500011c0b30000dd2000fbfa0700206c8000e2
:1035600000a0a000206c880000000600f06b800026
:103570000010a000f06b8800e1d820001140e800a6
:10358000804878000080fb00a2c1b300f1d8200081
:1035900002f07800306c80000000a000306c8800e1
:1035a00000000600f0d920001080fb000000400061
:1035b00081f0280060807800000001000000060013
:1035c000e225210092407800f0c5b30080cf500082
:1035d00002003e000149e80003003700a1c5b30026
:1035e000e02521000148780000000600e2252100c6
:1035f00092407800a0c5b30080cf50000200360092
:103600000149e9000300370001c6b300e0252100ad
:10361000014878000000060019ff0700306c8000a8
:103620000010a000306c8800000006005026210029
:1036300011c0b30090cf100003003e00306c80003a
:103640000020a000306c880000000600006c8000a4
:1036500000a8a3000b003200902621000048eb00d8
:10366000006c800000c0a100006c8800206c80000d
:103670000060a1000010a000206c8800f0fc070092
:1036800009003700f06b80000010a000f06b88008c
:10369000006c800000a0a000006c8800006c80001e
:1036a00000c0a000006c880000000600006c8000d4
:1036b00000a8a3000100320065fd0700000006001d
:1036c000006c800000a8a3001b003200006c80008a
:1036d00000e8a30007003200006c800000e0a100b9
:1036e000006c8800206c80000010a000206c880016
:1036f00012003700006c800000e0a000006c880021
:103700000000eb0043272100c2f0280081022000c6
:10371000e23178000080e800810f5000fcff3a00a1
:103720000040eb0080699800306c800000c0a00071
:10373000306c880001003700c1fc07000000060063
:10374000006c800000a8a30019003200832520002f
:103750001200200021c0b300802d21007afa07005a
:10376000c1968000b0122000808f500007003e00fc
:103770000000e8000100500000004000f16d8000f2
:1037800001004000e06d8800060037000180400025
:1037900081da2f0001004000f16d80008080500030
:1037a000e16d8800206c800000a0a000206c8800e3
:1037b00000000600006c800000a8a3001900320081
:1037c000832520001200200021c0b300802d21009d
:1037d0000afb0700c1968000b0122000808f5000c5
:1037e00007003e000000e80001005000000040001b
:1037f000f16d800001004000e06d88000600370098
:103800000180400081da2f0001004000f16d80004e
:1038100080805000e16d8800206c800000a0a00036
:10382000206c880000000600006c80000098a30057
:1038300004003200006c80000090a100006c880041
:1038400003003700006c80000090a000006c88002e
:103850005026210031c0b30090cf10000700360081
:10386000006c80000090a100006c8800206c80003b
:103870000010a000206c880071fc0700000006000a
:10388000006c80000098a30004003a00502621003c
:1038900031c0b30090cf100007003600006c8000ec
:1038a0000090a100006c8800206c80000010a00037
:1038b000206c880062fc07000000060001da20008e
:1038c0001104e00003003a0010c0b3008048780003
:1038d0000200370000da20000048eb00000006007c
:1038e00001da2000114078000004e00002003200fc
:1038f0008048e9000300370011c0b30000da20005f
:103900000148780000000600f06b80000010a00065
:10391000f06b8800006c80000060a000006c8800e4
:10392000206c80000090a000206c8800e1d820006e
:103930001140e800804878000080fb00f2c1b3002d
:10394000f1d8200002f0780000000600f06b800043
:103950000010a000f06b8800006c80000060a000e8
:10396000006c8800e1d820001140e8008048780011
:103970000080fb0012c2b300f1d8200002f07800f2
:10398000802821003096880021c0b300802c2100bf
:1039900001487800803e2000509688000000060014
:1039a00000da20001080fb000000400041f32800f6
:1039b000608078000000010000000600f06b8000cd
:1039c0000010a000f06b8800006c80000090a10047
:1039d000006c8800502621000048eb00e1d8200050
:1039e0001140e800804878000080fb0002c2b3006c
:1039f000f1d8200002f07800306c80000050a00068
:103a0000306c880000000600006c80000098a30065
:103a100004003a005026210071c0b30090cf10007e
:103a20000700360006fc0700006c80000090a10033
:103a3000006c8800206c80002020b300206c88007f
:103a4000000006005026210071c0b30090cf100086
:103a500008003600fafb0700006c80000090a1000f
:103a6000006c8800206c80002020b300206c88004f
:103a700003003700006c80000090a200006c8800fa
:103a80000000060091d920001104e00003003a0074
:103a900010c0b300804878000200370090d92000a1
:103aa0000048eb000000060091d92000114078008a
:103ab0000004e000020032008048e9000300370003
:103ac00011c0b30090d92000014878000000060022
:103ad00090d9200090407800a0d9200001487800bb
:103ae00080de200021409800028d020000000000ce
:103af000e3fd070000000600833e2000423820005e
:103b000021c0b300802821008ff9070000000600c3
:103b1000833e20004238200021c0b30080282100cd
:103b200036fa070000000600f06b80000010a000cd
:103b3000f06b8800e1d820001140e8008048780050
:103b40000080fb0052c2b300f1d8200002f07800e0
:103b500000000600f06b80000010a000f06b8800f1
:103b6000e1d820001140e800804878000080fb0088
:103b700062c2b300f1d8200002f078000000060015
:103b8000f06b80000010a000f06b8800e1d82000ee
:103b90001140e800804878000080fb0072c2b3004a
:103ba000f1d8200002f07800006c80000060a000d6
:103bb000006c8800206c80000090a000206c8800c1
:103bc00010da200010417800e54f51000b0036005c
:103bd0008280fb00f0e32800614078000080fb0059
:103be00001db2000010040003096880011c0b300c6
:103bf000802c2100014878000b0037008280fb00f8
:103c0000f0e32800614078000080fb0000004000e5
:103c100001db2000010040003096880021c0b30085
:103c2000802c2100014878000280fb000000400049
:103c300081e428006080780050968800000006002b
:103c4000f06b80000010a000f06b8800e1d820002d
:103c50001140e800804878000080fb0082c2b30079
:103c6000f1d8200002f07800206c80000090a000c5
:103c7000206c880000000600f06b80000010a0009f
:103c8000f06b8800e1d820001140e80080487800ff
:103c90000080fb0092c2b300f1d8200002f078004f
:103ca000306c800000a0a000306c8800006c8000a8
:103cb0000090a100006c8800502621000048eb0015
:103cc00000000600f06b80000010a000f06b880080
:103cd000e1d820001140e800804878000080fb0017
:103ce000a2c2b300f1d8200002f07800206c80005e
:103cf0000090a000206c8800006c80000090a10063
:103d0000006c880000000600f06b80000010a0002e
:103d1000f06b8800e1d820001140e800804878006e
:103d20000080fb00b2c2b300f1d8200002f078009e
:103d300040da20000048eb0000000600e0d9200037
:103d40001080fb000000400081f3280060807800b4
:103d5000000001000000060002db2000e258900095
:103d600000c4b30080cf500003003e000140e800d3
:103d7000605998000300370031c2b30000db200017
:103d80006158980070958000c06d8800206c80009c
:103d900000a0a000206c88000000060002db2000cc
:103da000e258900030c2b30080cf500003003600cc
:103db0000140e900605998000300370011c4b300c6
:103dc00000db20006158980070958000c06d88006d
:103dd000206c800000a0a000206c8800000006007d
:103de00011da200011407800e74f500002003e0039
:103df0008048e8000200370010da20000048eb009d
:103e000010da200010417800e54f51000b00360019
:103e10008280fb00f0e32800614078000080fb0016
:103e200001db2000010040003096880011c0b30083
:103e3000802c2100014878000b0037008280fb00b5
:103e4000f0e32800614078000080fb0000004000a3
:103e500001db2000010040003096880021c0b30043
:103e6000802c2100014878000280fb000000400007
:103e700081e42800608078005096880000000600e9
:103e800011da2000114078000004e0000200320046
:103e90008048e9000300370081c0b30010da200039
:103ea0000148780010da200010417800e54f5100f9
:103eb0000b0036008280fb00f0e3280061407800b0
:103ec0000080fb0001db20000100400030968800ec
:103ed00011c0b300802c2100014878000b0037008e
:103ee0008280fb00f0e32800614078000080fb0046
:103ef0000000400001db20000100400030968800f7
:103f000021c0b300802c2100014878000280fb0012
:103f10000000400081e4280060807800509688000e
:103f200000000600006c8000010028000100700005
:103f3000006c8800006c80000068a3002000320044
:103f400010da200010407800e54f50000e003600d7
:103f50008080fb0081814000a0e52800630178009b
:103f6000f0e32800614078000080fb0001db2000c6
:103f70000100400081e42800e381780011c0b30013
:103f80001ef907000e0037008080fb008181400091
:103f9000a0e5280063017800f0e328006140780084
:103fa0000080fb000000400001db20000100400019
:103fb00081e42800e381780021c0b3000ff90700f5
:103fc00000000600006c8000010028000100700065
:103fd000006c8800006c80000068a30020003200a4
:103fe00010da200010407800e54f50000e00360037
:103ff0008080fb0081814000a0e5280063017800fb
:10400000f0e32800614078000080fb0001db200025
:104010000100400081e42800e381780011c0b30072
:1040200049f807000e0037008080fb0081814000c6
:10403000a0e5280063017800f0e3280061407800e3
:104040000080fb000000400001db20000100400078
:1040500081e42800e381780021c0b3003af807002a
:1040600000000600006c80000068a30054003200cd
:10407000f06b80000010a000f06b8800c06d800025
:10408000fd0f500006003e0010da20000048eb0053
:1040900011c0b300c0d920000148780048003700a3
:1040a000e16d8000d02e2000808f500007003e0080
:1040b00021c0b30010da20000148780011c0b3001d
:1040c000c0d92000014878003d003700f16d800024
:1040d000d02e2000808f500007003e0031c0b3007a
:1040e00010da20000148780011c0b300c0d92000c8
:1040f0000148780032003700316e8000f01820004f
:10410000808f500007003e0041c0b30010da20004d
:104110000148780011c0b300c0d9200001487800e0
:1041200027003700416e8000f0182000808f50007b
:1041300007003e0051c0b30010da200001487800ab
:1041400011c0b300c0d92000014878001c0037001e
:1041500000db2000e058900020c2b30080cf500068
:1041600007003e0061c0b30010da2000014878006b
:1041700011c0b300c0d920000148780010003700fa
:1041800000db20008060900010c3b30080cf50009f
:1041900007003e0071c0b30010da2000014878002b
:1041a00011c0b300c0d920000148780004003700d6
:1041b000206c800000a0a000206c880030fc07006c
:1041c00000000600006c80000068a30007003200b9
:1041d000206c80000090a000206c8800e0d82000b7
:1041e0001048e8001bfc07000100370014fa070024
:1041f00000000600006c80000068a30003003a0085
:10420000006c80000060a000006c880000000600c8
:10421000006c80000068a3001600320021da200044
:1042200011407800e24f500002003e008048e80054
:104230000200370020da20000048eb0020da2000de
:104240001080fb000000400061f4280060807800ce
:104250000000400001db2000010040003096880093
:1042600021c0b300802c210001487800803e20004e
:104270005096880000000600006c80000068a300d3
:104280001700320021da2000114078000004e0001d
:10429000020032008048e9000300370031c0b3005b
:1042a00020da20000148780020da20001080fb008e
:1042b0000000400061f428006080780000004000a9
:1042c00001db2000010040003096880021c0b300cf
:1042d000802c210001487800803e20005096880004
:1042e00000000600006c80000068a3000c00320093
:1042f00020da20001080fb000000400061f428005c
:10430000608078000000400001db200001004000d8
:10431000833e20000001eb0021c0b30037f8070006
:1043200000000600006c80000068a3000c00320052
:1043300020da20001080fb000000400061f428001b
:10434000608078000000400001db20000100400098
:10435000833e20000001eb0021c0b3007af7070084
:1043600000000600006c80000068a3000700320017
:10437000206c800000a0a000206c8800e0d8200005
:104380001048e800befb070012003700502621004d
:104390000048eb00006c80000090a100006c8800d9
:1043a000f06b80000010a000f06b8800e1d82000c6
:1043b0001140e800804878000080fb0002c2b30092
:1043c000f1d8200002f07800306c80000070a0006e
:1043d000306c8800000006005026210061c0b30048
:1043e00090cf100005003600206c80000010a00067
:1043f000206c880092f9070003003700006c8000f1
:104400000090a200006c880000000600006c800094
:104410000098a30004003a005026210061c0b300b8
:1044200090cf100007003600006c80000090a100c3
:10443000006c8800206c80000010a000206c8800b8
:104440007ff9070000000600006c80000090a000cb
:10445000006c880000000600006c80000098a3003b
:1044600004003200006c80000090a100006c880005
:104470000100370072f9070000000600006c8000a0
:104480000098a30009003200006c80000090a10099
:10449000006c88006000b800906e8800a16e8800f3
:1044a000206c800000a0a000206c880000000600a6
:1044b000401380008820a9009820a80060f9070018
:1044c000000006006000b800206f8800316f88008f
:1044d000bc89020000000000f06b80000010a0000a
:1044e000f06b8800e1d820001140e8008048780097
:1044f0000080fb00b2c0b300f1d8200002f07800c9
:104500000000060081de20000040eb00c040980063
:10451000314090000004e000030032000040e90058
:10452000b040980004003700c02521009040e90009
:1045300080de2000314098000000060083de20006d
:104540000040eb00c0419800334190008280fb00a6
:10455000c02521001080fb000000e900808f500082
:1045600003003d000240e800b0419800030037001e
:104570008040eb0080de2000314098000000060003
:1045800080de2000304090000080fb000100200011
:104590004a09dd00c600de00810071004a00dd002e
:1045a00002402000030020000000410081804900fb
:1045b000206f8800316f8800bc8902000000000075
:1045c000f06b80000010a000f06b8800e1d82000a4
:1045d0001140e800804878000080fb00c2c0b300b2
:1045e000f1d8200002f078000000060081de2000f3
:1045f000414090000004e000030032000040e90068
:10460000c040980004003700d02521009040e90008
:1046100080de2000414098000000060083de20007c
:10462000434190008280fb00d02521001080fb00d8
:104630000000e900808f500003003d000240e800c8
:10464000c0419800030037008040eb0080de20006e
:104650004140980000000600006c80000068a30044
:104660000b003200512d21001140e80080487800f5
:10467000ea4f5000010036008048eb00006c8000db
:104680000100280001007000006c8800080037005d
:10469000806f8000e10f400005003200088a0200b0
:1046a00000000000006c80000060a000006c88002a
:1046b00000000600006c80000068a3000e003200bd
:1046c000512d2100114078000004e000020032006a
:1046d0008048e90003003700a1c0b300502d21003d
:1046e00001487800006c8000010028000100700083
:1046f000006c88000e003700406f8000806f8800db
:10470000302d21000048eb00f06b80000010a0006d
:10471000f06b8800e1d820001140e8008048780064
:104720000080fb0022c1b300f1d8200002f0780025
:1047300000000600881f7800006c80000068a3005d
:104740001a003200402d210031c1b30090cf10007b
:104750000f003a0040272100006890000004e000ac
:104760000b003200602d21001004e0000a0032002e
:10477000702d21001004e000020032000048eb0020
:1047800005003700602d21000048eb0002003700d3
:10479000602d21000048eb00006c80000100280023
:1047a00001007000006c88001700370088de2000d0
:1047b000384090000080fb00010020004a09dd0025
:1047c000c600de00810071004a00dd0002402000ca
:1047d000030020000000410081804900206f880014
:1047e000316f8800bc8902000000000094f80700c7
:1047f000c0122000980f100003003a00006c8000e7
:104800000060a000006c88004f04780000000600e3
:10481000006c80000068a3001c003200402d2100c5
:1048200031c1b30090cf100011003a0040272100a1
:10483000006890000004e0000d003200602d2100af
:104840001004e00006003200712d21001104e00088
:104850000a003a0010c0b300804878000700370013
:1048600011c0b300602d210001487800030037001b
:1048700011c0b300602d210001487800006c800059
:104880000100280001007000006c88000000060094
:10489000881f7800006c80000068a3000b003200c5
:1048a000f06b80000010a000f06b8800e1d82000c1
:1048b0001140e800804878000080fb00f2c0b3009f
:1048c000f1d8200002f078001700370088de2000c1
:1048d000384090000080fb00010020004a09dd0004
:1048e000c600de00810071004a00dd0002402000a9
:1048f000030020000000410081804900206f8800f3
:10490000316f8800bc890200000000004cf80700ed
:10491000c0122000980f100003003a00006c8000c5
:104920000060a000006c88004f04780000000600c2
:1049300043f80700006c80000060a000006c880055
:1049400000000600006c800000f0a100006c8800f0
:10495000006c80000068a300020032006df70700c1
:1049600003003700006c80000060a000006c88002d
:1049700000000600006c800000f0a100006c8800c0
:10498000006c80000068a30001003200c8f7070037
:1049900000000600f06b80000010a000f06b8800a3
:1049a000006c80000068a3001d0132002394800089
:1049b000c02b2000808f51000b0036000194800036
:1049c00030062000808f500007003e00602d21003f
:1049d0000048eb0041c0b300502d21000148780091
:1049e0009bf807003d01370042948000828f510000
:1049f00007003600602d21000048eb0051c0b300d5
:104a0000502d21000148780091f80700330137004c
:104a1000e1938000818f510007003100602d21005b
:104a20000048eb0021c0b300502d21000148780060
:104a300087f807002901370070948000800f51002b
:104a400007003100602d21000048eb0051c0b30089
:104a5000502d2100014878007df807001f01370024
:104a6000a4948000840f500007003100602d2100c5
:104a70000048eb0091c0b300502d210001487800a0
:104a800073f8070015013700a0938000f30f500062
:104a900007003e000040eb00612d210080487800b7
:104aa000512d21008048780069f807000b0137007c
:104ab000808f5000070031000040eb00612d210085
:104ac00080487800512d21008048780060f8070068
:104ad00002013700d0938000ef0f5000070036002e
:104ae00010c0b300612d210080487800512d2100b5
:104af0008048780056f80700f8003700519480008d
:104b00000100e00008003a0011c0b300602d210050
:104b10000148780051c0b300502d210001487800b1
:104b20004bf80700ed003700c0082000808f5000d0
:104b30000800360011c0b300602d21000148780044
:104b400051c0b300502d21000148780040f8070003
:104b5000e20037003194800000e12000808f500097
:104b60000800360011c0b300602d21000148780014
:104b700041c0b300502d21000148780034f80700ef
:104b8000d6003700004b2000800f51000700360090
:104b9000602d21000048eb0051c0b300502d2100d2
:104ba000014878002af80700cc00370061948000a3
:104bb00000e12000808f50000800360011c0b300d3
:104bc000602d21000148780061c0b300502d210004
:104bd000014878001ef80700c0003700c694800026
:104be000860f510007003100602d21000048eb00c6
:104bf000a1c0b300502d21000148780014f807002f
:104c0000b6003700d5948000858f50000c0031002d
:104c100040272100006890000004e00008003200f6
:104c200011c0b300602d210001487800a1c0b3007d
:104c3000502d21000148780005f80700a700370033
:104c4000850f51000c0031004027210000689000c2
:104c50000004e00008003a0011c0b300602d2100fc
:104c600001487800a1c0b300502d21000148780010
:104c7000f7f7070099003700f30f520007003e00d6
:104c8000602d21000048eb0091c0b300502d2100a1
:104c900001487800eef7070090003700b0948000dc
:104ca000ef0f50000800360011c0b300602d210046
:104cb0000148780091c0b300502d210001487800d0
:104cc000e3f7070085003700c1938000009480005f
:104cd000808f500007003600602d21000048eb0057
:104ce00011c0b300502d210001487800d8f707000b
:104cf0007a00370010948000ef0f50000800360053
:104d000011c0b300602d21000148780031c0b3000c
:104d1000502d210001487800cdf707006f003700c3
:104d200080948000ef0f50000800360011c0b300df
:104d3000602d21000148780071c0b300502d210082
:104d400001487800c2f707006400370090948000a3
:104d5000ef0f50000800360011c0b300602d210095
:104d60000148780081c0b300502d2100014878002f
:104d7000b7f707005900370040272100006890006e
:104d80000004e00009003a00868f5100010036005f
:104d9000d6948800d1948000c0948000808f500009
:104da00002003e000000eb00d09488005194800087
:104db00040062000808f500002003600c00820000e
:104dc00050948800006c80000060a100006c880096
:104dd000302d21000048eb00006c800000c8a300cb
:104de00004003200306c800000d0a000306c8800dd
:104df00002003700e0d820001048e800e0d820008a
:104e00001081fb0081c0b300f0d820000171780050
:104e1000406f80009a8b0200000000002f003700d6
:104e20008040eb000004210001487800600421006c
:104e3000014878000000eb0090958800106c880015
:104e4000e2d82000924178000340e8000049780051
:104e5000f4d820000080fb00e1c0b30001707a00ac
:104e6000006c800000c0a000006c8800e1252100db
:104e700000c6b300914f10000d003a0040272100fa
:104e8000006890000004e00009003200d194800026
:104e9000004b2000808f50000500360003c0e80062
:104ea000004978000080fb0001c1b30001707a0066
:104eb000028d020000000000006c80000090a10044
:104ec000006c8800006c800000d0a100006c88009d
:104ed000306c800000c0a000306c8800000006002c
:104ee00080de2000304090000080fb0001002000a8
:104ef0004a09dd00c600de00810071004a00dd00c5
:104f00000240200003002000000041008180490091
:104f1000206f8800316f8800bc890200000000000b
:104f2000c7f6070000000600c5f60700406f8000c6
:104f3000088a020000000000006c800000c8a30086
:104f400002003200e0d820001048e900000006000e
:104f50006000b800206f8800316f8800bc890200b3
:104f600000000000b6f6070000000600006c80009c
:104f70000090a100006c8800006c800000d0a100af
:104f8000006c8800006c800000c0a100006c8800ec
:104f9000f06b80000010a000f06b88008040eb00f8
:104fa000e0d82000014878009026210001487800d0
:104fb000f0d8200001487800206c80000060a1003b
:104fc0000010a000206c880000000600006c80002b
:104fd0000098a30003003a00006c800000d8a300f2
:104fe00001003200e1ff070000000600006c8000b5
:104ff00000d8a30002003200dcff070001003700e8
:1050000032f9070000000600006c800000d8a30001
:105010000c00320081de2000d0122000910f100021
:105020000c003a00006c800000a0a000006c88001a
:10503000c3f90700006c800000a0a100006c88008c
:1050400004003700206c800001002800010070007f
:10505000206c880000000600006c800000d8a300cf
:105060000c00320081de2000d0122000910f1000d1
:1050700015003a00006c800000a0a000006c8800c1
:10508000ccf90700006c800000a0a100006c880033
:105090000d003700f06b80000010a000f06b88005e
:1050a000e1d820001140e800804878000080fb0033
:1050b000d2c0b300f1d8200002f07800006c80006c
:1050c0000060a000006c8800000006004094800092
:1050d000c1c72f000100400041062000810f500091
:1050e0000a003e00406f80009a8b02000000000022
:1050f000206c80000090a000206c8800006c800074
:105100000060a100006c880022fe0700000006007d
:10511000330620001200200011c0b300d0de2000b2
:10512000b6f407000000060033062000120020003d
:1051300011c0b300d0de200003f407000000060019
:10514000c0122000406f8800c0c2b300088a02006d
:1051500000000000006c80000060a100006c88006e
:10516000f06b80000010a000f06b8800e1d82000f8
:105170001140e800804878000080fb00d2c0b300f6
:10518000f1d8200002f0780000000600f06b8000eb
:105190000010a000f06b8800e1d820001140e8006a
:1051a000804878000080fb0012c1b300f1d82000d5
:1051b00002f07800000006008040eb0090262100fd
:1051c00001487800e0d8200001487800f0d820009d
:1051d00001487800f06b80000010a000f06b8800a0
:1051e000206c80000060a1000010a000206c8800ee
:1051f00000000600f06b80000010a000f06b88003b
:10520000e1d820001140e800804878000080fb00d1
:10521000a2c0b300f1d8200002f078000000060020
:10522000f06b80000010a000f06b8800e1d8200037
:105230001140e800804878000080fb0012c0b300f5
:10524000f1d8200002f0780000000600234e200074
:105250000001eb0021c0b300c02d2100baf307000c
:1052600000000600234e20000001eb0021c0b30027
:10527000c02d210061f4070000000600f06b8000e3
:105280000010a000f06b8800e1d820001140e80079
:10529000804878000080fb0022c0b300f1d82000d5
:1052a00002f078000000060041da2000114078008a
:1052b0000004e000020032008048e90003003700eb
:1052c00081c0b30040da20000148780000000600e9
:1052d00041da200011407800e74f500002003e0004
:1052e0008048e8000200370040da20000048eb0068
:1052f000000006000000eb000c3e02000000000071
:10530000e1d820001140e800804878000080fb00d0
:1053100032c1b300f1d8200002f07800406c800068
:105320000020a000406c8800206c80000050a0008d
:10533000206c880000000600f06b80000010a000c8
:10534000f06b8800e0d820001048e900902621008a
:105350000048eb00406c80000030a000406c8800ea
:1053600000000600889fbe0020df20000076880035
:1053700060e5200010768800e20f020000000000c7
:1053800022c2bf000008a3000500320031118000d6
:1053900022c2bf000008a300fcff3a00816f880012
:1053a00032c2bf000008a30005003200b111800026
:1053b00032c2bf000008a300fcff3a00816f8800e2
:1053c0005a3b020000000000e1d820001140e80034
:1053d000804878000080fb0032c0b300f1d8200084
:1053e00002f078000080eb00806f8800808c020063
:1053f00000000000f0ff2c000c3e02000000000046
:10540000306c80000000a000306c8800406c800090
:105410000010a000406c8800206c80000028b300c1
:10542000206c8800f06b80000000a000f06b88000a
:1054300040a7a8000060fe00d07580000038a300df
:1054400008003200207b020000000000d0758000c0
:105450000030a100d0758800006c80000010a10011
:10546000006c8800d07580000098a300080032000e
:10547000e67f020000000000d07580000090a100cf
:10548000d0758800006c80000020a100006c8800ae
:10549000006c80000008a30072013200006c8000e4
:1054a0000038a30073003a00902621009040780055
:1054b00000c2b30080cf500027003a00006c80008b
:1054c00000c8a3006b003a00e1d820001140e800ba
:1054d000804878000080fb00e2c0b300f1d82000d3
:1054e00002f07800006c800000c0a000006c880012
:1054f000206c80000090a000206c8800f06b800081
:105500000010a000f06b880088de2000384090007a
:105510000080fb00010020004a09dd00c600de001b
:10552000810071004a00dd000240200003002000dd
:105530000000410081804900206f8800316f8800a1
:10554000bc8902000000000018007800088a0200f0
:105550000000000047003700facf500010003a006a
:10556000e2d8200092407800f3d820000180fb00b0
:1055700060c07900e54f50003e003200f06b8000c3
:105580000010a000f06b88000140e800004978009e
:105590000080fb0051c0b30001f0790035003700f6
:1055a000eacf500010003a00e2d820009240780084
:1055b000f3d820000180fb0060c07900f74f500055
:1055c0002c003200f06b80000010a000f06b88000f
:1055d0000140e800004978000080fb0071c1b30081
:1055e00001f0790023003700fecf50000f003a0091
:1055f000006c800000d0a000006c8800e3d8200080
:10560000134178008280fb00f0d8200061407800d0
:10561000ee4f5000170032008249e900f06b800025
:105620000010a000f06b88001200370020c2b30009
:1056300080cf50000f003a00e2d82000924078005e
:10564000f3d820000180fb0060c07900f34f5000c8
:10565000080032000140e800004978000080fb00ab
:1056600031c1b30001f079000000eb000c3e0200f4
:1056700000000000226c8000020078001004b300db
:10568000206c8800e0d82000104278008480fb0065
:10569000f0d82000e1417800f6cf510004003a0034
:1056a000f06b80000000a000f06b88000300370062
:1056b000020078005004b300206c8800c0d920009c
:1056c000104178000204e0000c003200102d21008f
:1056d0009040e80001487800e9cf5000070036000c
:1056e000e06b80000000a000e06b8800d022a800e2
:1056f00011c0b30090d72000014878000380fb0060
:105700000100200063005000e08058006302200088
:10571000830f5000e08f5800b1003e000060010090
:1057200026003700ae003700a700370033003700ef
:105730003200370038003700a9003700a8003700d2
:10574000a7003700a6003700a50037007300370018
:10575000a3003700370037006c0037002700370000
:105760009f0037009e0037009d0037009c003700e7
:10577000370037009a0037004300370098003700a1
:105780005d00370045003700950037009400370072
:105790009300370045003700910037009000370034
:1057a0008f0037008e003700480037004300370075
:1057b0008b0037008a00370048003700312d210068
:1057c0001140e80080487800f34f50008400360014
:1057d0008048eb00e0d820000448e900d022a8006f
:1057e00011c0b30090d7200001487800f06b800012
:1057f0000010a000f06b880079003700302d2100e8
:105800009040e80001487800e3cf50007400360073
:105810008bf4070072003700302d21009040e80023
:1058200001487800e3cf50006d003600acfd070062
:105830006b003700302d21009040e80001487800cf
:10584000eecf5000660036007df40700640037009c
:10585000206c800000c0a000206c88005026210031
:1058600061c0b30090cf10005d003600d022a800c8
:1058700090d7200011c0b3000148780051c0b30098
:105880000148780056003700206c80000120240079
:1058900001007000206c880051003700306c8000df
:1058a0000040a000306c88004d003700306c800054
:1058b0000060a000306c880049003700306c800028
:1058c0000080a000306c880045003700306c8000fc
:1058d0000030b300306c880041003700306c80002d
:1058e00000b0a000306c8800206c80000090a00008
:1058f000206c88003a003700306c800001002800de
:1059000001007000306c880035003700406c80006a
:105910000010a000406c880031003700306c80001f
:1059200011002c0001007000306c8800406c800079
:105930000000a000406c8800006c800000d8a3002c
:10594000270032000204e000010032003cf40700ae
:105950005193800070252000808f500006003e008b
:10596000d022a80090d7200011c0b30001487800d1
:1059700051c0b3000148780090958000e30f5000bb
:105980001700360081de2000c0122000910f1000a9
:1059900013003a006141900051409000804f510047
:1059a0000f0031000240e800e0409800e0d82000fd
:1059b0001048e900f06b80000010a000f06b880038
:1059c000f4fb070006003700d022a80090d7200083
:1059d00011c0b3000148780081c0b30001487800cd
:1059e000e0d820009080fb00f0d82000e140780053
:1059f000eccf500005003e00ebcf50000a00310014
:105a00000104e0000800320005003700f4cf500028
:105a10000500320040c2b30080cf500002003200c7
:105a20008004eb000c0037008904e800b01220006d
:105a3000808f540008003600106c8000f1f92f00b0
:105a400001006000106c8800206c80000050a000f5
:105a5000206c88008004eb00006c80000000a10036
:105a6000006c8800e06b80000008a3002400320076
:105a7000c0d920001004e000080032008040eb0094
:105a800001487800102d210001487800f06b80005b
:105a90000010a000f06b88000d003700e0d8200057
:105aa0009080fb00f0d820006140780092c0b300e5
:105ab0000440bc00d0da20001080fb00000141004f
:105ac00002014100e0ff28006200780000000100b0
:105ad000f06b80000000a000f06b8800f06b80008d
:105ae0000030a100f06b8800202d21000048eb0061
:105af000e06b80000000a100e06b88008004eb00f8
:105b0000f06b80000008a30018003200f06b8000ea
:105b10000000a100f06b8800f06b80000018a3006b
:105b200004003200d4f30700f06b80000010a100e5
:105b3000f06b8800e0d820009080fb00f0d82000b7
:105b4000614078000080fb0000004000c1d92000c7
:105b50009180fb00e18060000100400000004000f7
:105b6000e1f428006080780000000100006c8000f3
:105b70000018a30019013a00006c8000e8006000e2
:105b800016013a00d02621001040780067406000de
:105b9000226c80000248a3000f0032000040e900a0
:105ba000e14f500004003e00a0c0b300b8780200ee
:105bb000000000000400370021c0b300a0c0b30003
:105bc000b878020000000000206c80000000a000f7
:105bd000206c8800010137000258a3001000320039
:105be0000040e900e14f500005003e008040eb001e
:105bf000a0c0b300b8780200000000000400370025
:105c000011c0b300a0c0b300b878020000000000cb
:105c1000206c80000000a000206c8800ef0037009e
:105c20000238a300050032008040eb0000c1b30041
:105c3000b878020000000000e80037000228a30046
:105c4000050032008040eb00f0c0b300b8780200dd
:105c500000000000e1003700416c80000118a30043
:105c6000050032008040eb0010c0b300b87802009d
:105c700000000000d90037000200e00005003d00f0
:105c800031c0b30010c1b300b878020000000000ba
:105c9000d2003700306c80000058a30005003200ad
:105ca0008040eb0070c2b300b87802000000000032
:105cb000ca0037000078a300050032008040eb00e6
:105cc00080c2b300b878020000000000c3003700b3
:105cd00002d8a300050032008040eb00a0c2b30050
:105ce000b878020000000000bc00370002e8a30002
:105cf000050032008040eb00b0c2b300b87802006b
:105d000000000000b50037000038a3000500320095
:105d10008040eb00c0c2b300b87802000000000071
:105d2000ae0037000048a300050032008040eb00c1
:105d3000d0c2b300b878020000000000a70037000e
:105d400002b8a300050032008040eb00e0c2b300bf
:105d5000b878020000000000a000370002c8a300cd
:105d6000050032008040eb00f0c2b300b8780200ba
:105d700000000000990037000068a3000500320011
:105d80008040eb0000c3b300b878020000000000c0
:105d9000920037000278a300050032008040eb003b
:105da00050c3b300b8780200000000008b00370039
:105db0000288a300050032008040eb0060c3b300fe
:105dc000b8780200000000008400370002a8a30099
:105dd000050032008040eb0040c3b300b8780200f9
:105de000000000007d0037000298a300050032008b
:105df0008040eb0030c3b300b87802000000000020
:105e0000760037000088a300050032008040eb00d8
:105e100070c3b300b8780200000000006f003700c4
:105e20000000e00005003d008040eb0080c3b300af
:105e3000b878020000000000680037000098a30056
:105e4000050032008040eb0090c3b300b878020038
:105e500000000000610037000108a30005003200c7
:105e60008040eb00c0c3b300b8780200000000001f
:105e70005a00370000e8a300050032008040eb0024
:105e800060c4b300b878020000000000530037007f
:105e90000028a300050032008040eb0070c4b3006e
:105ea000b8780200000000004c0037000018a30082
:105eb000050032008040eb0080c4b300b8780200d7
:105ec00000000000450037000008a3000500320074
:105ed00001c8b30080c4b300b8780200000000001d
:105ee0003e00370000a8a300050032008040eb0010
:105ef000a0c4b300b87802000000000037003700eb
:105f000000b8a300050032008040eb00b0c4b3002d
:105f1000b8780200000000003000370000c8a3007d
:105f2000050032008040eb00e0c3b300b878020007
:105f3000000000002900370000d8a300050032004f
:105f40008040eb00f0c3b300b8780200000000000e
:105f5000220037000128a300050032008040eb003a
:105f6000c0c4b300b8780200000000001b00370076
:105f70000138a300050032008040eb00d0c4b3001c
:105f8000b878020000000000140037000268a30087
:105f9000050032008040eb0030c6b300b878020044
:105fa000000000000d0037000208a30005003200c9
:105fb0008040eb0030c0b300b87802000000000061
:105fc000060037000218a300040032008040eb00f6
:105fd00020c0b300b878020000000000006c800010
:105fe0000048a30040013200f095800001302000fd
:105ff00001006000810f500036013a00f0958000ea
:10600000020820000200600011968000810f5000fd
:1060100019013200f0958000020060000200320099
:1060200012968800020037000000eb0010968800ee
:10603000f09580000074a100112c210080487800a8
:106040000080fb0001002000b2032000820f5000fe
:10605000e08f5800e5003e00006001009b00370023
:10606000a1003700a7003700e0003700df0037004d
:10607000de003700dd003700dc003700a800370005
:10608000ae003700b400370030003700360037006c
:106090003c003700b7003700d4003700bb003700a2
:1060a000c1003700c7003700d0003700cf003700ed
:1060b0003b003700cd003700cc003700c800370068
:1060c000ca003700c9003700c8003700c7003700d2
:1060d000c600370039003700c4003700c30037005e
:1060e000c2003700c1003700c0003700bf003700d2
:1060f00054003700bd0037005c003700bb0037009c
:106100006b00370063003700b8003700b700370076
:10611000b6003700b5003700b4003700b3003700d1
:10612000b2003700b1003700b0003700af003700d1
:10613000ae003700270037002d003700ab003700d6
:1061400032003700a90037003700370041c0b300e4
:10615000d0da200001487800e06b80000000a00049
:10616000e06b8800a100370071c0b300d0da2000d6
:1061700001487800e06b80000000a000e06b880020
:106180009a00370011c0b300d0da2000014878002f
:10619000e06b80000000a000e06b880093003700f7
:1061a00021c0b300d0da200001487800e06b800005
:1061b0000000a000e06b88008c003700d0da2000df
:1061c0000048eb00e06b80000000a000e06b88005e
:1061d0008600370081c0b300d0da20000148780083
:1061e000e06b80000000a000e06b88007f003700bb
:1061f00061c0b300d0da200001487800e06b800075
:106200000000a000e06b88007800370031c0b300c8
:10621000d0da200001487800e06b80000000a00088
:10622000e06b88007100370051c0b300d0da200065
:1062300001487800e06b80000000a000e06b88005f
:106240006a003700006c80000068a300670032001d
:1062500051c0b300d0da200001487800e06b800024
:106260000000a000e06b880060003700006c800038
:106270000068a3005d00320021c0b300d0da200026
:1062800001487800e06b80000000a000e06b88000f
:1062900056003700206c80000040a000206c880071
:1062a000f06b80000000a000f06b88004f0037000a
:1062b000206c80000050a000206c8800f06b8000f3
:1062c0000000a000f06b88004800370011c0b30048
:1062d000102c210001487800106c800000a0a00064
:1062e000106c88004100370041c0b300102c210021
:1062f00001487800106c800000a0a000106c88009d
:106300003a00370071c0b300102c2100014878001a
:10631000106c800000a0a000106c880033003700d3
:1063200021c0b300102c210001487800106c8000bf
:1063300000a0a000106c88002c00370051c0b300f2
:10634000102c210001487800106c800000a0a000f3
:10635000106c88002500370081c0b300102c21008c
:1063600001487800106c800000a0a000106c88002c
:106370001e003700102c21000048eb00106c80003c
:1063800000a0a000106c88001800370031c0b300d6
:10639000102c210001487800106c800000a0a000a3
:1063a000106c88001100370061c0b300102c210070
:1063b00001487800106c800000a0a000106c8800dc
:1063c0000a00370091c0b300102c2100014878006a
:1063d000106c800000a0a000106c88000300370043
:1063e000106c800000a0a000106c8800006c800081
:1063f0000058a30004003a00d022a80011c0b30046
:1064000090d7200001487800006c80000050a10067
:10641000006c8800e06b80000020a100e06b880029
:10642000102c21009040780050c2b30080cf500063
:106430000a00320003003e00f5cf50000a003a0087
:106440000600370070c2b30080cf50000300320056
:106450007440400080cf500003003a00402c2100df
:106460000048eb001b003700a1c0b300402c210006
:106470000148780017003700412c21001140e80046
:1064800080487800e94f50000d003a00a0c0b300ea
:1064900080487800d022a80011c0b30090d7200017
:1064a00001487800e06b80000020a000e06b8800cd
:1064b000e06b80000000a000e06b88000500370062
:1064c000ea4f500003003600a1c0b300402c210069
:1064d000014878000000eb00f0958800006c800017
:1064e0000040a100006c8800106c800000a8a30090
:1064f000d0fb320000a0a100106c8800006c80006e
:106500000068a300cbfb3200e5d8200015427800dc
:10651000f6d820000480fb0060407b00ed4f500067
:10652000c8003a00402d2100104178008281fb0014
:106530008380410040e92800e10378007240510067
:10654000e14f50000c003e00f06b80000010a000f6
:10655000f06b880091c0b300f0da200001487800a9
:106560000440e800804a78000080fb0041c0b3008e
:1065700001707b00affb3700ec4f510082003a0006
:10658000602d21001004e00040003200102c21009a
:1065900090427800f8cf520014003a0061948000d5
:1065a000c2032000811f7800110009008280d800fa
:1065b00001007800cf007800a2002000809fbe007c
:1065c000110009000280d800000178004f00be00d1
:1065d000808050000101410062948800006c8000be
:1065e00000f0a100006c880092fb3700006c800076
:1065f0000000e0000e003d0060948000c203200017
:10660000801f7800110009000280d8004f00780038
:10661000010050008580fb0001004000609488006c
:10662000006c800000f0a100006c880081fb370046
:1066300063948000c2032000110009008281d80009
:10664000010278006a20b9000581fb00800041004a
:10665000b0032000808f50000800360004805100f5
:10666000b003b00060948800006c80000100280036
:1066700001007000006c88006efb37000480510040
:1066800000804000609488006afb3700102c2100d5
:1066900090427800f8cf520011003a0060948000d8
:1066a000c3032000801f7800110009000380d80078
:1066b000010278004f0078008225200011000900b7
:1066c0000280d8000380b900000242006494880070
:1066d000006c800000f0a100006c880055fb3700c2
:1066e000006c80000000e0000d003d006094800020
:1066f000c2032000110009000280d8008101780047
:106700000580fb000280b90080814100639488000d
:10671000006c800000f0a100006c880045fb370091
:1067200064948000c2032000110009000282d80096
:10673000010378006a00b9008581fb008081410077
:10674000828f51000800360050dd20000000430019
:1067500060948800006c8000010028000100700037
:10676000006c880033fb3700c203200011000900d1
:106770000282d8008000fd000299b90002004000aa
:10678000609488002bfb3700102c21001042780009
:10679000f84f52000e003a0083804100402721004c
:1067a0008080400011007800a2002000811f780046
:1067b000110009000280d800cf007800800878001e
:1067c000006c800000f0a100006c880019fb37000d
:1067d000006c80000000e00008003d0003814100e3
:1067e0008480fb004027210001317800006c80008c
:1067f00000f0a100006c88000efb37004627210046
:106800008382410065007b006a00b9000481fb00bf
:1068100000014100828f53000600310087327b0067
:10682000006c80000100280001007000006c8800ee
:1068300000fb370083804100402721008230780030
:10684000fcfa3700802c210010407800e14f500006
:1068500016003a0033968000102c21001041780079
:10686000f84f510006003a001380fb00a200200000
:10687000110009000280d80080497800edfa370045
:106880001380fb006a00b9000281fb000000410098
:1068900051968000810f5000020036008149780037
:1068a000e4fa370080497800e2fa3700e24f5000fe
:1068b000e0fa3a0033968000102c21001041780055
:1068c000f84f510006003a0013007800a2002000a3
:1068d000110009000280d80080097800d5fa37003d
:1068e000130078006a00b9000281fb00000041003b
:1068f00051968000810f5000020036008109780017
:10690000ccfa370080097800cafa3700809fbe00b1
:10691000821f780071d720009148e80070c2b30050
:10692000914f10000b0036008048eb00006c800097
:106930000000a000006c880061d720009148e800aa
:1069400030c6b300914f10000200360080c0b30083
:1069500080487800212d21009148e80070c2b300e2
:10696000914f1000040036008048eb00f06b80006f
:106970000030a200f06b8800006c80000018a300bb
:1069800011003200e20321001249e80070c2b30096
:10699000924f10000c0036008040eb000149780057
:1069a000c0eb20000148780020df2000007688003e
:1069b000006c80000010a100006c8800d075800081
:1069c0000020a100d0758800006c80000038a30072
:1069d00014003200f20321001249e80070c7b3002e
:1069e000924f10000f0036008040eb000149780004
:1069f000d0eb20000148780060e520001076880088
:106a0000006c80000020a100006c8800d075800020
:106a10000080a100d0758800006c80000030a100cb
:106a2000006c8800e0da200010407800e14f500050
:106a30002800320003003900e24f50006f003a0096
:106a400049003700d042a80000000000000000000c
:106a5000e002ab0006003200e06b80000030a000d6
:106a6000e06b8800d0da20000048eb00150037000a
:106a7000e022ab0007003200e06b80000030a00095
:106a8000e06b880011c0b300d0da20000148780024
:106a90000c003700e0c2ab0007003200e06b800062
:106aa0000030a000e06b880021c0b300d0da2000e5
:106ab0000148780003003700e06b80000030a1003f
:106ac000e06b8800d042a900e0da20001048e8001e
:106ad0004c003700d1a2a800000000000000000018
:106ae000e002ab0007003200e06b80000040a00035
:106af000e06b880031c0b300d0da20000148780094
:106b000015003700e022ab0007003200e06b800088
:106b10000040a000e06b880041c0b300d0da200044
:106b2000014878000c003700e0c2ab0007003200db
:106b3000e06b80000040a000e06b880051c0b30013
:106b4000d0da20000148780003003700e06b8000b5
:106b50000040a100e06b8800d1a2a900e0da20008b
:106b60001048e80027003700d1c2a800000000004c
:106b700000000000e002ab0007003200e06b800084
:106b80000050a000e06b880061c0b300d0da2000a4
:106b90000148780015003700e022ab000700320002
:106ba000e06b80000050a000e06b880071c0b30073
:106bb000d0da2000014878000c003700e0c2ab00ba
:106bc00007003200e06b80000050a000e06b8800fe
:106bd00081c0b300d0da20000148780003003700fc
:106be000e06b80000050a100e06b8800d1c2a900da
:106bf000e0da20000048eb0002003700e0da200075
:106c00000048eb00e06b8000e16b8000e26b8000ed
:106c100068006000f0806000010070000202b200b5
:106c20000200700042003200e06b80000018a300f8
:106c30001500320081d720009148e800b0c2b300af
:106c4000914f10002d0036006340500080487800be
:106c5000d022a80011c0b30090d7200001487800ce
:106c6000e06b80000000a000e06b8800006c8000fa
:106c70000068a30021003200e06b80000020a0002b
:106c8000e06b88001d003700e06b80000028a30047
:106c900005003200e06b80000020a100e06b88005e
:106ca00080d720000048eb0080d720001048e80083
:106cb00071c2b30090cf100003003600e06b80007b
:106cc0000010a000e06b880080d720009040780082
:106cd000e1cf500009003a00d022a80090d7200050
:106ce00001487800e06b80000000a000e06b8800a5
:106cf000e06b80000020a100e06b8800f06b80005a
:106d00000048a30029003a00f06b80000050a10069
:106d1000f06b8800f06b80000040a000f06b8800f2
:106d2000f06b80000000a000f06b88001f003700af
:106d3000e06b80000010a100e06b8800e06b800039
:106d40000028a3000b00320081d720009148e80002
:106d5000b0c2b300914f10000800360063405000ed
:106d600080487800e06b80000000a000e06b8800a5
:106d70000200370080d720000048eb00f06b800055
:106d80000058a30009003a00f06b80000040a10009
:106d9000f06b8800f06b80000050a000f06b880062
:106da000f06b80000000a000f06b880090d72000fe
:106db0001004e000020032001048e9000100370032
:106dc000d022a9008460a9004f0178004f00be00c6
:106dd00000400600809fbe0040138000006c8000d1
:106de0000008a30033003200e0dd200010407800ee
:106df000e14f50000d00320005003900e24f500015
:106e000011003200e34f500027003a001b0037000a
:106e1000e0dd20001048e80040de20002040900027
:106e20000080fb00401388002f003700e0dd2000c9
:106e30001048e80040de2000104090000080fb0079
:106e40004013880028003700e1dd20009148e80069
:106e500040de20001080fb0040138800606c800042
:106e60000028a300200032008048eb00006c800066
:106e70000000a100006c88001b003700006c80003f
:106e80000000a100006c88008000eb004113880026
:106e90009820a900e0dd20000148780081e3a800e7
:106ea0008de3a80010003700e0dd20000048eb0073
:106eb0000d003700606c80000018a3000a003a0043
:106ec000606c80000028a30007003200606c800026
:106ed0000040a100606c88009820a9008de3a80004
:106ee00081e3a80083e3a8008820a9004f00be002a
:106ef00000400600809fbe00821f780060c2a9008b
:106f0000e1d820001140e800804878000080fb00b4
:106f100042c0b300f1d8200002f0780011c0b300e5
:106f2000f0da2000014878008800a9004f017800bd
:106f30004f00be0000400600809fbe00829fbe0042
:106f4000b01180008041780087c0a900d075800012
:106f50000028a30018003200e1cf41000b003a00e6
:106f6000c1eb20001104e000040032000076800034
:106f70000000e900007688009148e900d0758000a3
:106f80000020a100d075880016003700e0eb20003b
:106f90000348780030df20000076880011c0b3007d
:106fa000c0eb200001487800d07580000020a100cf
:106fb000d07588000b003700e0eb200010c84100be
:106fc000e1cf410004003a00d07580000020a0000d
:106fd000d075880003003700d07580000020a10024
:106fe000d07588000076800003587800007688000d
:106ff000c2eb20001249e80040c0b300924f1000dd
:10700000210036009280fb0020df200030409000fd
:107010000080fb0064004000808f50001a003400a4
:10702000e0eb2000104078000340500080cf51007a
:1070300008003a000049eb00d07580000030a00045
:10704000d0758800d07580000020a100d075880020
:107050000d0037008040eb00c0eb200001487800b5
:10706000e00321000148780020df2000007688003e
:10707000006c80000010a100006c8800d0758000ba
:107080000020a100d07588004f01be004f00be0057
:1070900000400600809fbe00829fbe0087e0a900de
:1070a000c1eb2000c003210011417800904f510036
:1070b000020039008048eb0008003700c3eb2000d5
:1070c000134178008280fb0040ec20006140780092
:1070d0000080fb00a01188008249e8004f01be003b
:1070e0004f00be0000400600809fbe00821f780057
:1070f00022c2bf000028a3000300320041c0b30039
:10710000f0da20000148780022c2bf000018a30076
:10711000040032002222a90051c0b300f0da20009e
:1071200001487800e1d820001140e800804878004c
:107130000080fb0042c0b300f1d8200002f07800cc
:107140008c20a9004f0178004f00be0000400600cf
:10715000809fbe00829fbe00301180008041780079
:107160008560a900d07580000088a3001800320057
:10717000e1cf41000b003a00d1eb20001104e00008
:1071800004003200107680000000e90010768800cc
:107190009148e900d07580000080a100d07588007a
:1071a00016003700f0eb20000348780070e520005f
:1071b0001076880011c0b300d0eb200001487800a1
:1071c000d07580000080a100d07588000b003700ca
:1071d000f0eb200010c84100e1cf410004003a006c
:1071e000d07580000080a000d075880003003700b3
:1071f000d07580000080a100d075880010768000d6
:107200000358780010768800d2eb20001249e8007d
:1072100040c0b300924f1000210036009280fb0066
:1072200060e52000304090000080fb0064004000da
:10723000808f50001a003400f0eb200010407800de
:107240000340500080cf510008003a000049eb0095
:10725000d07580000090a000d0758800d0758000a7
:107260000080a100d07588000d0037008040eb0041
:10727000d0eb200001487800f0032100014878009d
:1072800060e5200010768800006c80000020a100de
:10729000006c8800d07580000080a100d075880047
:1072a0004f01be004f00be0000400600809fbe00a0
:1072b000821f780032c2bf000028a3000300320002
:1072c00021c0b300f0da20000148780032c2bf00cc
:1072d0000018a300040032003222a90031c0b3001c
:1072e000f0da200001487800e1d820001140e800e1
:1072f000804878000080fb0042c0b300f1d8200035
:1073000002f078008c40a9004f0178004f00be00c9
:1073100000400600809fbe00829fbe008580a900bd
:10732000d1eb2000d003210011417800904f510093
:10733000020039008048eb0008003700d3eb200042
:10734000134178008280fb0000f820006140780043
:107350000080fb00201188008249e8004f01be0038
:107360004f00be0000400600809fbe00821f7800d4
:107370004e01ab000400320020002000700a88009b
:107380000a21ef002d003700620a8000b0e02f00d4
:1073900000004100e14a2000810f50000b003e0038
:1073a000002c21001048e90090407800f295800000
:1073b0008180fb00100020000100dd000080ea0059
:1073c00002006000f095880012003700708f2f00d7
:1073d0000000410061892000810f50000a003e003a
:1073e000002c21001048e90090407800f2958000c0
:1073f0008180fb00100020000100dd000200700011
:10740000f095880003003700c1c0b300002c2100b4
:1074100001487800012c21001104e00005003a0029
:10742000c0c0b30080487800006c80000040a0001d
:10743000006c880030002000700a880088c0a90015
:107440004f0178004f00be0000400600801f78000a
:10745000606c80000018a30003003200606c8000a4
:107460000060a000606c88008de3a90085c0a900c1
:107470004f00780000400600809fbe00821f780009
:10748000e1d820001140e800804878000080fb002f
:1074900042c0b300f1d8200002f0780061c0b30010
:1074a000f0da20000148780080a0a9004f017800a0
:1074b0004f00be00004006003600f800809fbe006e
:1074c000829fbe00849fbe00869fbe00606c8000cd
:1074d0000028a3001b003200006f8000116f8000a5
:1074e0002004b0000180b000006f8800116f880098
:1074f000606c80000060a000606c8800006f8000fd
:10750000116f80000221200003002000800f020084
:1075100000000000e00f5000e08f580009003a0022
:10752000e922a800e0dd20000048eb00606c80004c
:107530000040a000606c8800606c80000030a000fb
:10754000606c880081e3a9008480a9004f03be001d
:107550004f02be004f01be004f00be003600f900d2
:1075600000400600809fbe00821f780071c0b300fb
:10757000f0da200001487800e1d820001140e8004e
:10758000804878000080fb0042c0b300f1d82000a2
:1075900002f078008040a900d022a8004f017800b6
:1075a0004f00be0000400600809fbe00821f780092
:1075b00081c0b300f0da200001487800e1d8200053
:1075c0001140e800804878000080fb0042c0b30012
:1075d000f1d8200002f078008060a900d022a80035
:1075e0004f0178004f00be0000400600e9e2a9000c
:1075f000b016880000ff2a00e822b600e9a2a90020
:107600005216880000000000e9a2a8000000060051
:107610000002be0000002800e822b70001ff2a0097
:107620008000fd00e822b6008000fd00040060003c
:1076300001003200e982a8000508a3000100320021
:10764000e9c2a800b4168800c529dd004b20de0081
:1076500000807100cb28de006f006000e822b700d8
:10766000e9a2a9005216880000000000e9a2a800c3
:1076700000000600889fbe008a1f78000045780041
:107680000204be000080fb0001002000d7ff0700bd
:107690004049de00030020000a80fb000000e800f3
:1076a000cf80de00d1ff07004f0578004f04be00f9
:1076b00000000600889fbe008a1f7800d022a80024
:1076c00011c0b30090d720000148780080672e00d9
:1076d0000000e900feff3a006831290069382900fe
:1076e0006a3829003980fb000000d1003801be0053
:1076f000e0ff0700880f5500faff3a004f057800b9
:107700004f04be0000000600889fbe008a9fbe0096
:107710008c1f7800030678000002be000005eb0015
:107720008285fb00000820000a80de0000806500e2
:10773000f2ff2c0001003a000c01780061044200c5
:10774000e0844a000400be00b1ff07000a05e8001b
:10775000e80f5500020032000802be00f1ff3700ba
:107760004f0678004f05be004f04be000000060023
:107770000f02b000889fbe008a9fbe008c9fbe0093
:107780008e1f780080b79f0091b79f00c2e79f00cf
:10779000e3e79f00c4b79f00d5b79f000300d10067
:1077a00061006000f0df9f000004e00004003a0088
:1077b00042372d00c2af9f0001c2b3000b0037005b
:1077c00000c2b300cfe1970080cf510004003a001f
:1077d000c0b22c00c0af9f00834078000300370088
:1077e000c1b22c00c1af9f0001c3b3004fa99700e5
:1077f00072419000c2d79f00a02d2100024878005e
:10780000cfe197000380fb008180fb000100500066
:107810004200dd00cfa89700008040001049900092
:10782000e2df9f0082467800a04890008180fb0044
:10783000304890004800dd0000877000cfd19700ed
:107840000304e000b3003200e3d79f00efe09700ad
:107850008180fb0081bf9f006fd197000280fb00f9
:107860008003e900613ab9009fb19700030242002a
:10787000e0824a00001420000021b80000a8b900ee
:10788000830140000fb0970000054100e0854900ea
:10789000ffd897000104e000070032006011b80033
:1078a000d2af9f00e3af9f0000c2b300cfe19700cb
:1078b00080cf510050003200f0cf56002900360032
:1078c000cfa897006ec078000000fb0001002000e8
:1078d000c800dd000000200002f02f00010261005e
:1078e00005002000cfa997000e83410016409000ac
:1078f0000000fb0001002000c000dd0000002000af
:10790000f30f2000018161000300200004017100d9
:1079100085817100c011dd0002002000264090002a
:107920004800dd0001f02f00010060000100200090
:1079300000017100818171003640900064074700aa
:107940000000fb00f10f200001006000010020009a
:107950000001710081817100d2af9f00e3af9f00f1
:1079600025003700e8cf56001a0036004fa99700cf
:107970006e4079000000fb0001002000c800dd001f
:107980000000200003f02f000181610003002000af
:10799000cfa897000e804000104090000000fb0030
:1079a0000e87e80001002000c000dd00000020007c
:1079b0000180fb0001002000020070008380700045
:1079c000c000dd0000002000d0af9f00e1af9f00ad
:1079d000090037004fa997006e4079000000fb00b6
:1079e0000e07e80001002000c800dd0000002000b4
:1079f000d0af9f00e1af9f00efd997000304e000f4
:107a00003a0032000006eb000fb89700e0b79f0085
:107a100087834300f7b79f00000020000100280083
:107a20000c0178000201e900030033008100d1005d
:107a30000080d300fbff3700dfa99700030160003f
:107a4000efa99700038060006102b800c020dd004c
:107a5000000020006112b8000400700085807000f2
:107a6000e00f5000e08f58000d0032006fe09700eb
:107a70000004e00011003d00f06b80000038a3001e
:107a80000e003200efb097000108a3000d00320095
:107a9000ffb19700403c2900630178000a003700dd
:107aa000efb097000108a30006003200ffb1970075
:107ab000403c290063017800030037005fb1970064
:107ac000010037004fb1970061044500e0844d008c
:107ad0000a00be00cefe07000c06e8008ccf560060
:107ae000020036000805be00cbff3700efd097003c
:107af0008140e900e1d79f000080eb004fd1970063
:107b00000090b90000404100efd1970080cf5100b4
:107b100051ff3a000d80fb004f0778004f06be0072
:107b20004f05be004f04be000f02b100000006006a
:107b3000889fbe008a9fbe008c9fbe008e1f78006b
:107b40008005780082047800034778008406780076
:107b5000050678000004780001057800250037004c
:107b6000ea4f510006003a00ef0f550001003600c1
:107b7000700555008904e8000b04780014003700f4
:107b8000e94f510009003a00c2022000110009002b
:107b90000284d8000100780000005400c8022000d0
:107ba000000444008904e800090037008904e80063
:107bb0008c0278000d0278008e4178008a007800ef
:107bc00008007800eafe07000080fb000004440083
:107bd000d00f2000800f540006003600ef0f550034
:107be00002003e000b0478000200370070055500cb
:107bf0000b047800194178000204e000d8ff3a0035
:107c0000080078004f0778004f06be004f05be0001
:107c10004f04be0000000600889fbe008a9fbe0081
:107c20008c1f7800000678006044b8000ac022006b
:107c30001b0020000c0178000800be0074fe070045
:107c400061044400e0844c008a0f54008b8f5c0078
:107c5000f8ff3a004f0678004f05be004f04be0003
:107c600000000600889fbe008a9fbe008c9fbe0059
:107c70008e1f7800000578008005eb006044b80096
:107c80000cc022001d002000fe132000040037005d
:107c90008e8f5500020036000a85ea008005eb0051
:107ca0000a0178000800be0059fe07008b05e800b5
:107cb00061044400e0844c008c0f54008d8f5c0004
:107cc000f3ff3a004f0778004f06be004f05be0095
:107cd0004f04be0000000600889fbe008a9fbe00c1
:107ce0006044b80002802f000800be0048fe070074
:107cf00061044400e0844c0000402600800f5400e2
:107d0000e08f5c001b003200f6ff37000a402600bf
:107d10000b002000027e20000800be003cfe070091
:107d200061044400e0844c0061055500e0855d007d
:107d3000f8ff3a00f0bf220011002000800f54002d
:107d4000818f5c0010003e00f20120000800be00a0
:107d50002ffe070061044400e0844c0000c02200b4
:107d600011002000800f5400818f5c00060032005b
:107d7000f5ff3700f07f2c00800f5400e08f5c008f
:107d8000f1ff3e00e1ff37004f05be004f04be008b
:107d9000000006001c00fa00889fbe008a9fbe00fb
:107da0008c9fbe006000b800c0af9f00d1af9f00a5
:107db0000c802f004fac9700dfac97000a0f20001b
:107dc000cfa89700c50ddd000c8175000800be002e
:107dd0000ffe07000a05e9000814b0000980b00092
:107de0000a00e000f8ff3a004fa89700dfa89700cc
:107df00061004000e0804800c0af9f00d1af9f000d
:107e0000f2032000820f5000e08f5800e9ff3a0093
:107e1000fd0120000c7e20004fac9700dfac9700e6
:107e20000a0f2000cb6ddd000c8175000800be003c
:107e3000f7fd07000a05e9000814b0000980b0004a
:107e40000a00e000f8ff3a004fa89700dfa897006b
:107e500061004000e0804800c0af9f00d1af9f00ac
:107e60008d06e900ecff3a000004be000a0f200076
:107e7000027e20000800be00e5fd07000a05e900bb
:107e80000814b0000980b0000a00e000f8ff3a00d2
:107e90004fa89700dfa8970061004000e0804800ed
:107ea000e0af9f00f1af9f006000b800a0b79f0057
:107eb000b1b79f000c7e2000afb597006fac970064
:107ec000ffac97000a0f20000c8175000800be006f
:107ed000cffd07000a05e9000814b0000980b000d2
:107ee0000a00e000f8ff3a006fa89700ffa897008b
:107ef00061004000e0804800e0af9f00f1af9f00cc
:107f00002fb09700bfb0970061004000e0804800ac
:107f1000a0b79f00b1b79f00ff0f5000e08f58003f
:107f2000e5ff3a00fd0320000c0f20006fac970026
:107f3000ffac97000005eb00c56ddd000b0178007c
:107f4000f201b3000800be00b1fd07000a05e80019
:107f50000814b0000980b0008c0f5500f7ff3a00fc
:107f60006fa89700ffa8970061004000e0804800dc
:107f7000e0af9f00f1af9f008d06e900ebff3a00f4
:107f80000004be000d0578000b0f2000f201200058
:107f90000800be009efd07000a05e8000814b000b6
:107fa0000980b0008b0f5500f8ff3a006fa89700ca
:107fb000ffa8970061004000e080480080bf9f005c
:107fc00091bf9f006000b800c0b79f00d1b79f006d
:107fd0000c0f20000fbc97009fbc97000005eb0022
:107fe000cfb09700cb0ddd000b017800f201b3009c
:107ff0000800be0086fd07000a05e8000814b0006e
:108000000980b0008c0f5500f7ff3a000fb89700b9
:108010009fb8970061004000e080480080bf9f004b
:1080200091bf9f004fb09700dfb097006100400004
:10803000e0804800c0b79f00d1b79f00ff0f5000fd
:10804000e08f5800e3ff3a00fb0120000d802f0075
:108050000c0f20000fbc97009fbc97000005eb00a1
:108060000d8175000800be0069fd07000a05e800e3
:108070000814b0000980b0008c0f5500f8ff3a00da
:108080000fb897009fb8970061004000e08048005b
:1080900080bf9f0091bf9f008b05e900edff3a0074
:1080a0000004be0002802f000800be0058fd07003b
:1080b0000a05e9000814b0000980b0000a00e000d9
:1080c000f8ff3a000fb897009fb897006100400092
:1080d000e080480080b79f0091b79f006000b80023
:1080e000e0b79f00f1b79f000c802f000fb49700fe
:1080f0009fb497000a0f2000efb09700c50ddd0078
:108100000c8175000800be0041fd07000a05e9006a
:108110000814b0000980b0000a00e000f8ff3a003f
:108120000fb097009fb0970061004000e0804800ca
:1081300080b79f0091b79f006fb09700ffb0970086
:1081400061004000e0804800e0b79f00f1b79f0069
:10815000f2032000820f5000e08f5800e3ff3a0046
:108160004b0020000fb497009fb497000a0f200027
:1081700002fe2f000800be0025fd07000a05e900e9
:108180000814b0000980b0000a00e000f8ff3a00cf
:108190000fb097009fb0970061004000e08048005a
:1081a00080b79f0091b79f008b05e900edff3a0073
:1081b0004f06be004f05be004f04be000080fa000f
:1081c00000000600ea874700889fbe008a9fbe0025
:1081d0008c9fbe008e1f7800e0b79f00f1b79f0014
:1081e0000404be000347780086f79f0087067800e6
:1081f0000281fb008202e9001a0020000b0020002f
:108200000042eb000003eb000500e00003003c002f
:10821000a4ef9f0004467800360037006a50b8008b
:108220006a59b900810041000005be000442e8001f
:108230000480fb00850f5000f8ff35000046eb007e
:10824000e00f5500e08f5d002f003200a6ef9f0089
:1082500006467800270037000040eb000a0454006f
:108260008b845c000040e800880f5500898f5d001a
:10827000faff360001c3b300014140000004e000f2
:108280000300320010c0b300a0ef9f0007003700ca
:10829000e10f5500e08f5d0004003600afe8970065
:1082a0000104e00001003a000ff197000c80fb0090
:1082b000efb09700010040009fb297000d027800d8
:1082c0008e417800ffb0970029fd07000046460068
:1082d000a2002000030020000a00be00860f02005a
:1082e000000000000005be00e00f5000e08f5800c5
:1082f000050032000040eb00880f5500898f5d00bb
:10830000dcff3e00d4ff37000c80fb004f077800f5
:108310004f06be004f05be004f04be00af00b100c7
:1083200000000600889fbe008a9fbe008c9fbe0092
:10833000000678008105780003007800820f56005f
:108340000200360082045600010037008c04510000
:10835000808f550002003600008455000100370070
:108360000b045000888f540042003600820f5600e4
:10837000200031000005eb000d142000808f550017
:108380000e0031000ac0b900110009000980d800b0
:10839000008045000d01b8000a00460000004100c1
:1083a000e080490002802f0099fc07000a05e800e0
:1083b0008a8f54007c003900f2ff37000ac0b900f0
:1083c000110009000980d800008055000d01b80097
:1083d0000a00460000004100e080490002802f00b2
:1083e0008bfc07000a05e8008a8f54006e003900f4
:1083f000f2ff37000005eb000d142000808f5500c0
:108400000e0031000ac0b900110009000980d8002f
:10841000008045000d01b8000a0056000000410030
:10842000e080490002802f0079fc07000a05e8007f
:108430008a8f54005c003900f2ff37000ac0b9008f
:10844000110009000980d800008055000d01b80016
:108450000a00560000004100e080490002802f0021
:108460006bfc07000a05e8008a8f54004e003900b3
:10847000f2ff3700820f5600260031000005eb00a6
:108480000d142000808f5500110031000a80450036
:108490000d00b8000ac9b900809fbe001100090094
:1084a0000881d800000178004f00be00020146009c
:1084b00002004000e080480002802f0054fc0700ca
:1084c0000a05e8008a0f540037003900efff370033
:1084d0000a8055000d00b8000ac9b900809fbe008f
:1084e000110009000881d800000178004f00be008b
:1084f0000201460002004000e080480002802f0098
:1085000043fc07000a05e8008a0f540026003900e2
:10851000efff37000005eb000d142000808f5500a1
:10852000110031000a8045000d00b8000ac9b900e9
:10853000809fbe00110009000881d800000178006a
:108540004f00be000201560002004000e0804800db
:1085500002802f002efc07000a05e8008a0f540055
:1085600011003900efff37000a8055000d00b800f8
:108570000ac9b900809fbe00110009000881d80017
:10858000000178004f00be000201560002004000ca
:10859000e080480002802f001dfc07000a05e8006b
:1085a0008a0f5400f0ff31004f06be004f05be0099
:1085b0004f04be0000000600889fbe008a1f78009e
:1085c000a4d920001482fb00253a29000080fb007a
:1085d000000040000400400060c57a008180fb007c
:1085e0008180400084804000e1c47a000281fb0069
:1085f000020141000401410062c47a008381fb0052
:10860000838141008481410063c17a0080d72000ca
:108610001004e00016003200d0da200031c0b300b0
:1086200090cf100002003a00794545001000370055
:10863000d0da200051c0b30090cf100002003a0001
:10864000f9c444000a003700d0da200021c0b3008a
:1086500090cf100002003a00794444000400370033
:10866000d0da20001004e00001003a007941410016
:108670008000eb0080102000de8d02000000000072
:1086800008417800c103200080102000de8d020028
:1086900000000000094178009107200080102000b0
:1086a000de8d0200000000000a417800610b20000e
:1086b00080102000de8d0200000000004f057800d1
:1086c0004f04be0000000600889fbe008a9fbe00c7
:1086d0008c1f78000004780001057800824578003e
:1086e000034678000204e00003003a00f101200094
:1086f0000304e00001003a008000eb0050da2000a3
:1087000020429000811f7800f7ff2c0006c2b300c2
:108710008041eb000482fb000500200022c0b30072
:108720008a00780008007800a6fe07000080fb00a1
:10873000000444008002eb00f4ff2c008541780027
:10874000a2c3b3008a0078000800780008fc070084
:108750000080fb00800444008f87e900e1cf5500d2
:1087600003003a00f00120000c04e00001003a0090
:108770000000eb0058da200018429000801f7800bb
:10878000f7ff2c0006c3b3008041eb000482fb001e
:108790000500200022c0b3008a007800090078009c
:1087a00088fe07000080fb00808444008002eb000c
:1087b000f4ff2c0085417800a2c3b3008a00780042
:1087c00009007800eafb0700184278000080fb00ef
:1087d000008044008001eb00831f7800f7ff2c002d
:1087e00006c3b3000482fb000500200022c0b300d2
:1087f0008a00780073fe0700e48757004f06780070
:108800004f05be004f04be0000000600889fbe005a
:108810008a9fbe000004be000245780083457800b0
:10882000e24f510003003a00f10120000304e00090
:1088300001003a008000eb0050da20004042900036
:10884000811f7800f7ff2c0006c2b3008041eb00c7
:108850000482fb000500200022c0b3000800be0017
:1088600058fe07000080fb00000444008002eb007b
:10887000f4ff2c0085417800e2c2b3000800be007e
:10888000bbfb07000080fb00000444008f87e90069
:10889000e34f550003003a00f10120000b04e00013
:1088a00001003a008000eb0050da200050429000b6
:1088b000811f7800f7ff2c0006c3b3008041eb0056
:1088c0000482fb000500200022c0b3000800be00a7
:1088d0003cfe07000080fb00000444008002eb0027
:1088e000f4ff2c0085417800e2c2b3000800be000e
:1088f0009ffb07000080fb00000444008f87e90015
:10890000e44f550003003a00f10120000b04e000a1
:1089100001003a008000eb0050da20006042900035
:108920000482fb00007d200000024200811f7800cd
:10893000f7ff2c0006c3b3008041eb00cfa2de009e
:1089400042c0b3000800be001efe07008f87e9008a
:108950004f05be004f04be0000000600889fbe0009
:108960008a9fbe008c9fbe000004780081067800bc
:108970008245780003467800040578000204e00090
:108980000d0032008044eb008a0278000a02780071
:108990008c41780002c2b3008d0078000800780096
:1089a00073fb07000080fb00000444008944e800da
:1089b00089cf5500f4ff3a004f06be004f05be00b8
:1089c0004f04be0000000600889fbe008a1f78008a
:1089d0000004eb00880478004a3e290004003700b8
:1089e000ea0f5400020036008904e8000004eb009e
:1089f0006b48b900000044000000400060017d00a9
:108a0000d00f20000800400004142000044ab800e1
:108a100000004200e0804a00048021001500200090
:108a20000000420081804a00f9fa07000804e800cb
:108a3000ef8f5400eaff36004f0578004f04be0068
:108a4000000006008000780002802f00f04a20001d
:108a5000808f500012003e0070252000808f500053
:108a60000900360080da2f0000804000420120001b
:108a7000110009000280d8007f00100001802f0043
:108a800001017000060037004201200011000900ba
:108a90008280d800000178004b11dd00f201b300a4
:108aa0000200780000000600889fbe008a9fbe007a
:108ab000c8822000aad920001a80fb0000004000d4
:108ac0006400400060017c008002eb00f457280045
:108ad00013c0b300010e20000500780014fc07004d
:108ae000b9ff07001a80fb00000040004002b00000
:108af00060017c00e5382700f4ff2c008041eb008a
:108b00008000eb000100780009fc07005093800012
:108b10006104b800cbff0700801f7800f7ff2c002e
:108b200006c2b30023c0b3000802be0042c0b300b7
:108b30006109200000022000a2fd07008002eb0076
:108b4000f4ff2c0023c0b300a2c3b30061092000ce
:108b5000000a200006fb07008002eb00f4ff2c0057
:108b600023c0b300b2c3b30061092000000c200091
:108b7000fffa0700c8da20008041eb0018417800b6
:108b80000106200080052000cffe07008041eb0099
:108b90001841780001042000d00420001bff0700ca
:108ba000106c80000b0220008f87e9000058a300a2
:108bb0002b003200688c20001a80fb00000040006f
:108bc000800ab00060017c008002eb00f4ff2c0002
:108bd000854178008b00780070032000d4fb0700eb
:108be0001a80fb0000004000000bb00060017c0018
:108bf0008002eb00f4ff2c00854178000101200089
:108c000070032000cafb0700800478000004eb001a
:108c1000881f7800f7ff2c000b437800884178000c
:108c2000e46e80000500200032c0b3000101200086
:108c300064fd0700e24580000080fb008084440062
:108c400088027800f4ff2c008841780001012000a0
:108c500009007800b6fb07008f87e9003c00370069
:108c60000068a3002c003200698c2000a8d92000e5
:108c70001880fb0000004000c00ab00060817c004a
:108c80008002eb00f4ff2c008541780001022000f7
:108c900070032000a6fb07001880fb0000004000c6
:108ca000000bb00060817c008002eb00f4ff2c0020
:108cb0008541780001012000700320009cfb070023
:108cc000800478000004eb00881f7800f7ff2c0078
:108cd00006c2b30088417800e46e800005002000e1
:108ce00032c0b3000101200036fd0700e2458000dc
:108cf0000080fb008084440088027800f4ff2c0090
:108d000088417800010120000900780088fb0700f5
:108d10008f87e9000e0037008002eb00f4ff2c0083
:108d20008541780042c1b3000102200060012000ab
:108d30000aff07008002eb00f4ff2c008541780059
:108d400042c1b300010120006001200003ff0700c1
:108d500073c0b30052c0b30061c0b3000040eb0069
:108d600015fe07004f05be004f04be0000000600c0
:108d7000889fbe008a9fbe008c9fbe008e1f780019
:108d8000006c80000a0420000a007000006c88005b
:108d9000a0d920001080fb000000400064004000cb
:108da000c1822000608178008002eb00f457280027
:108db00013c0b300010e2000050078005cfb070023
:108dc00001ff0700e09680006104b8001dff070066
:108dd000801f7800f7ff2c0006c2b30023c0b30049
:108de0000802be0042c0b30061092000000220005a
:108df000f4fc07008002eb00f4ff2c0023c0b3005a
:108e0000a2c3b30061092000000a200058fa07003d
:108e10008002eb00f4ff2c0023c0b300b2c3b30008
:108e200061092000000c200051fa0700c8da200078
:108e30008041eb00184178000106200080052000e9
:108e400021fe07008041eb00184178008a0078007d
:108e5000d00420006dfe07000007eb008cb82b004b
:108e60000d0020008f87e9000e007800f5fe070056
:108e7000800578000c04be008a0020000b017800f9
:108e80000800be00e2f907000a05e800610444009a
:108e9000e0844c00ec0f5500f8ff3a007e074700d5
:108ea0000c14b0000d80b000e04c2000800f570083
:108eb0003a003200ecff37007e60b900e1fe0700a7
:108ec00080057800001420000060b800d2b82b00a4
:108ed000030020000004410081844900ba00200002
:108ee0000b0178000800be00c9f907000a05e90077
:108ef00061044400e0844c000a00e000f8ff3a00fe
:108f00000c06e800e0968000e20120001100090054
:108f10000280d800800f5600e7ff39008002200051
:108f2000800f560013003e00001420000060b800bf
:108f3000d2b82b00030020000004410081844900c6
:108f4000ba002000f2ff2c000800be00b0f90700b4
:108f50000a05e90061044400e0844c000a00e000d6
:108f6000f8ff3a000c06e80090022000800f56003f
:108f7000edff3a0043c0b30052c0b30061c0b3007c
:108f8000c0c0b3008cfd07004f0778004f06be003d
:108f90004f05be004f04be0000000600e0968000b2
:108fa000e2012000110009000280d8008000fd00cd
:108fb0000006eb000100e000bfff3a000106780068
:108fc000d9ff3700a3002000c203200083007800ef
:108fd00003007800d3fc070063042000030178003d
:108fe000a1002000c0032000cefc07006304200085
:108ff000e20620008300780003007800c9fc070027
:10900000230820008207200061042000e0062000e1
:10901000c4fc070023082000020a20008300780017
:1090200080072000bffc0700830c2000020f2000f7
:1090300021082000000a2000bafc0700830c200051
:109040002212200083007800000f2000b5fc0700ea
:10905000030a200062132000810c2000201220004f
:10906000b0fc070000000600881f7800a8d9200087
:109070001880fb0000004000c18220006081780061
:109080008002eb00f457280013c0b300010e20004b
:1090900005007800a6fa07004bfe07001880fb00c9
:1090a0000000400001802000608178008002eb0019
:1090b000f4ff2c0085417800010d200005007800a8
:1090c0009bfa07001880fb0070004000213a29003d
:1090d00060c17800510520000000eb00de8d020029
:1090e0000000000051002000f00520002a8e020040
:1090f0000000000043c0b3000341780083407800c3
:10910000c0c0b3002cfd07004f047800000006002b
:10911000f0da20001080fb0000004000a1d9200000
:109120009180fb00010040000000400041802000d1
:10913000608178008002eb00f4ff2c00854178000c
:10914000010c20000500780079fa070043c0b30045
:109150000341780083407800c0c0b30016fd0700cb
:1091600000000600a0d920001080fb000000400095
:10917000618c2000608178008002eb00f4ff2c00fd
:109180008541780061092000b000200068fa0700de
:1091900043c0b3000341780083407800c0c0b300ef
:1091a00005fd070000000600a0d920001080fb008c
:1091b0000000400064004000618c20006081780065
:1091c0008002eb00f4ff2c0085417800610920004b
:1091d0001002200056fa070043c0b3000341780094
:1091e00083407800c0c0b300f3fc07000000060015
:1091f000889fbe008a1f78008004780001057800ef
:10920000e125210000c6b300914f10000800320094
:109210008002eb00f4ff2c0085417800a2c2b3006d
:109220008a0078000900780051f90700070037002c
:109230008002eb00f4ff2c008541780002c2b300ed
:109240008a0078000900780049f9070092458000fb
:109250006b8044008002eb00f4ff2c008541780015
:109260008a00780032fa0700c026210010427800f8
:1092700070032000090040000004eb00881f780004
:10928000f7ff2c0006c2b300884178000482fb007f
:109290000500200022c0b3008a007800c9fb070047
:1092a000d00420000900400088027800f4ff2c0060
:1092b0008841780052c2b3008a0078002cf9070078
:1092c0008f87e9004f0578004f04be0000000600bc
:1092d000889fbe008a9fbe008c1f78000105780021
:1092e00002067800eb3827000304e00001003a0092
:1092f0008005eb008b027800f4ff2c008041eb002e
:10930000624580008a00780009fa070000047800ae
:109310008004eb00891f7800f7ff2c0006c2b30021
:10932000894178006162b80042c0b3008a007800c9
:10933000a4fb0700e24580000080fb00000444001d
:109340008b027800f4ff2c00894178008a007800b5
:1093500008007800f6f907008f87e9004f067800cb
:109360004f05be004f04be0000000600889fbe00ef
:109370008a9fbe008c9fbe00002d21001041780006
:109380000281fb000300200000c028000010b8008c
:109390004211dd0081004100206f8800316f88009c
:1093a00026890200000000006066b800606c800042
:1093b0000068a300fdff3200606c80000060a10027
:1093c000606c88000c00be00ea7b24000b80240047
:1093d0003a01780061044000e08448008cf80700fe
:1093e0008b0f5500020032000800be00f8ff370066
:1093f00081e3a8008de3a8008fe3a80083e3a80021
:109400001c02b0000d80b000f0bf2200110020004f
:10941000800f5400818f5c00e4ff360081e3a900d7
:109420008de3a900606c80000010a100606c8800d2
:10943000e922a8004f06be004f05be004f04be0043
:1094400000000600889fbe008a9fbe008c9fbe0061
:109450008e1f7800a0d920001080fb000000400083
:109460007c004000c1822000608178008002eb0017
:10947000f457280013c0b300010e20000500780047
:10948000abf9070050fd07008040eb00c02521002c
:1094900001487800a0042100e212210013c0b300ab
:1094a00090cf110003003a00c02521000148780048
:1094b000060037008140e80073004000800f510033
:1094c000f6ff3a00c025210001487800c0252100a0
:1094d0001004e000460032008046eb00ae0421009c
:1094e00080de200030409000fc01200080cf56003c
:1094f00001003200ec3827000d80fb004400dd0045
:10950000010c2000008550008c027800f4ff2c0034
:109510008041eb0002c2b3008a0078000000eb003b
:1095200093f80700804478001e4178000204e000b0
:10953000230032000e0478008045eb00e14f41002b
:10954000020032008045eb00030037008b45e80045
:10955000e3cf55000d003e000804e8000980fb0041
:109560008c027800f4ff2c008041eb008a00780028
:109570007ff8070080c44400184178000204e0002e
:10958000eeff3a00e3cf55000d003600a0d92000d1
:109590001080fb0000004000c004b000618c20007f
:1095a000608178008c027800f4ff2c008041eb0091
:1095b000010d20000000eb005df9070011003700ed
:1095c0000980fb008c027800f4ff2c008041eb0046
:1095d00002c2b3008a00780065f8070073074700ed
:1095e0008d46e800c025210090cf5600bcff390011
:1095f00093c0b30052c0b30061c0b300c0c0b30099
:10960000edfb07004f0778004f06be004f05be0078
:109610004f04be0000000600889fbe008a9fbe0067
:109620008c9fbe008e1f7800a0d920001080fb0008
:10963000000040000002b000c1822000608178007c
:109640008002eb00f457280013c0b300010e200085
:109650000500780036f90700dbfc07008040eb00ce
:10966000d025210001487800a0042100e212210049
:1096700013c0b30090cf11000b0032008140e8000e
:1096800073004000800f5100f9ff3a00d0252100ff
:1096900001487800a004210011c0b30090cf100051
:1096a00050003a0053003700d025210001487800cf
:1096b000f8ff37008046eb00ae04210080de20007a
:1096c00040409000fc01200080cf56000100320095
:1096d000ec3827000d80fb004400dd00010c200069
:1096e000008550008c027800f4ff2c008041eb00d4
:1096f00002c2b3008a0078000000eb001cf80700eb
:10970000804478001e4178000204e000230032000b
:109710000e0478008045eb00e14f4100020032006a
:109720008045eb00030037008b45e800e3cf550090
:109730000d003e000804e8000980fb008c02780060
:10974000f4ff2c008041eb008a00780008f8070045
:1097500080c44400184178000204e000eeff3a00a3
:10976000e3cf55000d003600a0d920001080fb008b
:1097700000004000c004b000618c200060817800cf
:109780008c027800f4ff2c008041eb00010c2000db
:109790000000eb00e6f80700160037000980fb0028
:1097a0008c027800f4ff2c008041eb0002c2b30071
:1097b0008a007800eef707008d46e800730747003f
:1097c000d025210090cf5600bcff390043c0b30024
:1097d00052c0b30061c0b300c0c0b30076fb070045
:1097e00004003700d02521001004e000b1ff3a004a
:1097f000f6ff37004f0778004f06be004f05be004a
:109800004f04be0000000600e4874700889fbe00aa
:109810008a9fbe008c9fbe008e1f78008006eb00e2
:109820000a0c2000b055290080bf9f005e5429001b
:10983000006c80000004b20002003a008002780050
:1098400005003700f5012000522d210092cf1600af
:1098500001003200e53827000d804600a2d9200023
:109860009280fb000100400000004000a1ba2000ef
:1098700060817800f4ff2c008041eb008a007800c2
:109880000000eb00aaf80700512d21001180fb0019
:1098900000014000602d21009040780044542900d0
:1098a0000180fb000000410060407a00432d210050
:1098b00080497800f44f50000500360001407800e0
:1098c0000004a2000080fb0000004100e0497a0093
:1098d0008e0478007ef99700006c80000004b200ce
:1098e00002003a000004780005003700f80120006b
:1098f000402d2100904f510001003200e838270030
:10990000fd4f51002d003e00f24f51000c003a0077
:10991000c194800020948000808f500008003100a6
:10992000b245800088027800f4ff2c008041eb00f3
:109930008a007800300620007df8070026003700f6
:109940000280fb00000040004227210060027900f5
:10995000881f7800f7ff2c0006c2b3008041eb009f
:109960000500200042c0b3008a00780030062000c5
:1099700014fa0700ffb0970071f897000080fb0011
:1099800000004000a2d920009280fb0001004000ae
:1099900000004000e1bd200060817800880278006e
:1099a000f4ff2c008041eb008a007800f0082000d2
:1099b0005ff807008f87e900070037008002eb009f
:1099c000f4ff2c008541780062c0b3008a00780063
:1099d00030062000e1fb070019447800006c80008d
:1099e0000004b20002003a000006780005003700cb
:1099f000fc012000402d2100904f54000100320056
:109a0000ec382700fd4f540004013e00eb4f54009a
:109a10000c003a0051948000c0082000808f500054
:109a20008f003a00c24580008c027800f4ff2c00c1
:109a30008041eb008a007800790040003cf8070084
:109a400095003700f34f540083003a00d99480000a
:109a5000c0948000808f540013003e0040272100f6
:109a6000806d90000b04e0000f003a00b2458000ca
:109a70008c027800f4ff2c008b4178008a0078007b
:109a8000500a20002af807008002eb00f4ff2c00a7
:109a90008b41780022c0b3008a007800100d2000ae
:109aa000aefb07007c0037000900e00013003a001d
:109ab00041272100016890000004e0000f003200ff
:109ac000b24580008c027800f4ff2c0089417800b8
:109ad0008a007800500a200015f8070089027800f3
:109ae000f4ff2c008941780022c0b3008a0078007e
:109af000100d200099fb0700670037004227210066
:109b000002689000e14f500047003a00006c80006e
:109b10000004b20002003a00800078000c00370018
:109b2000a1c0b300502d210090cf100007003a00d3
:109b3000602d21001004e00004003200f10120003b
:109b4000702d21001004e00001003200e1382700f0
:109b5000c4032000811f7800110009008484d8000c
:109b600000027800cf007800811f7800f7ff2c00fa
:109b700006c2b3008041eb000500200022c0b30004
:109b80008a007800500a20008ef907008002eb005e
:109b9000f4ff2c0085417800a2c3b3008a0078004e
:109ba000b00b2000f2f60700006c80000004b20049
:109bb0008f87e9000000e00002003a00000678000c
:109bc00009003700a0c0b300522d2100924f1000b1
:109bd00004003a00fc012000702d21001004e00078
:109be00001003a00ec382700d0948000c203200026
:109bf000110009000280d800010278008c1f780053
:109c0000f7ff2c0006c3b3008041eb0005002000e5
:109c100022c0b3008a007800600c200069f90700b8
:109c20008f87e9001c0037008c1f7800f7ff2c009d
:109c300006c2b3008041eb00d494800005002000f0
:109c400042c0b3008a007800500a20005df9070086
:109c50008f87e90010003700ec4f540002013200fa
:109c60000880fb000000400041272100608278004e
:109c70008c1f7800f7ff2c0006c2b3008041eb0078
:109c80000500200042c0b3008a007800500a20007e
:109c90004cf907008f87e9004027210000699000f8
:109ca000e14f510045003a004100370062c0b30067
:109cb000512d2100914f110004003a00f1012000c4
:109cc000602d21001004e00001003200e13827007f
:109cd00064948000c2032000811f780011000900f5
:109ce0000282d80000027800cf007800811f78003f
:109cf000f7ff2c0006c2b3008041eb0005002000f6
:109d000022c0b3008a007800500a20002df9070015
:109d10008002eb00f4ff2c0085417800a2c3b30061
:109d20008a007800b00b200091f60700006c8000dc
:109d30000004b2008f87e9000000e00002003a0052
:109d4000800078000900370061c0b300502d210069
:109d500090cf100004003a00f1012000602d210096
:109d60001004e00001003a00e13827006094800010
:109d7000c203200001027800110009000280d8000f
:109d80000102fd00811f7800f7ff2c0006c3b3001d
:109d90008041eb000500200022c0b3008a0078005b
:109da000600c200007f907008f87e90022003700c8
:109db000f34f540009003a001f003700f34f5400de
:109dc00006003a00d1948000c0948000808f50003b
:109dd00002003e000204e000170032000fb99700b5
:109de0001280fb0000004000a2d920009280fb00fe
:109df0000100400000004000e1bd200060817800cb
:109e00008c027800f4ff2c008041eb008a0078007f
:109e1000100d200046f70700070037008002eb0016
:109e2000f4ff2c008541780062c0b3008a007800fe
:109e3000a0092000c9fa07008d06e800700555004a
:109e40000fb897000080e80080bf9f000e87e800f1
:109e5000eb8f560076fe3a00416f8000c012200062
:109e6000808f50000e003a00a1d920001180fb0025
:109e700000004000780040004185200060817800ab
:109e80008002eb00f457280013c0b300010e20003d
:109e90000500780026f70700cbfa070063003700bb
:109ea000d0122000808f50000e003a00a2d920006e
:109eb0001280fb00000040006400400061aa200006
:109ec000608178008002eb00f457280013c0b300d3
:109ed000010e20000500780015f70700bafa070008
:109ee0005200370080de20004040900032c1b300b5
:109ef0000440bc00a0042100000441001841780087
:109f00008004eb000204e00011003a001d0037005d
:109f100090072000808f54000d0036008002eb0077
:109f2000f457280013c0b300e2c2b300010e2000b2
:109f3000090078000ef607000080fb0080844400d2
:109f4000e0082000808f54001b003e000e00370008
:109f50000804e8008002eb00f457280013c0b300a7
:109f6000010e20000900780001f607000080fb00c8
:109f700080844400184178000204e000e4ff3a00c5
:109f8000efff37008004eb008002eb00f45728005d
:109f900013c0b30002c2b300010e20000900780014
:109fa000f3f507000080fb0080844400e0082000f7
:109fb000808f5400f4ff3600006c80000068a3001e
:109fc0000d003200a1d920001180fb0000004000ec
:109fd000400ab000618c2000608178008002eb00b4
:109fe000f457280013c0b300010e200009007800c8
:109ff000cff607000c003700a2d920001280fb002a
:10a0000000004000000ab000618c200060817800f0
:10a010008002eb00f457280013c0b300010e2000ab
:10a0200009007800c2f6070067fa0700006c80009c
:10a030000068a3000600320083c0b300a2c0b300d2
:10a04000b1c0b300c0c0b3005bf907000b0037001c
:10a0500083c0b30042c0b30031c0b300c0c0b3007e
:10a0600055f9070005003700006c80000004b200bd
:10a070000eff3a008000780015ff37004f07780088
:10a080004f06be004f05be004f04be004f00b1009a
:10a0900000000600d0262100904078000148a3006f
:10a0a00004003200106c80000000a000106c8800da
:10a0b00003003700106c80000000a100106c8800c5
:10a0c0000104e00004003d00106c80000010a000be
:10a0d000106c880003003700106c80000010a10095
:10a0e000106c880000000600889fbe008a9fbe009a
:10a0f0008c1f780000042100104078007f4660002b
:10a10000e34f560008003200e64f560006003200ca
:10a11000e94f560004003200ec4f560002003200b6
:10a12000ef4f56000a003a00929380000280e80048
:10a1300051938000810f5000060039000280e90031
:10a14000808f5000030039000100780001003700c3
:10a15000509380006104b8003afa0700801f78002d
:10a16000f7ff2c0006c2b30023c0b3000802be00f4
:10a1700042c0b300610920000002200011f807006e
:10a180008002eb00f4ff2c0023c0b300a2c3b30095
:10a1900061092000000a200075f507008002eb002d
:10a1a000f4ff2c0023c0b300b2c3b3006109200048
:10a1b000000c20006ef50700416f80008f87e900da
:10a1c000c0122000808f50000d003a00a0d920005e
:10a1d0001080fb0000004000c008b000618c20002f
:10a1e000608178008002eb00f457280013c0b300b0
:10a1f000010e2000050078004df6070045003700ed
:10a20000d0122000808f50000d003a00a0d920000d
:10a210001080fb00000040006c00400021ab2000db
:10a22000608178008002eb00f457280013c0b3006f
:10a23000010e2000050078003df6070035003700cc
:10a2400080de20004040900032c1b3000440bc00da
:10a25000a004210000044100184178008004eb00b4
:10a260000204e00011003a001d00370090072000b2
:10a27000808f54000d0036008002eb00f457280058
:10a2800013c0b300e2c2b300010e20000900780041
:10a2900037f507000080fb0080844400e0082000c0
:10a2a000808f54001b003e000e0037000804e800b9
:10a2b0008002eb00f457280013c0b300010e200009
:10a2c000090078002af507000080fb008084440024
:10a2d000184178000204e000e4ff3a00efff370085
:10a2e0008004eb008002eb00f457280013c0b30099
:10a2f00002c2b300010e2000090078001cf507001f
:10a300000080fb0080844400e0082000808f54001f
:10a31000f4ff3600acf90700e14f56001700320099
:10a32000e34f560015003200e44f56001300320090
:10a33000e64f560011003200e74f56000f00320082
:10a34000e94f56000d003200ec4f56000b00320072
:10a35000ee4f560009003200ef4f56000700320062
:10a36000f24f5600050032008026210011c0b300d4
:10a3700090cf100029003a00040037008026210009
:10a3800011c0b30090cf100002003a00309380005b
:10a390000100370090958000c403200011000900df
:10a3a0000480d80000027800810478000004eb00eb
:10a3b000881f7800f7ff2c0006c3b300884178009f
:10a3c0000500200022c0b30001082000b0002000da
:10a3d0007cf7070088027800f4ff2c0088417800a1
:10a3e000a2c3b3000108200010022000e0f407001f
:10a3f000881f7800f7ff2c0006c3b300884178005f
:10a40000614ab80022c0b30001082000c002200049
:10a410006cf70700e4875700070037008002eb0065
:10a42000f4ff2c008541780052c0b30001082000e1
:10a43000b000200049f9070001082000f0082000c2
:10a440006bfb0700006c800000d8a30011003200f5
:10a4500082de2000c0122000920f1000c7053a00d3
:10a46000e24090005240900080cf5000c30532007f
:10a470008002eb00f457280013c0b30092c0b30071
:10a48000010e2000f008200034f907004ef9070003
:10a49000230037000c80fb0000004000a1d9200001
:10a4a0009180fb000100400000004000e1cf20004f
:10a4b000608178008002eb00f457280013c8b300d5
:10a4c000010e2000f008200099f507003ef9070072
:10a4d00090262100e1c1b30090cf100003003a00a4
:10a4e000f06b80000010a000f06b8800e9fe070010
:10a4f000106c80000008a30002003a000018a300be
:10a50000070032000048a30005003a000040a00008
:10a51000106c8800006c80000090a000006c880027
:10a52000006c800000d8a3006600320081de2000ad
:10a53000d0122000910f100056003a00a0d9200040
:10a540001080fb00000040004006b000618c20003d
:10a55000608178008002eb00f4ff2c0085417800d8
:10a56000010620006001200071f5070012468000fe
:10a570008002eb00f4ff2c008541780001052000eb
:10a58000700320006af50700e24580008002eb00be
:10a59000f4ff2c008541780001052000f008200020
:10a5a00063f50700e16d8000f06d8000808f500042
:10a5b00005003100010050000000d100c012b000c1
:10a5c000c096880005003700808050008100d100cf
:10a5d000c012200001005000c0968800c196800083
:10a5e000b0122000808f500015003e008002eb006a
:10a5f000f4ff2c0085417800d2c2b3000105200091
:10a60000300620005af40700c4122000c0968000d3
:10a61000000252008001eb00831f7800f7ff2c003e
:10a6200006c2b3000500200032c0b30001052000bf
:10a63000e0062000e3f607008f87e90036053700c3
:10a640008002eb00f4ff2c008541780002c2b300c9
:10a65000010520003006200045f40700c496800064
:10a6600040ed2f00000242008001eb00831f7800c4
:10a67000f7ff2c0006c2b3000500200032c0b30073
:10a6800001052000e0062000cef607008f87e900d4
:10a6900021053700c8da20008041eb00184178001e
:10a6a000010620008005200007f807008041eb002c
:10a6b0001841780001042000d004200053f807005e
:10a6c000150537008bde2000c01220009b0f100004
:10a6d0002e003a006a8c2000a9d920001980fb00c6
:10a6e000000040008007b00060017d008002eb00a8
:10a6f000f4ff2c0085417800010d2000b0002000ff
:10a700000bf507006b4290000004eb00881f7800f7
:10a71000f7ff2c0006c2b300884178000482fb00da
:10a720000500200022c0b300010d2000d00420004d
:10a73000a4f607001980fb0000004000c006b0002e
:10a7400060017d0088027800f4ff2c0088417800c9
:10a75000010d2000f0082000f5f407005b42900096
:10a76000881f7800f7ff2c0006c2b30088417800ec
:10a770000482fb000500200022c0b300010d200070
:10a78000000b20008ff60700e4875700006c800064
:10a790000098a3005d003200688c2000a9d9200039
:10a7a0001980fb00000040006800400060017c0050
:10a7b0008002eb00f4ff2c008541780001022000ac
:10a7c00060012000daf407001980fb00000040005f
:10a7d0006c00400060017c008002eb00f4ff2c0064
:10a7e0008541780001012000c0022000d0f407005c
:10a7f000126c80000208a3002f003200d022a800b3
:10a8000090d7200011c0b3000148780031c0b300d8
:10a81000014878000228a3000c0032001980fb00d8
:10a82000000040000005b000219f200060817800fa
:10a830008002eb00f4ff2c0003c8b30001072000e6
:10a8400005007800baf40700b30437000238a3000b
:10a850000d003200a0d920001080fb000000400055
:10a860004002b000219f2000608178008002eb0050
:10a87000f4ff2c0003c8b300010720000500780096
:10a88000abf40700a4043700c126210090c5b30033
:10a89000914f100004003600020078000020a00054
:10a8a000106c88009c043700020078000030a00083
:10a8b000106c8800980437000218a3009604320038
:10a8c000d022a80091d7200010c0b30080487800a3
:10a8d00030c0b30080487800a0d920001080fb0071
:10a8e000000040008002b000219f200060817800bd
:10a8f0008002eb00f4ff2c0003c8b3000107200026
:10a90000050078008af40700830437008002eb001a
:10a91000f4ff2c008541780042c1b3000102200001
:10a92000600120000df807008002eb00f4ff2c000e
:10a930008541780042c1b300010120006001200080
:10a9400006f807008026210011c0b30090cf100048
:10a950000d003a00a0d920001080fb00000040004c
:10a960004005b000618c2000608178008002eb001f
:10a97000f4ff2c008541780001032000c002200074
:10a980006bf40700240037006b8c2000aad920004c
:10a990001a80fb00000040008005b00060817d004f
:10a9a0008002eb00f4ff2c008541780001032000b9
:10a9b000c00220005ef40700800478000004eb0071
:10a9c000881f7800f7ff2c0006c2b300884178008a
:10a9d000448280000500200032c0b3000103200043
:10a9e000f8f507009a80fb0081804000c105b000a7
:10a9f00061817d000080fb00808444008802780033
:10aa0000f4ff2c0088417800010320000900780041
:10aa100047f407008f87e9000c80fb00010020004d
:10aa2000f20f5000e08f580081033e0000600100eb
:10aa30001200370011003700540037005300370070
:10aa40009a003700df003700de00370025013700ad
:10aa50006a01370069013700b0013700f50137009e
:10aa6000440237009a02370099023700e0023700ab
:10aa7000270337002603370025033700ead42000d8
:10aa8000a9d920001980fb000000400060017d0072
:10aa90008002eb00f4ff2c008541780001072000c4
:10aaa000b000200022f407000004eb00881f7800ab
:10aab000f7ff2c0006c2b300884178006022b8007e
:10aac00042c0b30001072000a0092000bdf5070027
:10aad0001980fb0000004000e1bd2000608178008b
:10aae00088027800f4ff2c008841780001072000dc
:10aaf000600c20000ef407001980fb0000004000ed
:10ab00006800400060017d0088027800f4ff2c009e
:10ab10008841780001062000b000200004f40700fe
:10ab2000881f7800f7ff2c0006c3b3008841780027
:10ab30006022b80022c0b30001062000a009200056
:10ab4000a0f5070088027800f4ff2c008841780007
:10ab5000a2c3b30001062000000b200004f307008d
:10ab6000881f7800f7ff2c0006c3b30088417800e7
:10ab70006022b80022c0b30001062000b00b200004
:10ab800090f50700e687570045033700ead4200018
:10ab9000a9d920001980fb0000004000640040009b
:10aba00060017d008002eb00f4ff2c0085417800fd
:10abb00001072000b0002000ddf307000004eb00d7
:10abc000881f7800f7ff2c0006c2b3008841780088
:10abd000a49380000500200042c0b30001072000bc
:10abe000a009200077f507001980fb000000400055
:10abf00068004000e1bd2000608178008802780094
:10ac0000f4ff2c008841780001072000600c200030
:10ac1000c7f307001980fb000000400068004000f7
:10ac200060017d0088027800f4ff2c0088417800e4
:10ac300001062000b0002000bdf30700881f780047
:10ac4000f7ff2c0006c3b30088417800b49380005e
:10ac50000500200022c0b30001062000a00920004a
:10ac600058f5070088027800f4ff2c00884178002e
:10ac7000a2c3b30001062000000b2000bcf20700b5
:10ac8000881f7800f7ff2c0006c3b30088417800c6
:10ac90006022b80022c0b30001062000b00b2000e3
:10aca00048f50700e6875700fd023700ead4200088
:10acb000a9d920001980fb000000400060017d0040
:10acc0008002eb00f4ff2c00854178000107200092
:10acd000b000200096f307000004eb00881f780006
:10ace000f7ff2c0006c2b30088417800c4938000af
:10acf0000500200042c0b30001072000a009200089
:10ad000030f507001980fb0000004000e1bd200085
:10ad10006081780088027800f4ff2c008841780078
:10ad200001072000600c200081f307001980fb0060
:10ad3000000040006800400060017d00880278004b
:10ad4000f4ff2c008841780001062000b0002000ac
:10ad500077f30700881f7800f7ff2c0006c3b300c5
:10ad600088417800d49380000500200022c0b30001
:10ad700001062000a009200012f5070088027800d3
:10ad8000f4ff2c0088417800a2c3b3000106200024
:10ad9000000b200076f20700881f7800f7ff2c00d8
:10ada00006c3b300884178006022b80022c0b30017
:10adb00001062000b00b200002f50700e6875700cf
:10adc000b9023700ead42000a9d920001980fb007d
:10add000000040006400400060017d008002eb0044
:10ade000f4ff2c008541780001072000b00020000e
:10adf0004ff307000004eb00881f7800f7ff2c00da
:10ae000006c2b30088417800e4938000050020006a
:10ae100042c0b30001072000a0092000e9f40700a8
:10ae20001980fb000000400068004000e1bd2000e8
:10ae30006081780088027800f4ff2c008841780057
:10ae400001072000600c200039f307001980fb0087
:10ae5000000040006800400060017d00880278002a
:10ae6000f4ff2c008841780001062000b00020008b
:10ae70002ff30700881f7800f7ff2c0006c3b300ec
:10ae800088417800f49380000500200022c0b300c0
:10ae900001062000a0092000caf4070088027800fb
:10aea000f4ff2c0088417800a2c3b3000106200003
:10aeb000000b20002ef20700881f7800f7ff2c00ff
:10aec00006c3b300884178006022b80022c0b300f6
:10aed00001062000b00b2000baf40700e6875700f7
:10aee0006f023700ead42000a9d920001980fb00a6
:10aef0000000400060017d008002eb00f4ff2c00a8
:10af00008541780001072000b000200008f3070009
:10af10000004eb00881f7800f7ff2c0006c2b30086
:10af200088417800049480000500200042c0b300ee
:10af300001072000a0092000a2f407001980fb00ef
:10af400000004000e1bd20006081780088027800a8
:10af5000f4ff2c008841780001072000600c2000dd
:10af6000f3f207001980fb00000040006800400079
:10af700060017d0088027800f4ff2c008841780091
:10af800001062000b0002000e9f20700881f7800c9
:10af9000f7ff2c0006c3b3008841780014948000aa
:10afa0000500200022c0b30001062000a0092000f7
:10afb00084f4070088027800f4ff2c0088417800b0
:10afc000a2c3b30001062000000b2000e8f1070037
:10afd000881f7800f7ff2c0006c3b3008841780073
:10afe0006022b80022c0b30001062000b00b200090
:10aff00074f40700e68757002b023700ead42000dc
:10b00000a9d920001980fb00000040006400400026
:10b0100060017d008002eb00f4ff2c008541780088
:10b0200001072000b0002000c1f207000004eb007f
:10b03000881f7800f7ff2c0006c2b3008841780013
:10b04000249480000500200042c0b30001072000c6
:10b05000a00920005bf407001980fb0000004000fd
:10b0600068004000e1bd200060817800880278001f
:10b07000f4ff2c008841780001072000600c2000bc
:10b08000abf207001980fb000000400068004000a0
:10b0900060017d0088027800f4ff2c008841780070
:10b0a00001062000b0002000a1f20700881f7800f0
:10b0b000f7ff2c0006c3b300884178003494800069
:10b0c0000500200022c0b30001062000a0092000d6
:10b0d0003cf4070088027800f4ff2c0088417800d7
:10b0e000a2c3b30001062000000b2000a0f107005e
:10b0f000881f7800f7ff2c0006c3b3008841780052
:10b100006022b80022c0b30001062000b00b20006e
:10b110002cf40700e6875700e1013700ead420004d
:10b12000a9d920001980fb00000040006400400005
:10b1300060017d008002eb00f4ff2c008541780067
:10b1400001072000b000200079f207000004eb00a6
:10b15000881f7800f7ff2c0006c2b30088417800f2
:10b16000440620000500200042c0b3000107200073
:10b17000a009200013f407001980fb000000400024
:10b18000e1bd20006081780088027800f4ff2c0087
:10b190008841780001072000600c200064f207005d
:10b1a0001980fb00000040006800400060017d0045
:10b1b00088027800f4ff2c00884178000106200006
:10b1c000b00020005af20700881f7800f7ff2c001b
:10b1d00006c3b300884178006022b80022c0b300e3
:10b1e00001062000a0092000f6f30700880278007d
:10b1f000f4ff2c0088417800a2c3b30001062000b0
:10b20000000b20005af10700881f7800f7ff2c0080
:10b2100006c3b300884178006022b80022c0b300a2
:10b2200001062000b00b2000e6f30700e687570078
:10b230009d013700e9d42000a8d920001880fb0028
:10b24000000040006400400060817c008002eb0050
:10b25000f4ff2c008541780001072000b000200099
:10b2600033f207000005eb008a1f7800f7ff2c007f
:10b2700006c2b3008a417800449480000500200093
:10b2800042c0b30001072000a0092000cdf3070051
:10b290001880fb000000400068004000e1bd200075
:10b2a000608178008a027800f4ff2c008a417800df
:10b2b00001072000600c20001df207001880fb0031
:10b2c000000040007000400060817c008a0278002d
:10b2d000f4ff2c008a41780001062000b000200015
:10b2e00013f20700519480008f87e9004006200088
:10b2f000808f500008003600c24580008a02780026
:10b30000f4ff2c008a41780001062000a0092000eb
:10b3100007f207000a0037008001eb00831f780066
:10b32000f7ff2c0006c2b300610ab80042c0b300a8
:10b3300001062000a0092000a2f307008f87e90082
:10b34000a0d920001080fb00000040006c004000ed
:10b35000e1bd2000608178008002eb00f4ff2c004a
:10b360008541780001062000600c2000f0f1070004
:10b370004d013700ead42000a9d920001980fb0034
:10b38000000040006400400060017d008002eb008e
:10b39000f4ff2c008541780001072000b000200058
:10b3a000e3f107000004eb00881f7800f7ff2c0092
:10b3b00006c2b30088417800449480000500200054
:10b3c00042c0b30001072000a00920007df3070060
:10b3d0001980fb000000400068004000e1bd200033
:10b3e0006081780088027800f4ff2c0088417800a2
:10b3f00001072000600c2000cdf107001980fb0040
:10b40000000040006800400060017d008802780074
:10b41000f4ff2c008841780001062000b0002000d5
:10b42000c3f1070064948000c903200011000900e3
:10b430000982d80000027800881f7800f7ff2c00ee
:10b4400006c3b300884178000500200022c0b30085
:10b4500001062000a00920005af3070088027800a6
:10b46000f4ff2c0088417800a2c3b300010620003d
:10b47000000b2000bef0070060948000110009005e
:10b480000980d80001027800881f7800f7ff2c009f
:10b4900006c3b300884178000500200022c0b30035
:10b4a00001062000b00b200046f307008802780058
:10b4b000f4ff2c008841780002c2b300010620008e
:10b4c000100d2000aaf00700e6875700f6003700ad
:10b4d000ead42000a9d920001980fb000000400018
:10b4e0006400400060017d008002eb00f4ff2c004e
:10b4f0008541780001072000b00020008cf1070092
:10b500000004eb00881f7800f7ff2c0006c2b30090
:10b5100088417800749480000500200042c0b30088
:10b5200001072000a009200026f307001980fb0076
:10b530000000400068004000e1bd2000608178000c
:10b5400088027800f4ff2c00884178000107200071
:10b55000600c200076f107001980fb00000040001d
:10b560006800400060017d0088027800f4ff2c0034
:10b570008841780001062000b00020006cf107002f
:10b58000881f7800f7ff2c0006c3b30088417800bd
:10b59000849480000500200022c0b3000106200032
:10b5a000a009200007f3070088027800f4ff2c00b0
:10b5b00088417800a2c3b30001062000000b2000e0
:10b5c0006bf00700881f7800f7ff2c0006c3b3005c
:10b5d000884178006022b80022c0b3000106200034
:10b5e000b00b2000f7f20700e6875700ac003700e9
:10b5f000ead42000a9d920001980fb0000004000f7
:10b600006400400060017d008002eb00f4ff2c002c
:10b610008541780001072000b000200044f10700b8
:10b620000004eb00881f7800f7ff2c0006c2b3006f
:10b6300088417800749480000500200042c0b30067
:10b6400001072000a0092000def207001980fb009e
:10b650000000400068004000e1bd200060817800eb
:10b6600088027800f4ff2c00884178000107200050
:10b67000600c20002ef107001980fb000000400044
:10b680006800400060017d0088027800f4ff2c0013
:10b690008841780001062000b000200024f1070056
:10b6a000881f7800f7ff2c0006c3b300884178009c
:10b6b000949480000500200022c0b3000106200001
:10b6c000a0092000bff2070088027800f4ff2c00d8
:10b6d00088417800a2c3b30001062000000b2000bf
:10b6e00023f00700881f7800f7ff2c0006c3b30083
:10b6f000884178006022b80022c0b3000106200013
:10b70000b00b2000aff20700e6875700f4003700c7
:10b71000ead42000a9d920001980fb0000004000d5
:10b720006400400060017d008002eb00f4ff2c000b
:10b730008541780001072000b0002000fcf00700e0
:10b740000004eb00881f7800f7ff2c0006c2b3004e
:10b7500088417800a49480000500200042c0b30016
:10b7600001072000a009200096f207001980fb00c5
:10b770000000400068004000e1bd200060817800ca
:10b7800088027800f4ff2c0088417800010720002f
:10b79000600c2000e6f007001980fb00000040006c
:10b7a0006800400060017d0088027800f4ff2c00f2
:10b7b0008841780001062000b0002000dcf007007e
:10b7c000881f7800f7ff2c0006c3b300884178007b
:10b7d000b49480000500200022c0b30001062000c0
:10b7e000a009200077f2070088027800f4ff2c00ff
:10b7f00088417800a2c3b30001062000000b20009e
:10b80000dbef0700881f7800f7ff2c0006c3b300aa
:10b81000884178006022b80022c0b30001062000f1
:10b82000b00b200067f20700e68757001c003700c6
:10b830008002eb00f4ff2c008541780042c1b30088
:10b8400001072000b000200044f407008002eb0054
:10b85000f4ff2c008541780042c1b30001062000ae
:10b86000b00020003df407008002eb00f4ff2c0044
:10b870008541780042c1b30001052000b0002000de
:10b8800036f407008002eb00f4ff2c0085417800bd
:10b8900042c1b30001042000b00020002ff40700d3
:10b8a000ec4f56008e003e00c19480002094800032
:10b8b000808f500008003100b24580008002eb000c
:10b8c000f4ff2c008541780001052000a00920002c
:10b8d00097f007000a0037008001eb00831f780013
:10b8e000f7ff2c0006c2b300610ab80042c0b300e3
:10b8f00001052000a009200032f207008f87e9002f
:10b90000a0d920001080fb0000004000680040002b
:10b91000e1bd2000608178008002eb00f4ff2c0084
:10b920008541780001052000600c200080f00700b0
:10b9300040272100006890000004e0002f00320042
:10b94000d09480000000e00024003200c9032000f1
:10b95000110009000980d800000278000004eb0003
:10b96000881f7800f7ff2c0006c2b30088417800da
:10b970000500200022c0b30001042000a00920001f
:10b9800010f2070088027800f4ff2c00884178004c
:10b99000a2c3b30001042000000b200074ef0700d5
:10b9a000d0948000110009000980d80001027800bd
:10b9b000881f7800f7ff2c0006c3b3008841780089
:10b9c0000500200022c0b30001042000b00b2000bd
:10b9d000fcf10700e48757002a003700b2458000d9
:10b9e0008002eb00f4ff2c00854178000104200068
:10b9f000a00920004ef0070022003700d1948000fb
:10ba0000c0948000808f500008003e00b245800046
:10ba10008002eb00f4ff2c00854178000104200037
:10ba2000a009200042f007000a0037008001eb0067
:10ba3000831f7800f7ff2c0006c2b300610ab8002c
:10ba400042c0b30001042000a0092000ddf107007e
:10ba50008f87e900a0d920001080fb000000400083
:10ba600068004000e1bd2000608178008002eb00aa
:10ba7000f4ff2c008541780001042000600c2000b8
:10ba80002bf00700a9ba2000a8d920001880fb00dd
:10ba900000004000c002b00060817c008002eb002a
:10baa000f4ff2c0085417800010520000500780096
:10bab0001ff007001880fb00000040000003b000ea
:10bac00060817c008002eb00f4ff2c00854178004f
:10bad000010420000500780015f007000e00370073
:10bae0008002eb00f4ff2c008541780042c1b300d6
:10baf000010520000500780098f307008002eb00a4
:10bb0000f4ff2c008541780042c1b30001042000fd
:10bb10000500780091f30700006c800000d8a300b6
:10bb20001000320081de2000d0122000910f1000a2
:10bb300006003a0043c0b300a2c0b300b1c0b300d6
:10bb4000c0c0b3009cf207001900370043c0b30027
:10bb50000341780083407800c0c0b30096f207002c
:10bb60001300370083c0b30032c0b30011c0b3006c
:10bb7000c0c0b30090f207000d003700a0d920002c
:10bb80001080fb00000040000006b000618c200027
:10bb9000608178008002eb00f457280013c8b300de
:10bba000010e2000f0082000e1ef070037fa37000f
:10bbb0004f0678004f05be004f04be00000006008f
:10bbc000889fbe00a8d920001880fb00000040001c
:10bbd00078004000c1822000608178008002eb0084
:10bbe000f457280013c0b300010e200005007800b0
:10bbf000cfef070074f30700698c20001880fb006a
:10bc0000000040000005b00060817c008002eb0075
:10bc1000f4ff2c00854178006109200060012000bc
:10bc2000c3ef07001880fb00000040006c004000dc
:10bc300060817c008002eb00f4ff2c0085417800dd
:10bc40006106200010022000b9ef070043c0b300d6
:10bc50000341780083407800c0c0b30056f207006b
:10bc60004f04be0000000600881f7800a8d92000fd
:10bc70001880fb000000400068004000c1822000e6
:10bc8000608178008002eb00f457280013c0b300f5
:10bc9000010e200005007800a5ef07004af3070019
:10bca0001880fb00000040004005b000219f2000ec
:10bcb000608178008002eb00f4ff2c008541780061
:10bcc000010d20000500780099ef070043c0b30084
:10bcd0000341780083407800c0c0b30036f207000b
:10bce0004f04780000000600889fbe008a9fbe00b7
:10bcf000e8d62000f02521001080fb000000400065
:10bd0000a9d920009980fb000100400000004000fc
:10bd10000800400040a197008002eb00f457280083
:10bd200013c0b300010e20000500780080ef07006b
:10bd300025f307001980fb000000400060017c0033
:10bd40008002eb00f4ff2c0085417800010d2000fb
:10bd50000500780076ef07006a8c20001980fb0050
:10bd6000000040004008b00060017d008002eb0050
:10bd7000f4ff2c00854178000103200005007800c5
:10bd80006bef07001980fb0000004000c007b00007
:10bd900060017d008002eb00f4ff2c0085417800fb
:10bda000010220000500780061ef0700800578009f
:10bdb00000262100104278000004eb00881f780064
:10bdc000f7ff2c0006c2b300884178000482fb0014
:10bdd0000500200022c0b300010220000b00780003
:10bde000f8f007000080fb0080854500880278009d
:10bdf000f4ff2c0088417800e2c2b3000102200069
:10be00000b0078005aee070011262100114278003d
:10be10000080fb0000804500881f7800f7ff2c00a1
:10be200006c3b300884178000482fb0005002000af
:10be300022c0b30001022000e2f007001980fb00dd
:10be4000000040000008b00060017d00880278001a
:10be5000f4ff2c00884178000102200090072000a8
:10be600033ef070080047800881f7800f7ff2c006c
:10be700006c2b3008841780084002000050020003d
:10be800022c0b30001022000cef007000080fb00ba
:10be90008084440088027800f4ff2c0088417800f8
:10bea000e2c2b300010220000900780030ee070072
:10beb0000080fb0000804400881f7800f7ff2c0002
:10bec00006c3b300884178006022b80022c0b300e6
:10bed00001022000bbf0070020262100104278005c
:10bee000881f7800f7ff2c0006c2b3008841780055
:10bef0000482fb000500200022c0b30001012000e5
:10bf000008007800aff007008084fb00880278000a
:10bf1000f4ff2c0088417800e2c2b3000101200048
:10bf20000900780012ee07000080fb0080844400c6
:10bf30003026210010427800881f7800f7ff2c007f
:10bf400006c3b300884178000482fb00050020008e
:10bf500022c0b300010120000900780099f0070019
:10bf60000080fb008084440088027800f4ff2c00ed
:10bf700088417800e2c2b300010120000900780086
:10bf8000fbed0700412621001182fb00017d20000e
:10bf9000010242000080fb0000804400881f7800fe
:10bfa000f7ff2c0006c3b30088417800cfa2de0063
:10bfb00042c0b3000101200082f00700881f780012
:10bfc000f7ff2c0006c2b30088417800440020002f
:10bfd0000500200022c0b3000101200090072000ce
:10bfe00078f007000080fb0099072000808444005f
:10bff00088027800f4ff2c0088417800e2c2b30088
:10c000000101200009007800d9ed07000080fb0045
:10c0100080844400881f7800f7ff2c0006c3b3001b
:10c0200088417800440020000500200022c0b300b1
:10c03000010120000900780062f007000080fb0089
:10c040008084440088027800f4ff2c008841780046
:10c05000e2c2b3000101200009007800c4ed07002e
:10c060000080fb0000804400881f7800f7ff2c0050
:10c0700006c3b30088417800847d200005002000bd
:10c0800042c0b300010120004ef0070043c0b300de
:10c090000341780083407800c0c0b30046f1070038
:10c0a000f48757004f05be004f04be000000060095
:10c0b000a0d920001080fb00000040008008b000e4
:10c0c000618c2000608178008002eb00f4ff2c007e
:10c0d00085417800010a20000500780094ee0700f1
:10c0e00043c0b3000341780083407800c0c0b30070
:10c0f00031f1070000000600881f780063d7200098
:10c100001380fb00a2002000110009000280d8006b
:10c1100000447800a0d72000904f54001400320053
:10c1200094c0b300934f1200010036000842e900aa
:10c13000a0d920001080fb0000004000400bb000a0
:10c14000618c2000608178008480fb00c408dd00e1
:10c150000103b0008002eb00050278008541780001
:10c160008005200072ee0700a0d720000848780064
:10c17000a0d920001080fb0000004000400bb00060
:10c18000618c2000608178008880fb00c408dd009d
:10c190000103b000e53827000002eb00844178007d
:10c1a0008005200062ee07004f04780000000600c2
:10c1b000889fbe008a1f7800a0d920001080fb0055
:10c1c000000040006c004000c182200060817800c7
:10c1d0008002eb00f457280013c0b300010e2000ca
:10c1e0000500780052ee0700f7f107000004eb00ad
:10c1f000090c20000a882000f5012000b0d9200099
:10c20000904f140001003200e53827000800440078
:10c21000a1d920009180fb000100400000004000f7
:10c2200060017d00f4ff2c008041eb008900780064
:10c230000000eb003eee07000804e800f084540024
:10c24000ea0f5400ecff3a00c8da20008041eb000e
:10c250001841780001012000600120001af1070058
:10c260008041eb00184178008000eb00b000200016
:10c2700066f1070083c0b30052c0b30061c0b300d1
:10c28000c0c0b300ccf007004f0578004f04be00db
:10c2900000000600881f7800b0d920001080fb0045
:10c2a00000004000a1d920009180fb000100400067
:10c2b0000000400041852000608178008002eb0092
:10c2c000f457280013c0b300010e200005007800c9
:10c2d00017ee0700bcf10700e5382700f4ff2c003b
:10c2e0008041eb0062458000010c2000b00020007e
:10c2f0000fee07006b044000f0012000801f780063
:10c30000f7ff2c0006c2b30003c4b300e46e800044
:10c310000500200032c0b300010c200008007800a6
:10c32000a8ef0700724580000080fb000000440079
:10c33000e5382700f4ff2c008041eb00010c2000c1
:10c34000fbed070083c0b300a2c0b300b1c0b300cf
:10c35000c0c0b30098f007008f87e9004f04780051
:10c3600000000600881f7800b0d920001080fb0074
:10c3700000004000a1d920009180fb000100400096
:10c380000000400041852000608178008002eb00c1
:10c39000f457280013c0b300010e200005007800f8
:10c3a000e3ed070088f10700c8da200013c0b300ee
:10c3b000184178000106200080052000c2f0070027
:10c3c00013c0b3001841780001042000d0042000fd
:10c3d0000ef1070083c0b300a2c0b300b1c0b30028
:10c3e000c0c0b30074f007004f04780000000600de
:10c3f000881f7800a8d920001880fb0000004000aa
:10c4000074004000c1822000608178008002eb004f
:10c41000f457280013c0b300010e20000500780077
:10c42000c3ed070068f10700c02b21001080fb005e
:10c43000000040009880fb00010040000000400028
:10c44000219f2000608178008002eb00f4ff2c0027
:10c45000854178000107200005007800b4ed070051
:10c4600043c0b3000341780083407800c0c0b300ec
:10c4700051f007004f04780000000600889fbe00be
:10c48000006c80000088a300b7003200c02b2100a0
:10c490001004e00002003200d5ff0700ac003700b6
:10c4a000a0d920001080fb00000040008002b000f6
:10c4b00041852000608178008002eb00f45728005d
:10c4c00013c0b300010e20000500780098ed0700ae
:10c4d0003df10700509380006104b80059f1070056
:10c4e000801f7800f7ff2c0006c2b30023c0b30002
:10c4f0000802be0042c0b300010a20000002200072
:10c5000030ef07008002eb00f4ff2c0023c0b300e3
:10c51000a2c3b300010a20000100780094ec0700d8
:10c520008002eb00f4ff2c0023c0b300b2c3b300c1
:10c53000010a2000000c20008dec0700949580007b
:10c54000c8032000110009000882d800000278000a
:10c550008004eb00891f7800f7ff2c0006c3b300ae
:10c56000894178000500200022c0b30001082000a6
:10c57000b000200013ef070089027800f4ff2c00c0
:10c5800089417800a2c3b3000108200010022000f6
:10c5900077ec070090958000110009000880d80012
:10c5a00001027800891f7800f7ff2c0006c3b30052
:10c5b000894178000500200022c0b3000108200056
:10c5c000c0022000ffee070001082000f008200054
:10c5d00007f30700a245800089027800f4ff2c00d1
:10c5e0008941780001072000a009200050ed0700d4
:10c5f00000047800a0958000e68757000000e00066
:10c600000d003400891f7800f7ff2c0006c2b3002c
:10c61000894178006102b90042c0b30001072000df
:10c6200008007800e7ee07000080fb0000034400ec
:10c630008f87e9000c0037008001eb00831f780032
:10c64000f7ff2c0006c2b3006022b80042c0b3005e
:10c650000107200008007800daee07000080fb00e8
:10c66000000344008f87e900698c2000a8d92000ce
:10c670001880fb00000040007400400060817c00d6
:10c680008002eb00f4ff2c008541780001072000b8
:10c690000600780026ed0700006c80000098a300db
:10c6a000150032001880fb000000400068004000c8
:10c6b00060817c008002eb00f4ff2c008541780053
:10c6c000010520006001200019ed07001880fb0023
:10c6d000000040006c00400060817c008002eb00a4
:10c6e000f4ff2c008541780001042000c0022000e6
:10c6f0000fed070016003700502621001080fb00c8
:10c7000000004000a1d920009180fb000100400002
:10c7100000004000a1a42000608178008002eb00ae
:10c72000f4ff2c0003c8b3000105200060012000c5
:10c73000ffec07008002eb00f4ff2c00854178003d
:10c7400042c1b300010420006001200083f0070013
:10c7500043c0b3000341780083407800c0c0b300f9
:10c7600095ef07003b003700b0d920001080fb0098
:10c7700000004000a8d920009880fb000100400084
:10c780000000400041852000608178008002eb00bd
:10c79000f457280013c0b300010e200005007800f4
:10c7a000e3ec070088f007001880fb000000400061
:10c7b00070004000618c2000608178008002eb00f6
:10c7c000f4ff2c0085417800010c20000500780062
:10c7d000d7ec07001880fb00000040007400400008
:10c7e000619d2000608178008002eb00f4ff2c0046
:10c7f0008541780001072000c0022000ccec070032
:10c80000823e200003002000906e8000a16e800018
:10c81000860f0200000000008001eb00831f7800fb
:10c82000f7ff2c0006c2b3000002be0072c0b300c6
:10c83000010520008005200062ee070043c0b30020
:10c8400052c0b30061c0b300c0c0b3005aef0700cc
:10c850008f87e9004f04be0000000600889fbe00dd
:10c860008a1f7800b0d920001080fb000000400033
:10c87000a1d920009180fb00010040000000400091
:10c8800041852000608178008002eb00f457280089
:10c8900013c0b300010e200005007800a4ec0700cf
:10c8a00049f007000004eb00090c20002aa7200033
:10c8b000f5012000f0d92000904f14000100320053
:10c8c000e538270008004400a1d920009180fb0032
:10c8d000010040000000400060017d00f4ff2c00da
:10c8e0008041eb00890078000000eb0090ec07002d
:10c8f0000804e800f0845400e20f5400ecff3a0012
:10c9000083c0b30052c0b30061c0b300c0c0b30065
:10c9100029ef07004f0578004f04be000000060015
:10c92000889fbe008a1f7800f0d920001080fb008d
:10c9300000004000aad920009a80fb0001004000be
:10c9400000004000a1a62000608178008002eb007a
:10c95000f457280013c0b300010e20000500780032
:10c9600073ec070018f00700509380006104b800d2
:10c9700034f00700801f7800f7ff2c0006c2b300d8
:10c9800023c0b3000802be0042c0b300010a200069
:10c99000000220000bee07008002eb00f4ff2c00e9
:10c9a00023c0b300a2c3b300010a20000100780035
:10c9b0006feb07008002eb00f4ff2c0023c0b300f4
:10c9c000b2c3b300010a2000000c200068eb07008e
:10c9d00094958000c8032000110009000882d80047
:10c9e000000278008004eb00891f7800f7ff2c001c
:10c9f00006c3b300894178000500200022c0b300bf
:10ca000001082000b0002000eeed07008902780048
:10ca1000f4ff2c0089417800a2c3b3000108200074
:10ca20001002200052eb07009095800011000900d1
:10ca30000880d80001027800891f7800f7ff2c00d9
:10ca400006c3b300894178000500200022c0b3006e
:10ca500001082000c0022000daed070001082000d4
:10ca600030062000e2f10700688c20001a80fb00ed
:10ca7000000040007800400060017c0089027800de
:10ca8000f4ff2c008941780001072000e006200017
:10ca900027ec070001db200001629000891f78006d
:10caa000f7ff2c0006c2b30003c8b3000482fb00ea
:10cab0000500200032c0b30001072000c1ed0700cf
:10cac0001a80fb000000400064004000a1a8200084
:10cad0006081780005802f00f4ff2c0089417800e8
:10cae000010420000900780011ec070005802f00e8
:10caf000f4ff2c0089417800b2c4b3000104200087
:10cb0000000b20001aeb07000080fb00000bb000b8
:10cb100005802f00f4ff2c008941780022ceb3005d
:10cb20000104200012eb0700006c8000e88757002a
:10cb30000098a300150032001a80fb00000040009e
:10cb40006800400060017c0089027800f4ff2c003e
:10cb5000894178000106200060012000f4eb070005
:10cb60001a80fb00000040006c00400060017c0067
:10cb700089027800f4ff2c0089417800010520002b
:10cb8000c0022000eaeb07000e0037008002eb0035
:10cb9000f4ff2c008541780042c1b300010620005b
:10cba000600120006def07008002eb00f4ff2c0015
:10cbb0008541780042c1b3000105200060012000da
:10cbc00066ef070043c0b300a2c0b300b1c0b3001a
:10cbd000c0c0b30078ee07004f0578004f04be00d8
:10cbe00000000600f0d920001080fb00000040008b
:10cbf000a1d920009180fb0001004000000040000e
:10cc0000a1a62000608178008002eb00f457280084
:10cc100013c0b300010e200005007800c4eb07002c
:10cc200069ef0700e025210090407800f0c5b300cf
:10cc300080cf500007003e006440500080cf50007d
:10cc4000100031000040e90080cf500028003a0079
:10cc50000400370000c6b30080cf500024003a0023
:10cc60001c003700b24580008002eb00f4ff2c006e
:10cc700085417800010c2000b0002000aceb0700db
:10cc80001b003700d24580008002eb00f4ff2c002f
:10cc900085417800010c2000b0002000a4eb0700c3
:10cca000e1252100114278008001eb00831f78000c
:10ccb000f7ff2c0006c2b3000482fb000500200031
:10ccc00022c0b300010c20003eed07008f87e90071
:10ccd00007003700c24580008002eb00f4ff2c0003
:10cce00085417800010c2000b000200090eb070087
:10ccf000a0d920001080fb00000040006c00400024
:10cd0000a1a72000608178008002eb00f4ff2c00d6
:10cd100085417800010820000500780084eb0700b9
:10cd200083c0b300a2c0b300b1c0b300c0c0b300a1
:10cd300021ee070000000600889fbe008a9fbe000b
:10cd4000006c800000a8a300ee0032000004210067
:10cd500010407800ff456000b0d920001080fb0033
:10cd600000004000a1d920009180fb00010040009c
:10cd70000000400041852000608178008002eb00c7
:10cd8000f457280013c0b300010e200005007800fe
:10cd900067eb07000cef0700509380006104b800b8
:10cda00028ef0700801f7800f7ff2c0006c2b300b1
:10cdb00023c0b3000802be0042c0b300010a200035
:10cdc00000022000ffec07008002eb00f4ff2c00c3
:10cdd00023c0b300a2c3b300010a20000100780001
:10cde00063ea07008002eb00f4ff2c0023c0b300cd
:10cdf000b2c3b300010a2000000c20005cea070067
:10ce00008f87e900eccf550028003a0089252000e3
:10ce10009495800004825400ca0320001100090088
:10ce20000a82d800000278000004eb00881f780016
:10ce3000f7ff2c0006c3b3008841780005002000ee
:10ce400022c0b30001082000b0002000ddec070084
:10ce500088027800f4ff2c0088417800a2c3b30058
:10ce6000010820001002200041ea07009095800090
:10ce700080845400110009008a84d80001027800df
:10ce8000881f7800f7ff2c0006c3b30088417800a4
:10ce90000500200022c0b30001082000c0022000cd
:10cea000c8ec0700e4875700070037008002eb005a
:10ceb000f4ff2c008541780052c0b3000108200027
:10cec000b0002000a5ee07008002eb00f4ff2c006c
:10ced00085417800d2cab3000108200080052000f7
:10cee00023ea07008002eb00f4ff2c008541780064
:10cef0006245800001082000300620000ceb07008e
:10cf0000e16d8000f06d8000808f500005003100e1
:10cf1000010050000000d100c012b000c09688008f
:10cf200005003700808050008100d100c012200031
:10cf300001005000c0968800c1968000b012200009
:10cf4000808f500015003e008002eb00f4ff2c00a3
:10cf500085417800d2c2b30001082000900720006c
:10cf600003ea0700c4122000c096800000025200ad
:10cf70008001eb00831f7800f7ff2c0006c2b3008e
:10cf80000500200032c0b300010820004008200046
:10cf90008cec07008f87e900140037008002eb005b
:10cfa000f4ff2c008541780002c2b3000108200084
:10cfb00090072000eee90700c496800040ed2f00a6
:10cfc000000242008001eb00831f7800f7ff2c0075
:10cfd00006c2b3000500200032c0b30001082000e3
:10cfe0004008200077ec07008f87e900e2458000c9
:10cff0008002eb00f4ff2c0085417800010820003e
:10d00000500a2000caea0700a0d920001080fb00c7
:10d010000000400064004000a1a82000608178006a
:10d0200005802f00f4ff2c008041eb00010420005c
:10d030000000eb00beea070005802f00f4ff2c0083
:10d040008041eb00d2cab30001042000000b200095
:10d05000c7e9070005802f00f4ff2c008041eb009a
:10d0600042c5b30001042000b00b2000c0e9070056
:10d07000e2cf550004003200ebcf55000200320031
:10d08000eccf550012003a00a0d920001080fb0020
:10d090000000400070004000a1a4200060817800e2
:10d0a0008002eb00f4ff2c0003c8b300010620004f
:10d0b000c00220009eea070083c0b300a2c0b300f4
:10d0c000b1c0b300c0c0b3003bed0700290037007a
:10d0d0008002eb00f4ff2c008541780042c1b300d0
:10d0e00001062000c00220001cee070083c0b30030
:10d0f000a2c0b300b1c0b30020c0b3002eed070042
:10d100001c003700a8d920001880fb000000400058
:10d1100078004000c1822000608178008002eb002e
:10d12000f457280013c0b300010e2000050078005a
:10d130007fea070024ee07001880fb000000400093
:10d14000a1a82000608178008002eb00f4ff2c0091
:10d1500085417800010c20000500780074ea070082
:10d1600043c0b3000341780083407800c0c0b300df
:10d1700011ed07004f05be004f04be000000060081
:10d18000889fbe00b0d920001080fb000000400046
:10d19000a1d920009180fb00010040000000400068
:10d1a00041852000608178008002eb00f457280060
:10d1b00013c0b300010e2000050078005cea0700f0
:10d1c00001ee07005026210010407800e24f500089
:10d1d0001b00320003003900e34f50002f003a00db
:10d1e00023003700698c2000a8d920001880fb009c
:10d1f000000040007c00400060817c008002eb0069
:10d20000f4ff2c0085417800010b20002004200051
:10d2100047ea07001880fb00000040000002b00051
:10d2200060817c008002eb00f4ff2c0085417800d7
:10d2300001092000200420003dea07001700370004
:10d240008001eb00831f7800f7ff2c0006c2b300bb
:10d25000949580000500200022c0b300010b20003f
:10d26000b00b2000d7eb07008f87e9000b003700d9
:10d270008001eb00831f7800f7ff2c0006c2b3008b
:10d28000949580000500200022c0b3000109200011
:10d29000b00b2000cbeb07008f87e9005026210060
:10d2a00031c0b30090cf10000d003600a0d920008f
:10d2b0001080fb00000040004002b000618c2000a4
:10d2c000608178008002eb00f4ff2c0003c8b300fb
:10d2d000010720001002200015ea0700280037008f
:10d2e000006c80000098a30017003200698c2000b9
:10d2f000a8d920001880fb00000040006800400012
:10d3000060817c008002eb00f4ff2c0085417800f6
:10d31000010720006001200005ea07001880fb00db
:10d32000000040006c00400060817c008002eb0047
:10d33000f4ff2c008541780001062000c002200087
:10d34000fbe907000e0037008002eb00f4ff2c0021
:10d350008541780042c1b300010720006001200030
:10d360007eed07008002eb00f4ff2c008541780081
:10d3700042c1b300010620006001200077ed0700e4
:10d3800043c0b3000341780083407800c0c0b300bd
:10d3900089ec07004f04be0000000600889fbe0015
:10d3a000b0d920001080fb0000004000a8d9200068
:10d3b0009880fb00010040000000400041852000f3
:10d3c000608178008002eb00f457280013c0b3009e
:10d3d000010e200005007800d5e907007aed07006e
:10d3e000698c20001880fb00000040008006b0001f
:10d3f00060817c008002eb00f4ff2c008541780006
:10d400000109200010022000c9e907001880fb0074
:10d4100000004000c006b00060817c00e5382700b5
:10d42000f4ff2c008041eb0001072000e006200003
:10d43000bfe9070080de200050429000801feb0013
:10d44000f7ff2c0006c2b30003c4b3000482fb0044
:10d450000500200022c0b30001072000f0082000d2
:10d4600058eb070083c0b300a2c0b300b1c0b30043
:10d47000c0c0b30050ec07008f87e9004f04be0026
:10d4800000000600889fbe008a1f7800b0d92000e7
:10d490001080fb0000004000a1d920009180fb001b
:10d4a00001004000000040004185200060817800bc
:10d4b0008002eb00f457280013c0b300010e2000d7
:10d4c000050078009ae907003fed07000004eb0033
:10d4d000090c20006aaa2000f501200000da2000d3
:10d4e000904f140001003200e53827000800440086
:10d4f000a1d920009180fb00010040000000400005
:10d5000060017d00f4ff2c008041eb008900780071
:10d510000000eb0086e907000804e800f0845400ee
:10d52000e20f5400ecff3a0043c0b300034178001f
:10d5300083407800c0c0b3001fec07004f0578009f
:10d540004f04be0000000600889fbe008a9fbe00f8
:10d5500000da20001080fb0000004000aad9200063
:10d560009a80fb00010040000000400021ab200039
:10d57000608178008002eb00f457280013c0b300ec
:10d58000010e20000500780069e907000eed070094
:10d590002bac20001a80fb0000004000640040001b
:10d5a00060817d008002eb00f4ff2c008541780053
:10d5b000010c2000100220005de9070080047800c3
:10d5c0000004eb00881f7800f7ff2c0006c2b300b0
:10d5d00088417800546e80000500200042c0b300ee
:10d5e000010c2000f7ea0700e24580000080fb0004
:10d5f0008084440088027800f4ff2c008841780081
:10d60000010c20000900780049e907001a80fb009e
:10d61000000040006800400060817d0088027800c2
:10d62000f4ff2c0088417800010a200008007800ef
:10d630003fe90700881f7800f7ff2c0006c2b300ff
:10d6400088417800b46d80000500200042c0b3001e
:10d650000109200030062000daea07001a80fb00ea
:10d66000000040006c00400060817d00880278006e
:10d67000f4ff2c008841780001092000a009200057
:10d680002be9070043c0b3000341780083407800d2
:10d69000c0c0b300c8eb0700e48757004f05be00c9
:10d6a0004f04be0000000600124680008002eb001e
:10d6b000f4ff2c00854178000107200020042000a1
:10d6c0001be90700516e8000d0958000808f5000cc
:10d6d000150031008002eb00f4ff2c00854178003a
:10d6e00002c2b300010720003006200020e8070036
:10d6f000d4958000506e8000000252008001eb0043
:10d70000831f7800f7ff2c0006c2b300050020003d
:10d7100042c0b30001072000e0062000a9ea07008c
:10d720008f87e900140037008002eb00f4ff2c0023
:10d7300085417800d2c2b3000107200030062000e6
:10d740000be80700546e8000d09580000002520064
:10d750008001eb00831f7800f7ff2c0006c2b300a6
:10d760000500200042c0b30001072000e0062000b1
:10d7700094ea07008f87e90000000600889fbe003a
:10d780008a9fbe00abd920001b80fb000000400038
:10d790006800400021ab2000608178008002eb002f
:10d7a000f457280013c0b300010e200005007800d4
:10d7b000dfe8070084ec0700509380006104b800a4
:10d7c000a0ec0700801f7800f7ff2c0006c2b30012
:10d7d00023c0b3000802be0042c0b300010a20000b
:10d7e0000002200077ea07008002eb00f4ff2c0023
:10d7f00023c0b300a2c3b300010a200001007800d7
:10d80000dbe707008002eb00f4ff2c0023c0b3002d
:10d81000b2c3b300010a2000000c2000d4e70700c7
:10d8200094958000c8032000110009000882d800e8
:10d83000000278008004eb00891f7800f7ff2c00bd
:10d8400006c3b300894178000500200022c0b30060
:10d8500001082000b00020005aea07008902780081
:10d86000f4ff2c0089417800a2c3b3000108200016
:10d8700010022000bee7070090958000110009000b
:10d880000880d80001027800891f7800f7ff2c007b
:10d8900006c3b300894178000500200022c0b30010
:10d8a00001082000c002200046ea0700f24580007f
:10d8b00089027800f4ff2c008941780001082000db
:10d8c000e00620009ae80700891f7800f7ff2c0087
:10d8d00006c2b300894178007493800005002000df
:10d8e00042c0b300010820004008200035ea0700cc
:10d8f0006a8c20001b80fb00000040008002b0000a
:10d9000060017d0089027800f4ff2c0089417800d5
:10d9100001082000000b200085e8070058262100a0
:10d920001880fb00000040009b80fb0001004000cd
:10d930000000400021ad200060817800890278005d
:10d94000f4ff2c0003c8b3000103200010022000e4
:10d9500077e8070018407800e8875700e64f500046
:10d960003e003a001b80fb0000004000c002b000f7
:10d9700060017d0089027800f4ff2c008941780065
:10d9800001072000e006200069e80700891f7800f1
:10d99000f7ff2c0006c2b30089417800b4958000df
:10d9a0000500200042c0b30001072000b00b20009a
:10d9b00004ea07001b80fb00000040000003b000e9
:10d9c00060017d0089027800f4ff2c008941780015
:10d9d00001062000e006200055e80700891f7800b6
:10d9e000f7ff2c0006c2b30089417800c49580007f
:10d9f0000500200042c0b30001062000b00b20004b
:10da0000f0e907001b80fb00000040004003b0006d
:10da100060017d0089027800f4ff2c0089417800c4
:10da200001052000e006200041e80700891f78007a
:10da3000f7ff2c0006c2b30089417800d49580001e
:10da40000500200042c0b30001052000b00b2000fb
:10da5000dce90700e687570029003700e74f500050
:10da600002003a0010ff070025003700e84f500081
:10da700023003a00e0d820001080fb000000e900fd
:10da8000f1d82000e0c0780080c2b30080cf500001
:10da900018003a00a0d920001080fb0000004000d0
:10daa0008003b000618c2000608178008002eb0070
:10dab000f4ff2c008541780001042000e0062000de
:10dac0001be807008001eb00831f7800f7ff2c00a4
:10dad00006c2b300246e80000500200042c0b300df
:10dae00001042000b00b2000b6e907008f87e90091
:10daf00003003700ffcf500001003a00eafe0700a4
:10db0000006c80000098a30017003200698c200090
:10db1000a8d920001880fb000000400068004000e9
:10db200060817c008002eb00f4ff2c0085417800ce
:10db30000102200060012000fde707001880fb00c3
:10db4000000040006c00400060817c008002eb001f
:10db5000f4ff2c008541780001012000c002200064
:10db6000f3e707000e0037008002eb00f4ff2c0003
:10db70008541780042c1b30001012000600120000e
:10db800076eb07008002eb00f4ff2c008541780063
:10db900042c1b30085007800600120006feb0700f0
:10dba00043c0b3000341780083407800c0c0b30095
:10dbb00081ea07004f05be004f04be0000000600ca
:10dbc000889fbe0000da20001080fb0000004000ab
:10dbd000a8d920009880fb00010040000000400010
:10dbe00021ab2000608178008002eb00f457280010
:10dbf00013c0b300010e200005007800cce7070039
:10dc000071eb07001880fb00000040006800400036
:10dc100061aa2000608178008002eb00f4ff2c00f4
:10dc200085417800010c200070032000c0e7070048
:10dc30001880fb0000004000c003b000618c200091
:10dc400060817800e5382700f4ff2c008041eb006c
:10dc50000109200020042000b5e707000004780037
:10dc60008004eb00891f7800f7ff2c0006c2b30088
:10dc700089417800449480000500200042c0b30030
:10dc8000010920004fe90700e24580000080fb0009
:10dc900000044400e5382700f4ff2c008941780097
:10dca0000109200008007800a1e7070083c0b30045
:10dcb000a2c0b300b1c0b300c0c0b3003eea0700c9
:10dcc0008f87e9004f04be0000000600889fbe0059
:10dcd0008a9fbe00b0d920001080fb0000004000e9
:10dce000a1d920009180fb0001004000000040000d
:10dcf00041852000608178008002eb00f457280005
:10dd000013c0b300010e20000500780088e707006b
:10dd10002deb07000004eb00aaaf2000090c200047
:10dd20009bd92000f00120009b4f1400010032001d
:10dd3000e038270080027800f4ff2c008041eb00df
:10dd40003a017800890078000000eb0078e70700ce
:10dd50000804e800f0845400e20f5400f1ff3a0098
:10dd600043c0b3000341780083407800c0c0b300d3
:10dd700011ea07004f05be004f04be000000060078
:10dd8000881f7800b0d920001080fb000000400000
:10dd9000a8d920009880fb0001004000000040004e
:10dda00041852000608178008002eb00f457280054
:10ddb00013c0b300010e2000050078005ce70700e7
:10ddc00001eb07001880fb00000040008002b0005b
:10ddd00001882000608178008002eb00f4ff2c00b5
:10dde00085417800010c20008000200050e70700ea
:10ddf00043c0b3000341780083407800c0c0b30043
:10de0000ede907004f04780000000600889fbe007f
:10de10008a1f7800a0d920001080fb00000040007d
:10de200070004000c1822000608178008002eb0019
:10de3000f457280013c0b300010e2000050078003d
:10de40003be70700e0ea07000004eb00090c2000b4
:10de50006a9d2000f5012000e0d92000904f1400b9
:10de600001003200e538270008004400a1d9200055
:10de70009180fb00010040000000400060017d0037
:10de8000f4ff2c008041eb00890078000000eb00db
:10de900027e707000804e800f0845400e70f540067
:10dea000ecff3a0043c0b30052c0b30061c0b300fe
:10deb000c0c0b300c0e907004f0578004f04be00a2
:10dec00000000600881f7800e0d920001080fb00c9
:10ded00000004000a8d920009880fb00010040000d
:10dee0000000400021b12000608178008002eb003a
:10def000f457280013c0b300010e2000050078007d
:10df00000be70700b0ea07008293800013c0b3005c
:10df1000010c2000e0062000edec07001880fb005b
:10df20000000400064004000a1a82000608178004b
:10df300005802f00f4ff2c008041eb00010420003d
:10df40000000eb00fae6070005802f00f4ff2c002c
:10df50008041eb0042c5b30001042000000b20000b
:10df600003e6070043c0b300a2c0b300b1c0b300d2
:10df7000c0c0b30090e907004f047800000006001d
:10df8000889fbe008a9fbe008c9fbe008e1f7800b7
:10df9000e0d920001080fb0000004000a1d9200043
:10dfa0009180fb00010040000000400021b12000f2
:10dfb000608178008002eb00f457280013c0b300a2
:10dfc000010e200005007800d9e607007eea070070
:10dfd0008005eb000a0c2000eeaf2000add9200038
:10dfe0000b067800005729006b4478000b80450031
:10dff0009d80fb00010040000000400060017f00a8
:10e000008002eb00f4ff2c00854178008a00780044
:10e01000b0002000c6e60700800478008002eb0014
:10e02000f4ff2c0085417800a2c3b3008a00780079
:10e03000cfe507000080fb00808444000884fb00db
:10e0400008044400e0292100680278008c1f780051
:10e05000f7ff2c0006c2b3008c41780005002000b9
:10e0600042c0b3008a0078000900780055e8070034
:10e070009d80fb00818040008102b000628c200006
:10e08000610179000080fb00008044008c02780070
:10e09000f4ff2c008c4178008a007800a4e6070089
:10e0a0008b05e800700555008f87e900e58f550066
:10e0b000ccff3a0043c0b3000341780083407800ae
:10e0c000c0c0b3003ce907004f0778004f06be0010
:10e0d0004f05be004f04be0000000600889fbe0032
:10e0e0008a9fbe008c9fbe008e1f7800e0d9200062
:10e0f0001080fb0000004000a1d920009180fb00af
:10e10000010040000000400021b120006081780043
:10e110008002eb00f457280013c0b300010e20006a
:10e120000500780082e6070027ea07000005eb00fb
:10e13000fde328000c0c20000edb20000a447800d0
:10e14000f901200010da2000904f15000100320084
:10e15000e93827000a004500a1d920009180fb0082
:10e160000100400000004000e1b220006081780022
:10e1700089027800f4ff2c008041eb008c007800cd
:10e180000000eb006ae6070080057800e54f5400c8
:10e190000e0036001d80fb0060427f00891f780062
:10e1a000f7ff2c0006c2b3008041eb000482fb00a5
:10e1b0000500200042c0b3008c0078000b007800fe
:10e1c00000e807008f87e9000d0037001d80fb0085
:10e1d0000000400060027f00891f7800f7ff2c00dc
:10e1e00006c2b3008041eb000500200042c0b3002e
:10e1f0008c0078000b007800f2e707008f87e900b9
:10e200000a05e8008d06e80070065600e90f550083
:10e21000caff3a0083c0b300a2c0b300b1c0b300cc
:10e22000c0c0b300e4e807004f0778004f06be0007
:10e230004f05be004f04be0000000600889fbe00d0
:10e240008a9fbe008c9fbe008e1f7800e0d9200000
:10e250001080fb0000004000a1d920009180fb004d
:10e26000010040000000400021b1200060817800e2
:10e270008002eb00f457280013c0b300010e200009
:10e28000050078002ae60700cfe907000a0c200005
:10e290006066b8000edc2000abd92000006c800066
:10e2a0000004b20002003a00800478000500370044
:10e2b000f901200020da2000904f560001003200c2
:10e2c000e93827001b80fb000000400021ac200043
:10e2d0006081780089027800f4ff2c008041eb0017
:10e2e0008a0078006001200011e607000004780031
:10e2f00061064600e0864e00891f7800f7ff2c007b
:10e3000006c2b3008041eb000c02be0012c0b30095
:10e310008a007800abe707000080fb00000444009f
:10e3200089027800f4ff2c008041eb00a2c3b30007
:10e330008a007800080078000de507000080fb00e7
:10e34000000444003e027800891f7800f7ff2c008b
:10e3500006c2b3008041eb000500200042c0b300bc
:10e360008a0078000800780096e707009b80fb0091
:10e37000818040008102b000628c20006101790040
:10e380000080fb000000440089027800f4ff2c00ac
:10e390008041eb008a007800e5e507007005550034
:10e3a000e487570000092000800f5500bbff3a00aa
:10e3b0008c407800006c80000004b20002003a003b
:10e3c0008006780006003700fd01200020da2000da
:10e3d00032c0b300904f110001003200ed38270029
:10e3e0000180fb004400dd00010c2000008650008d
:10e3f0002aac2000a9d920001980fb0000004000b1
:10e400006400400060017d008d027800f4ff2c0064
:10e410008041eb008c00780010022000c4e507006a
:10e42000000478008d1f7800f7ff2c0006c2b300af
:10e430008041eb00546e80000500200042c0b30014
:10e440008c0078005fe70700e24580000080fb0059
:10e45000000444008d027800f4ff2c008041eb00a2
:10e460008c00780008007800b1e507001980fb00f7
:10e47000000040006800400060017d008002eb0069
:10e48000f4ff2c008541780001072000050078008a
:10e49000a7e507000004eb00881f7800f7ff2c00b9
:10e4a00006c2b30088417800b46d800005002000ea
:10e4b00042c0b300010620003006200041e70700fb
:10e4c0001980fb00000040006c00400060017d00ee
:10e4d00088027800f4ff2c008841780001062000b3
:10e4e000a009200092e50700006c8000e487570037
:10e4f000a2c0b300b1c0b30043c0b3000068a30022
:10e5000003003a0042c0b3008240780033c0b30039
:10e51000c0c0b30028e807004f0778004f06be00d0
:10e520004f05be004f04be0000000600889fbe00dd
:10e530008a9fbe008c1f7800e0d920001080fb006d
:10e5400000004000a9d920009980fb000100400094
:10e550000000400021b12000608178008002eb00c3
:10e56000f457280013c0b300010e20000500780006
:10e570006fe5070014e90700006c80000098a30015
:10e5800016003200688c20001980fb00000040005b
:10e590006800400060017c008002eb00f4ff2c006a
:10e5a00085417800010220006001200060e507003d
:10e5b0001980fb00000040006c00400060017c00fe
:10e5c0008002eb00f4ff2c0085417800010120005f
:10e5d000c002200056e507001f003700502621002a
:10e5e00061c0b30090cf10000d003600a0d920000c
:10e5f0001080fb00000040004002b000618c200051
:10e60000608178008002eb00f4ff2c0003c8b300a7
:10e61000010320006001200045e507000e003700df
:10e620008002eb00f4ff2c008541780042c1b3006a
:10e630000102200060012000c8e807008002eb0012
:10e64000f4ff2c008541780042c1b3000101200095
:10e6500060012000c1e80700509380006104b80009
:10e66000f8e80700801f7800f7ff2c0006c2b3000f
:10e6700023c0b3000802be0042c0b30061092000fd
:10e6800000022000cfe607008002eb00f4ff2c0020
:10e6900023c0b300a2c3b30061092000000a200018
:10e6a00033e407008002eb00f4ff2c0023c0b3002a
:10e6b000b2c3b30061092000000c20002ce4070065
:10e6c00094958000c8032000110009000882d8003a
:10e6d000000278008004eb00891f7800f7ff2c000f
:10e6e00006c3b300894178000500200022c0b300b2
:10e6f00001082000b0002000b2e60700890278007f
:10e70000f4ff2c0089417800a2c3b3000108200067
:10e710001002200016e40700909580001100090007
:10e720000880d80001027800891f7800f7ff2c00cc
:10e7300006c3b300894178000500200022c0b30061
:10e7400001082000c00220009ee60700502621009c
:10e7500010407800e6875700e14f500004003a006f
:10e76000094678008945780009c8b30010003700d1
:10e77000e24f500004003a000046eb000bc8b30023
:10e780008c4478000a00370064405000e14f50008c
:10e7900004003e000cc8b3008045eb008b447800b9
:10e7a000030037000046eb008c4578008c4478006d
:10e7b0000004eb00881f7800f7ff2c0006c2b300ae
:10e7c00088417800a44b20000500200042c0b3001f
:10e7d00001062000a00920007ae60700e24580003b
:10e7e00088027800f4ff2c008841780001062000a0
:10e7f000600c2000cee40700881f7800f7ff2c0093
:10e8000006c3b300884178001400200005002000f2
:10e8100022c0b30001052000a009200069e607001e
:10e8200088027800f4ff2c0088417800a2c3b3006e
:10e8300001052000000b2000cde30700881f7800b1
:10e84000f7ff2c0006c3b300884178006022b800af
:10e8500022c0b30001052000b00b200059e60700dc
:10e8600000db2000705a9000881f7800f7ff2c0012
:10e8700006c2b300884178000482fb000500200036
:10e8800042c0b30001042000a00920004de60700ab
:10e890002246800088027800f4ff2c00894178002d
:10e8a00001062000b0002000a1e407006a8c2000cf
:10e8b000a9d920001980fb00000040000004b0002e
:10e8c00060017d0088027800f4ff2c008b41780005
:10e8d00001052000b000200095e407001980fb002e
:10e8e000000040004004b00060017d008802780014
:10e8f000f4ff2c008c41780001042000b0002000bf
:10e900008be4070043c0b3000341780083407800e4
:10e91000c0c0b30028e70700e88757004f0678001b
:10e920004f05be004f04be0000000600889fbe00d9
:10e930008a1f7800e0d920001080fb000000400012
:10e94000a9d920009980fb00010040000000400090
:10e9500021b12000608178008002eb00f45728008c
:10e9600013c0b300010e20000500780070e407001a
:10e9700015e807006a8c20001980fb0000004000a9
:10e980008009b00060017d008002eb00f4ff2c00e4
:10e9900085417800010c2000c002200064e40700db
:10e9a000823e200003002000906e8000a16e800057
:10e9b000860f0200000000000004eb00881f7800b2
:10e9c000f7ff2c0006c2b300884178000002be00a9
:10e9d00072c0b300010a200020042000f9e50700fe
:10e9e000823e200003002000806d8000916d800039
:10e9f000860f020000000000e2382700821f780026
:10ea0000f7ff2c0006c2b300884178000002be0068
:10ea100072c0b3000108200020042000e9e50700cf
:10ea2000006c8000e48757000098a3001a003200b1
:10ea30001980fb00000040008004b00060017d00f0
:10ea400088027800f4ff2c0088417800010520003e
:10ea50006001200036e407001980fb000000400040
:10ea60006c00400060017d0088027800f4ff2c00fb
:10ea70008841780001042000c00220002ce4070037
:10ea800043c0b3000341780083407800c0c0b300a6
:10ea9000c9e60700130037008002eb00f4ff2c00ea
:10eaa0008541780042c1b3000105200060012000cb
:10eab000aae707008002eb00f4ff2c0085417800f4
:10eac00042c1b3000104200060012000a3e7070059
:10ead00033c0b30042c0b30082407800c0c0b3006e
:10eae000b5e607004f0578004f04be0000000600a1
:10eaf00040da200010407800e44f50001c00320043
:10eb000008003e00e14f5000110032000d003900b6
:10eb1000e24f500011003200e34f500021003a0054
:10eb200011003700e64f5000160032001200390085
:10eb3000e74f500016003200e84f500019003a002d
:10eb40001600370000802f0033e40700150037005f
:10eb5000007e200030e4070012003700f0012000a2
:10eb60002de407000f0037005be407000d003700bd
:10eb700088e407000b0037000080eb0026e4070064
:10eb8000080037000000eb0023e407000500370011
:10eb90000080eb0033e40700020037000000eb00c8
:10eba00030e4070000000600889fbe00a8d92000be
:10ebb0001880fb00000040007800400021b12000d8
:10ebc000608178008002eb00f457280013c0b30086
:10ebd000010e200005007800d5e307007ae7070062
:10ebe000698c20001880fb00000040000009b00084
:10ebf00060817c008002eb00f4ff2c0085417800ee
:10ec0000010c200005007800c9e307001880fb0014
:10ec1000000040004009b00060817c00e53827001a
:10ec2000f4ff2c008041eb0001072000b000200021
:10ec3000bfe30700002d2100104278008001eb00a7
:10ec4000831f7800f7ff2c0006c2b3000482fb008c
:10ec50000500200022c0b30001072000000b2000a7
:10ec600058e507008f87e9004f04be00000006004a
:10ec70000042eb00e2dd2000044978006011b8009a
:10ec8000026f8800136f88000001eb007296880005
:10ec9000f2dd200004497800026c80001208b30005
:10eca000026c8800626c80000240a000626c8800e8
:10ecb000626c80000220a000626c8800626c8000a0
:10ecc0000270a100626c8800626c80000230a100ba
:10ecd000626c8800206f8800316f8800e07b200024
:10ece000201c8800c0772000801c8800e922a90031
:10ecf000401380008820a9009820a8002008200048
:10ed00004013880000000600606c80000030a10005
:10ed1000606c8800006c80000000a000006c88001f
:10ed2000606c80000040a000606c8800606c800017
:10ed30000408200004006800606c8800206f8000d8
:10ed4000316f800002c02f0000016100610bb8002c
:10ed5000c030dd00000020006113b8000600700024
:10ed600087807000206f8800316f8800206f8000de
:10ed7000316f8000024020000300200000004100ad
:10ed800081804900206f8800316f88007096800074
:10ed90000000e80070968800e07b2000201c8800be
:10eda000c0772000801c8800e922a9004013800061
:10edb0008820a9009820a800606c800004006000f2
:10edc0000300320050082000401388000200370082
:10edd000200820004013880000000600c403210022
:10ede000944178000381fb0041ec200000f17800a1
:10edf000034ae80000000600d40321009441780093
:10ee00000381fb0001f8200000f17800034ae800cc
:10ee100000000600889fbe008a9fbe008044eb0071
:10ee2000c00321000948780028df200010c0b3008b
:10ee30001044980000c0eb00e8ff07001840900065
:10ee4000e6ff070028409000e4ff070038409000ec
:10ee5000e2ff070018409000a840900001404000e9
:10ee6000b8409000014540000104e0000f0032006e
:10ee7000880578000984fb00640444000b04440006
:10ee80001840780000454500d4ff070000c0eb00a3
:10ee9000984f100001003a00d0ff07008944e800b5
:10eea0003b40900080cf5400f2ff39000a407800c8
:10eeb000caff0700c3eb2000134178008280fb00eb
:10eec00040ec2000614078000080fb00a011880029
:10eed0008249e8004f05be004f04be000000060056
:10eee000889fbe008a9fbe008044eb00f003210093
:10eef00009487800006c80000030a000006c880099
:10ef0000c0eb200009487800c003210009487800c0
:10ef100068e5200010c0b3001044980000c0eb006a
:10ef2000aeff070018409000acff0700284090009b
:10ef3000aaff070038409000a8ff07001840900083
:10ef4000a840900001404000b840900001454000ba
:10ef50000104e0000f003200880578000984fb00fe
:10ef6000640444000b044400184078000045450048
:10ef70009aff070000c0eb00984f100001003a0014
:10ef800096ff07008944e8003b40900080cf540082
:10ef9000f2ff39000a40780090ff0700c3eb200021
:10efa000134178008280fb0040ec20006140780033
:10efb0000080fb00a01188008249e8004f05be00d8
:10efc0004f04be0000000600889fbe008a9fbe005e
:10efd0008044eb00d003210009487800d0eb2000ea
:10efe0000948780068e5200010c0b300104498007c
:10eff00000c0eb0080ff0700184090007eff070074
:10f00000284090007cff0700384090007aff0700fe
:10f0100018409000a840900001404000b840900087
:10f02000014540000104e0000f003200880578002f
:10f030000984fb00640444000b0444001840780079
:10f04000004545006cff070000c0eb00984f100022
:10f0500001003a0068ff07008944e8003b40900047
:10f0600080cf5400f2ff39000a40780062ff0700a9
:10f07000d3eb2000134178008280fb0000f82000d1
:10f08000614078000080fb00201188008249e80080
:10f090004f05be004f04be0000000600889fbe0062
:10f0a0008a9fbe008044eb00d0032100094878000d
:10f0b000d0eb20000948780028df200010c0b30002
:10f0c0001044980000c0eb004bff07001840900070
:10f0d00049ff07002840900047ff07003840900094
:10f0e00045ff070018409000a840900001404000f4
:10f0f000b8409000014540000104e0000f003200dc
:10f10000880578000984fb00640444000b04440073
:10f11000184078000045450037ff070000c0eb00ad
:10f12000984f100001003a0033ff07008944e800bf
:10f130003b40900080cf5400f2ff39000a40780035
:10f140002dff0700d3eb2000134178008280fb00e5
:10f1500000f82000614078000080fb00201188004a
:10f160008249e8004f05be004f04be0000000600c3
:10f17000889fbe008a1f7800004178008141780096
:10f180008040eb00e003210001487800006c800023
:10f190000010a000006c8800c0eb2000014878003f
:10f1a00020df2000224098000280fb0001002000a8
:10f1b0006a005000e080580002052000820f5000d5
:10f1c000e08f580016013e0000600100500037003b
:10f1d0004f0037004e003700110137001001370093
:10f1e0000f0137004f003700490037000c0137008e
:10f1f0000b0137000a013700090137000801370009
:10f200000701370006013700050137000401370008
:10f210000301370002013700010137000001370008
:10f220004b00370056003700fd003700fc00370068
:10f23000fb003700fa003700f9003700f80037000c
:10f24000f7003700f6003700f5003700f40037000c
:10f25000f3003700f2003700f1003700f00037000c
:10f26000ef003700ee003700ed003700ec0037000c
:10f27000eb00370042003700e90037004c00370050
:10f28000e7003700e6003700e5003700e40037000c
:10f29000e3003700e2003700e10037004f0037009d
:10f2a0004e003700de003700dd003700dc0037009d
:10f2b000db003700da003700d9003700d80037000c
:10f2c000d7003700cf003700d5003700d400370013
:10f2d000d3003700d2003700d1003700d00037000c
:10f2e000cf003700ce003700cd003700cc0037000c
:10f2f000cb003700ca003700c9003700c80037000c
:10f30000c7003700c6003700c500370000003700cf
:10f3100021df200010c0b300b0409800c340980027
:10f32000c300370071c0b30020df200031409800d7
:10f330000000eb0062df200051da200061717800ec
:10f340000000e800e70f5000b9003200fbff370073
:10f3500041c2b30020df2000314098000000eb00e4
:10f3600083df20006227210091022000e2717800f3
:10f370000000e800810f5000ad003200fbff3700b5
:10f3800061c2b30020df2000314098000000eb0094
:10f3900063df200002db200061022000e2717800c0
:10f3a0000000e800810f5000a1003200fbff370091
:10f3b00081c0b30020df2000314098000000eb0046
:10f3c00062df200061dd2000617178000000e8004c
:10f3d000e80f500096003200fbff370081c5b300f4
:10f3e00020df200031409800c2948000d26f880056
:10f3f000d3948000e36f88002a9480008a0f510024
:10f40000040031000000eb00b06f8800c06f88007e
:10f410001400370040948000800f51000f0031002d
:10f420000194800040062000808f500008003a00c0
:10f430008a0f510006003a00309480000000e0007e
:10f440000300320090002000b06f880005003700f4
:10f45000b0002000b06f880002003700c00020001c
:10f46000b06f88000300e0000d003200402721004b
:10f47000006890000004e00006003a00409480001c
:10f48000808f510008003e00b0002000c06f88004f
:10f4900005003700c0002000c06f88000200370060
:10f4a000d0002000c06f880009002100f96f88009b
:10f4b0000001eb000270880008002200187088002c
:10f4c000227088000500240040272100108072006f
:10f4d00030708800040f200044708800c7032000ab
:10f4e000b09380000780b900030025000080710000
:10f4f000507088006270880006002300c09380006e
:10f500000600700070708800d093800080708800c2
:10f51000e09380000500700090708800a47088005f
:10f52000f09380000780b90000807100b0708800ff
:10f53000c27088000094800006007000d0708800bf
:10f5400010948000e070880005007500f07088005d
:10f5500004718800309480000780b9000080710039
:10f5600010718800227188004006230030718800e5
:10f57000427188004094800005007000507188003e
:10f5800054948000647188006094800003007000cf
:10f5900070718800827188000000260090718800d8
:10f5a000a27188000400270070948000040070009d
:10f5b000b071880080948000c071880090948000b1
:10f5c0000780b90080817100d3718800e2718800e2
:10f5d000a094800004007000f0718800027288001e
:10f5e000197288002272880038728800b3948000f3
:10f5f0004372880000002800507288006272880000
:10f600000b00370021df200010c0b300b04098008d
:10f61000e025210010c07100c040980004003700b0
:10f6200021df20000040eb00b0409800c04098006f
:10f63000f8fd07004f0578004f04be0000000600eb
:10f6400020df2000204090000080fb00010020000f
:10f6500061005000e080580022062000820f500018
:10f66000e08f580052023e00006001006200370047
:10f670007b00370085003700970037004c023700c9
:10f680004b0237009b003700490237004802370021
:10f69000a200370046023700450237004402370017
:10f6a00043023700a9003700ba003700c400370012
:10f6b000ce0037003e0237003d0237003c023700e3
:10f6c0003b0237003a023700390237003802370070
:10f6d0003702370036023700350237003402370070
:10f6e000c9003700320237003102370030023700dc
:10f6f0002f0237002e0237002d0237002c02370070
:10f700002b023700ce003700d80037002802370020
:10f71000e1003700eb003700f70037000101370048
:10f720000d0137001701370025013700200237008f
:10f730001f023700370137004701370051013700fa
:10f740005f0137006601370075013700800137001f
:10f7500017023700160237008701370014023700fe
:10f760008f0137009901370011023700100237006e
:10f770000f0237000e0237000d0237000c0237006f
:10f780009d013700a6013700b0013700080237009d
:10f79000c0013700ca013700d6013700e001370049
:10f7a000030237000202370001023700000237006f
:10f7b000ff013700fe013700fd013700fc01370073
:10f7c000fb013700fa013700f9013700f801370073
:10f7d000f7013700f6013700f5013700f401370073
:10f7e000f3013700f2013700f1013700f001370073
:10f7f000ef013700d501370021df200031409000b4
:10f80000e64f5000ea013a00406c80000010a10071
:10f81000406c8800f0252100c14190000348780029
:10f820000026210051429000044878001026210053
:10f83000e1429000054878002026210071419000a7
:10f840000248780030262100814990000348780062
:10f85000402621009148900001487800d4013700eb
:10f8600021df200031409000e14f5000d0013a00ec
:10f8700041409000e14f5000cd013a00206c8000e3
:10f880000010a100206c8800c901370021df200092
:10f8900031409000e54f5000c5013a00206c8000d7
:10f8a0000000a100206c8800b46f80005493880091
:10f8b000c0262100e142900005487800d0262100b2
:10f8c00071419000024878000004210081489000b6
:10f8d00001487800b601370020df2000304090005a
:10f8e000e24f5000b2013a00b36f800013828800eb
:10f8f000af01370021df200031409000e24f50007f
:10f90000ab013a0000db20004142900054589800bf
:10f91000d140900041589800a501370021df200018
:10f9200031409000e14f5000a1013a004140900069
:10f93000e14f50009e013a00206c8000f1fc2f0046
:10f9400001006000206c88009901370020df200052
:10f9500030409000e74f500095013a00206c800045
:10f960000020a100206c8800f06b80000000a00047
:10f97000f06b88000000eb0052da200061df20000d
:10f98000617178000000e800e70f50008801320044
:10f99000fbff370021df200031409000e14f500095
:10f9a00083013a0041409000e14f500080013a004d
:10f9b000206c80000030a100206c88007c013700a2
:10f9c00021df200031409000e14f500078013a00e3
:10f9d00041409000e14f500075013a00206c8000da
:10f9e00000f0a100206c88007101370020df2000aa
:10f9f00030409000e24f50006d013a00b06f80003f
:10fa0000208288006a01370020df2000b04090008b
:10fa100040c2b30080cf500065013a000000eb0007
:10fa20004327210062df200041022000e2717800bc
:10fa30000000e800810f50005d013200fbff37003d
:10fa400021df200031409000e14f500058013a0082
:10fa500041409000e14f500055013a00306c800069
:10fa60000050a100306c88005101370021df2000d8
:10fa700031409000e14f50004d013a00414090006c
:10fa8000e14f50004a013a00306c80000070a10044
:10fa9000306c88004601370021df200031409000a3
:10faa000e14f500042013a0041409000e14f5000c8
:10fab0003f013a00206c800000d0a100206c88003b
:10fac0003b01370021df200031409000e34f500020
:10fad00037013a0050262100e140900001487800ab
:10fae000b56f800095958800206c800000e0a10033
:10faf000206c88002e01370021df2000314090006b
:10fb0000e14f50002a013a0041409000e14f50007f
:10fb100027013a00306c80000030a100306c880072
:10fb20002301370021df200031409000e34f5000d7
:10fb30001f013a00306c80000040a100306c88004a
:10fb400050262100e140900001487800b06f80000d
:10fb5000909588001601370021df20003140900089
:10fb6000e14f500012013a0041409000e14f500037
:10fb70000f013a00206c800000b0a100206c8800ca
:10fb80000b01370021df200031409000e54f50008d
:10fb900007013a0050262100814890000148780072
:10fba000b26f800092958800c36f8000a395880093
:10fbb000206c800000c0a100206c8800fc00370091
:10fbc00021df200031409000eb4f5000f8003a0058
:10fbd000306c80000060a100306c8800502621004d
:10fbe000e148900001487800b46f80009495880047
:10fbf000c56f800075938800d06f8000b095880035
:10fc0000e26f8000c2958800f36f8000d395880072
:10fc1000e700370020df2000b040900060c2b30052
:10fc200080cf5000e2003a00206c80000090a100dc
:10fc3000206c88000000eb0003db200062df200066
:10fc400061022000e27178000000e800810f50009e
:10fc5000d7003200fbff370021df20003140900049
:10fc6000e14f5000d2003a0041409000e14f500077
:10fc7000cf003a00206c800000a0a100206c88001a
:10fc8000cb00370020df200030409000e84f5000cc
:10fc9000c7003a00206c80000070a100206c880032
:10fca0000000eb0062dd200061df20006171780060
:10fcb0000000e800e80f5000bd003200fbff3700f5
:10fcc00020df200030409000e84f5000b8003a009c
:10fcd000206c80000080a100206c8800b4003700f8
:10fce00020df200030409000f24f5000b0003a007a
:10fcf000316c80000000eb00e429210063df20006c
:10fd0000f2ef2f0063327800828060000080e8000c
:10fd1000f20f5000fbff3a00316c8800a40037005e
:10fd200020df200030409000e44f5000a0003a0057
:10fd3000306c800000f0a100306c8800b06f800053
:10fd400090958800c26f80009293880098003700d9
:10fd500020df200030409000e24f500094003a0035
:10fd6000306c80000090a100306c8800b36f800080
:10fd7000839388008e00370020df20003040900001
:10fd8000e24f50008a003a00406c80000000a10061
:10fd9000406c8800b46f8000349388008400370082
:10fda00021df200031409000e14f500080003a00f8
:10fdb00041409000e14f50007d003a00306c8000df
:10fdc00000c0a100306c88007900370021df2000de
:10fdd00031409000e14f500075003a0041409000e2
:10fde000e14f500072003a00306c800000d0a1005a
:10fdf000306c88006e00370020df2000304090001b
:10fe0000e24f50006a003a00b56f800045828800da
:10fe1000306c800000e0a100306c88006400370086
:10fe200021df200031409000e14f500060003a0097
:10fe300041409000e14f50005d003a00306c80007e
:10fe40000020a100306c88005900370022df20001c
:10fe500032409000e14f500055003a00306c800075
:10fe6000c1ff2f0001006000306c8800424090000c
:10fe7000e22521000049780061cab300014040003a
:10fe8000e64f50004a00360000c6b3000049780033
:10fe90004700370021df200031409000e14f500043
:10fea00043003a0041409000e14f500040003a00ca
:10feb000306c800000a0a100306c88003c0037004e
:10fec00021df200031409000e34f500038003a001d
:10fed000306c800000b0a100306c880050262100fa
:10fee000e140900001487800b06f80009095880054
:10fef0002f00370021df200031409000e14f5000fb
:10ff00002b003a0041409000e14f500028003a0099
:10ff1000406c80000020a100406c88002400370065
:10ff200021df200031409000e14f500020003a00d6
:10ff300041409000e14f50001d003a00406c8000ad
:10ff40000030a100406c88001900370022df20003b
:10ff500032409000e34f500015003a00206c8000c2
:10ff6000800078000160a100216c880091262100aa
:10ff700042419000824878000018a30003003a0034
:10ff8000406c80000038a30002003200902621005f
:10ff90000048eb0020df2000c12b210050419000e1
:10ffa00082487800812621006040900080487800d7
:10ffb000006c80000018a30001003a0037fc070025
:10ffc000c0eb20000048eb0000000600881f78000e
:10ffd000f00321000048eb00026c80000202780070
:10ffe0000430a000046c880060e52000a040900070
:10fff00040c6b30080cf50004300320007003e00ef
:020000040001f9
:10000000e6cf5000140032008101390068c0500072
:10001000e14f50007e013e0023003700e0c6b300f0
:1000200080cf5000be00320004003e006940500006
:1000300080cf500076013a0079003700f0c6b30057
:1000400080cf5000ee0032000040e80080cf50002a
:100050006f013a005101370060e52000b040900088
:10006000a0c2b30080cf50006a013a000000eb004c
:1000700043272100a2e5200091022000e2717800d0
:100080000000e800810f5000fcff3a0060e520000e
:1000900011c0b3003140980051c5b30041409800f1
:1000a000c9fb07005b013700d1728000d192880044
:1000b00060e52000b0419000e2cf51000b00360017
:1000c00022c0b3000000eb00a5042100c4e520001d
:1000d000e47278008100e8000241e8000000e800d6
:1000e00082cf5100faff3a00d192880060e52000eb
:1000f00011c0b3003140980051c5b3004140980091
:10010000b1fb07004301370062e52000b2409000d8
:100110000104e00012003a0010c0b3004041980012
:10012000040078000070a100006c8800606c800002
:100130000030a100606c8800606c80000060a1004d
:10014000606c8800f0dd200001487800e922a800fa
:10015000606c80000020a100606c88002b003700dc
:1001600020c4b30080cf500025003a000000eb000f
:10017000e37b2400a2e5200021042000e271780046
:100180000000e800810f5000fcff3a00f0dd200085
:100190000048eb000478a3000a003a00002d21007b
:1001a000104178000281fb000300200000c02800fd
:1001b0000010b8004211dd0081004100acfa0700d8
:1001c0000b003700606c80000028a300080032009c
:1001d000606c80000038a30002003200cafa0700f9
:1001e000030037008de3a80081e3a80083e3a800a3
:1001f00021c0b30060e520004140980003003700b3
:1002000031c0b30060e520004140980011c0b30048
:1002100060e52000314098006bfb0700fd003700cf
:1002200062e52000b24090000104e00012003a00b4
:1002300010c0b30040419800040078000070a10095
:10024000006c8800606c80000030a100606c880049
:10025000606c80000060a100606c8800f0dd200010
:1002600001487800e922a800606c80000020a1000d
:10027000606c88002500370020c4b30080cf500098
:100280001f003a000000eb00e37b2400a2e5200001
:1002900021042000e27178000000e800810f500086
:1002a000fcff3a00f0dd20000048eb000478a300da
:1002b00004003a0000002000310020006cfa070022
:1002c0000b003700606c80000028a300080032009b
:1002d000606c80000038a300020032008afa070038
:1002e000030037008de3a80081e3a80083e3a800a2
:1002f00021c0b30060e520004140980003003700b2
:1003000031c0b30060e520004140980011c0b30047
:1003100060e52000314098002bfb0700bd0037004e
:1003200062e52000b24090000104e00012003a00b3
:1003300010c0b30040419800040078000070a10094
:10034000006c8800606c80000030a100606c880048
:10035000606c80000060a100606c8800f0dd20000f
:1003600001487800e922a800606c80000020a1000c
:10037000606c88001d00370020c4b30080cf50009f
:1003800017003a000000eb00e37b2400a2e5200008
:1003900021042000e27178000000e800810f500085
:1003a000fcff3a000478a30003003a006000b800a4
:1003b0002ffa070006003700606c80000028a300b9
:1003c000030032008de3a80081e3a80083e3a800c6
:1003d00021c0b30060e520004140980003003700d1
:1003e00031c0b30060e520004140980011c0b30067
:1003f00060e5200031409800f3fa070085003700df
:1004000063e52000b34090000104e00012003a00d0
:1004100010c0b300c0419800040078000070a10033
:10042000006c8800606c80000030a100606c880067
:10043000606c80000060a100606c8800f0dd20002e
:100440001048e800e922a800606c80000020a100ac
:10045000606c88004c00370020c4b30080cf50008f
:1004600046003a000000eb00e57b2400a3e52000f5
:1004700021042000e37278000000e800810f5000a2
:10048000fcff3a00050820000478a30031003a0080
:10049000020078009008b300006c8800606c800057
:1004a0000040a000606c8800606c80000020a0000c
:1004b000606c8800606c800005006800606c8800db
:1004c000606c80000030a100606c88006000b800a3
:1004d000006f8800116f8800f0dd20001040780068
:1004e0000080fb00010020004a09dd00c600de009c
:1004f000810071004a00dd0002402000030020005e
:100500000000410081804900206f8800316f880021
:10051000e07b2000201c8800c0772000801c880021
:10052000e922a900401380008820a9009820a80093
:10053000606c80000500600003003200500820005d
:10054000401388000900370020082000401388006d
:1005500006003700606c80000028a3000300320012
:100560008de3a80081e3a80083e3a80021c0b300c5
:1005700060e52000414098000300370031c0b3001f
:1005800060e520004140980011c0b30060e5200004
:10059000314098008cfa07001e00370060e520000b
:1005a000b0409000a0c2b30080cf500010003a00cd
:1005b0000000eb0043272100a2e52000910220006b
:1005c000e27178000000e800810f5000fcff3a0063
:1005d00068e52000586890000080fb009a8b0200bc
:1005e0000000000010c0b300404498000300370032
:1005f00031c0b30060e520004140980011c0b30055
:1006000060e52000314098006ffa070001003700d4
:1006100033fa07004f04780000000600889fbe00f0
:10062000a8d920001880fb000000400068004000ae
:10063000c1822000608178008002eb00f45728001e
:1006400013c0b300010e200005007800983d0200a1
:1006500000000000e444020000000000e9972000d0
:100660001880fb000000400060817c008002eb00ed
:10067000f4ff2c0085417800010d20009007200038
:10068000983d0200000000001880fb0000004000c0
:100690006400400060817c008002eb00f4ff2c00cd
:1006a000854178000109200090072000983d020054
:1006b000000000001880fb000000400068004000bf
:1006c00060817c008002eb00f4ff2c008541780003
:1006d0000105200090072000983d02000000000066
:1006e000293a29001880fb0060c17c00610a2000c3
:1006f0000000eb00de8d0200000000001880fb000f
:100700006e00400060c17c00610a2000c003200030
:10071000de8d0200000000001880fb006a0040002f
:1007200060c17c00410620000000eb00de8d02006d
:10073000000000001880fb006c00400060c17c00dd
:1007400041062000c0032000de8d020000000000f2
:100750001880fb007e00400060c17c002102200068
:100760000000eb00de8d0200000000001880fb009e
:100770000002b00060c17c0021022000c003200004
:10078000de8d02000000000043c0b300034178008a
:1007900083407800c0c0b300dc42020000000000cb
:1007a0004f04be0000000600889fbe008a9fbe0066
:1007b000a0d920001080fb0000004000680040002d
:1007c000c1822000608178008002eb00f45728008d
:1007d00013c0b300010e200005007800983d020010
:1007e00000000000e444020000000000006c8000f3
:1007f0000068a300450032004027210000689000f7
:100800000004e0000500320051c0b300402d21007b
:1008100032c1b300904f1100010032008040eb0064
:100820008185fb005a2d21001a80fb00000040004a
:10083000692d21009980fb00010040000b00500051
:1008400000004000a8d920009880fb000100400073
:1008500000004000e1c42000608178008002eb00cd
:10086000f4ff2c0085417800010d20000500780080
:10087000983d0200000000001a80fb0000004000cc
:100880009980fb00010040000b0050000000400078
:100890009880fb00010040000000400061bf200084
:1008a000608178008002eb00f4ff2c008541780025
:1008b000010a200005007800983d020000000000b9
:1008c0001a80fb00000040009980fb0001004000fe
:1008d0000b005000000040009880fb000100400029
:1008e0000000400061ca2000608178008002eb00b7
:1008f000f4ff2c00854178000107200005007800f6
:10090000983d02000000000015003700a8d9200023
:100910001880fb0066004000213a290060c1780081
:10092000610a20000000eb00de8d020000000000e4
:100930001880fb000000400070004000e19720009c
:10094000608178008002eb00f4ff2c008541780084
:100950000109200005007800983d02000000000019
:1009600043c0b3000341780083407800c0c0b300a7
:10097000dc420200000000004f05be004f04be0034
:1009800000000600889fbe00a9d920001980fb0046
:100990000000400068004000c182200060817800b3
:1009a0008002eb00f457280013c0b300010e2000b2
:1009b00005007800983d020000000000e4440200b9
:1009c0000000000028d620001980fb000000400035
:1009d00060017c008002eb00f4ff2c008541780070
:1009e000010d200020042000983d020000000000be
:1009f0001980fb00000040006400400060017c00a2
:100a00008002eb00f4ff2c008541780001052000f6
:100a100020042000983d020000000000283a290030
:100a20001980fb000080e80060417c00610a200022
:100a30000000eb00de8d0200000000001980fb00ca
:100a40006600400060417c00210220000000eb00b5
:100a5000de8d02000000000043c0b30003417800b7
:100a600083407800c0c0b300dc42020000000000f8
:100a70004f04be0000000600881f7800a8d920009f
:100a80001880fb000000400068004000c182200088
:100a9000608178008002eb00f457280013c0b30097
:100aa000010e200005007800983d020000000000c3
:100ab000e444020000000000b0d920001080fb00d8
:100ac000000040009880fb00010040000000400052
:100ad00061992000608178008002eb00f4ff2c0017
:100ae00085417800010c200005007800983d020047
:100af0000000000043c0b300034178008340780049
:100b0000c0c0b300dc420200000000004f047800c7
:100b100000000600889fbe00a9d920001980fb00b4
:100b20000000400068004000c18220006081780021
:100b30008002eb00f457280013c0b300010e200020
:100b400005007800983d020000000000e444020027
:100b500000000000689920001980fb0000004000a0
:100b60000003b00060017c008002eb00f4ff2c0069
:100b700085417800010c200090072000983d02007c
:100b8000000000001980fb00000040004003b0009e
:100b900060017c008002eb00f4ff2c0085417800ae
:100ba0000108200090072000983d0200000000008e
:100bb000283a29001980fb007400400060417c0045
:100bc000610a20000000eb00de8d02000000000042
:100bd0001980fb007600400060417c00610a200023
:100be000c0032000de8d0200000000001980fb0021
:100bf0007800400060417c0041062000c0032000d6
:100c0000de8d02000000000043c0b3000341780005
:100c100083407800c0c0b300dc4202000000000046
:100c20004f04be0000000600889fbe00a8d9200027
:100c30001880fb000000400068004000c1822000d6
:100c4000608178008002eb00f457280013c0b300e5
:100c5000010e200005007800983d02000000000011
:100c6000e444020000000000699920001880fb00a5
:100c7000000040008003b00060817c008002eb0037
:100c8000f4ff2c0085417800010c20009007200023
:100c9000983d0200000000001880fb0000004000aa
:100ca000c003b00060817c008002eb00f4ff2c00e8
:100cb000854178000108200090072000983d02003f
:100cc000000000001880fb00000040004003b0005e
:100cd00060817c008002eb00f4ff2c0085417800ed
:100ce0000105200090072000983d02000000000050
:100cf000293a29001880fb007400400060c17c0084
:100d0000610a20000000eb00de8d02000000000000
:100d10001880fb007600400060c17c00610a200062
:100d2000c0032000de8d0200000000001880fb00e0
:100d30007a00400060c17c00410620000000eb000a
:100d4000de8d0200000000001880fb007c004000e7
:100d500060c17c0041062000c0032000de8d02003f
:100d6000000000001880fb007800400060c17c009b
:100d700021022000c0032000de8d020000000000e0
:100d800043c0b3000341780083407800c0c0b30083
:100d9000dc420200000000004f04be00000006001c
:100da000881f7800a8d920001880fb0000004000b0
:100db00068004000c1822000608178008002eb0062
:100dc000f457280013c0b300010e2000050078007e
:100dd000983d020000000000e44402000000000012
:100de000f0d920001080fb00000040009880fb003c
:100df0000100400000004000a1a7200060817800b1
:100e00008002eb00f4ff2c0085417800010d2000ea
:100e100005007800983d02000000000043c0b300c8
:100e20000341780083407800c0c0b300dc42020078
:100e3000000000004f04780000000600881f7800c2
:100e4000a8d920001880fb00000040006800400086
:100e5000c1822000608178008002eb00f4572800f6
:100e600013c0b300010e200005007800983d020079
:100e700000000000e4440200000000001880fb00b5
:100e80000000400068004000a1a7200060817800b9
:100e90008002eb00f4ff2c0085417800010c20005b
:100ea00005007800983d02000000000043c0b30038
:100eb0000341780083407800c0c0b300dc420200e8
:100ec000000000004f04780000000600889fbe006c
:100ed000a9d920001980fb000000400068004000f4
:100ee000c1822000608178008002eb00f457280066
:100ef00013c0b300010e200005007800983d0200e9
:100f000000000000e444020000000000a8a8200047
:100f10001980fb00000040006800400060017c0078
:100f20008002eb00f4ff2c0085417800010d2000c9
:100f300005007800983d0200000000001980fb00c9
:100f4000000040006c00400060017c008002eb006b
:100f5000f4ff2c0085417800010c2000050078008a
:100f6000983d0200000000001980fb0000004000d6
:100f70007000400060017c008002eb00f4ff2c0058
:100f800085417800010b200020042000983d0200dc
:100f9000000000001980fb000000400074004000c9
:100fa00060017c008002eb00f4ff2c00854178009a
:100fb0000107200020042000983d020000000000ee
:100fc0001980fb00000040007800400060017c00b8
:100fd0008002eb00f4ff2c00854178000103200023
:100fe00020042000983d020000000000283a29005b
:100ff0001980fb007600400060417c003108200031
:101000000000eb00de8d0200000000001980fb00f4
:101010007400400060417c00610420000000eb008f
:10102000de8d0200000000001980fb00640040001b
:1010300060417c00a10020000000eb00de8d02007a
:101040000000000043c0b3000341780083407800f3
:10105000c0c0b300dc420200000000004f04be002c
:1010600000000600889fbe00a8d920001880fb0061
:101070000000400068004000c182200060817800cc
:101080008002eb00f457280013c0b300010e2000cb
:1010900005007800983d020000000000e4440200d2
:1010a00000000000698c20001880fb000000400058
:1010b0000007b00060817c008002eb00f4ff2c0090
:1010c00085417800010b200005007800983d020062
:1010d000000000001880fb00000040004007b00046
:1010e00060817c008002eb00f4ff2c0085417800d9
:1010f0000108200030062000983d0200000000009a
:1011000043c0b3000341780083407800c0c0b300ff
:10111000dc420200000000004f04be000000060098
:10112000881f7800a8d920001880fb00000040002c
:1011300068004000c1822000608178008002eb00de
:10114000f457280013c0b300010e200005007800fa
:10115000983d020000000000e4440200000000008e
:101160001880fb0000004000c009b000618c200026
:10117000608178008002eb00f4ff2c00854178004c
:10118000010b2000b0002000983d0200000000008c
:1011900043c0b3000341780083407800c0c0b3006f
:1011a000dc420200000000004f047800000006004e
:1011b000881f7800a8d920001880fb00000040009c
:1011c00068004000c1822000608178008002eb004e
:1011d000f457280013c0b300010e2000050078006a
:1011e000983d020000000000e444020000000000fe
:1011f00010da20001080fb00000040009880fb0007
:10120000010040000000400021b52000608178000e
:101210008002eb00f4ff2c0085417800010a2000d9
:1012200060012000983d02000000000043c0b300b0
:101230000341780083407800c0c0b300dc42020064
:10124000000000004f04780000000600e922a8001a
:101250000041eb00e0dd20000248780041138000ef
:10126000f0dd200001487800024878006000b800f6
:10127000006f8800116f8800006c80000000a000e3
:10128000006c8800606c80000010a000606c88001a
:10129000606c80000070a100606c8800606c800051
:1012a0000060a100606c8800e07b2000801c88004a
:1012b000c0772000201c8800e922a9008820a9000e
:1012c0009820a8003000200040138800000006008d
:1012d000006c80000000a000006c8800606c800042
:1012e0000040a000606c8800606c80000020a000be
:1012f000606c8800606c80000208200002006800ba
:10130000606c8800606c80000030a100606c880018
:10131000606c80000060a100606c8800e07b2000b1
:10132000201c8800c0772000801c880040138000ab
:1013300001002000006f8800116f88006000b80075
:10134000006f8800116f8800e922a9008820a90099
:101350009820a800606c800002006000030032004a
:1013600050082000401388000200370020082000a9
:101370004013880000000600881f7800b3ff0700b4
:101380000041eb0006042000f7fb2f0018cdb3004e
:10139000606c800006006000fdff3200606c800021
:1013a00007006000606c8800e17b2400a504210038
:1013b00014cdb300038024000280fb0011f07a00fa
:1013c0000241e800844f510003003e008100e80024
:1013d000818f5100f8ff3a0081e3a8008de3a80057
:1013e0008fe3a80083e3a800884f5100e8ff360090
:1013f00081e3a9008de3a900606c80000010a100ca
:10140000606c8800e922a8004f0478000000060004
:10141000a2002000110009000280d8008000fd0019
:101420006109b8004a1add00c612de0085027200aa
:101430004a12dd00920220000280b900040140003f
:1014400085814800000027000100200002004000c4
:1014500083804800206f8800316f88007bff070081
:1014600001042000606c800001006000fdff32007c
:10147000606c80000060a100606c88000000eb00e0
:1014800043272100e27b240091022000e2717800d2
:101490000000e800810f5000fcff3a0081e3a90042
:1014a0008de3a900606c80000010a100606c8800d2
:1014b000e922a800b0948000ef0f5000020036002f
:1014c00010002000b0948800d0938000ef0f5000ef
:1014d0000200360020002000d09388001094800085
:1014e000ef0f5000020036000000eb00109488005f
:1014f000f0938000ef0f5000020036000000eb0078
:10150000f0938800b0938000ef0f50000200360087
:1015100020002000b09388004227210012007800ac
:10152000f4005000802a2000808f50000200360016
:10153000f023200000097800e09380007400500040
:10154000a1462000810f50000200360080252000b7
:10155000e093880022948000f4005100a04620000f
:10156000808f5000030036008025200020948800e2
:1015700005003700a0938000800f51000200310069
:101580000000e80020948800509480000000e900ea
:10159000f10e2000810f5000020036007003200081
:1015a0005094880030948000ef0f50000200360005
:1015b000200020003094880042948000f400510004
:1015c000c0492000808f500003003600e038200022
:1015d000409488000500370020948000800f51005f
:1015e000020031000000e80040948800619480000f
:1015f00000e12000808f500002003600c003200070
:1016000060948800c1948000004b2000808f5000bf
:10161000020036000000eb00c0948800d1948000e6
:1016200000e12000808f5000020036000000eb0037
:10163000d0948800a2948000f4005100c04920009a
:10164000808f50000300360000322000a0948800f4
:101650000900370040272100900f51000300390096
:1016600040948000800f51000300360040948000b9
:101670000000e900a094880070948000740050007d
:10168000c1492000810f50000200360020352000a3
:10169000709488004194800070948000810f500005
:1016a000020036000100e900709488007194800007
:1016b000a0948000808f500002003e000100e900ed
:1016c000a0948800c193800040062000808f5000c5
:1016d000020036006a005000c0938800d09380005a
:1016e000ef0f50000200360020002000d093880049
:1016f0000194800040062000808f500002003600d8
:101700006a0050000094880080948000ef0f500021
:10171000020036000000eb00809488009094800066
:10172000ef0f5000020036000000eb00909488009c
:1017300000000600881f780000047800a200200046
:10174000110009000280d800000178000300200089
:101750004a18dd00c611de00830170004a11dd0069
:1017600000002700010020000201400083814800a2
:10177000226f8800336f8800b4fe07000002eb0080
:1017800003042000f5fb2f00a60421000721200000
:10179000606c800003006000fdff3200606c800020
:1017a00005006000606c880086004200e07b240039
:1017b00002802400b0587800820f5000fdff3a00ec
:1017c0002404b000870f52000500320081e3a80016
:1017d0008de3a8008fe3a80083e3a800ecff3700a7
:1017e00081e3a9008de3a900606c80000010a100d6
:1017f000606c8800e922a800a20020001100090006
:101800000284d80001007800920220000280b90012
:10181000a20421000000410041272100d22921001b
:1018200031587800828f5000fdff3a000004eb0031
:10183000e27b2400a10421002004200061717c00cf
:101840000804e800800f5400fcff3a00a0fe0700e7
:101850007400200003042000f5fb2f00a6042100e3
:10186000606c800003006000fdff3200606c80004f
:1018700005006000606c880086004400e07b240066
:101880000280240031587800820f5000fdff3a009a
:101890008de3a80081e3a80083e3a8000402e90027
:1018a0002804b0000400e000edff3a00010420002d
:1018b000606c800001006000fdff3200606c800001
:1018c0000060a100606c8800e922a8008de3a900f7
:1018d00081e3a900606c80000020a100606c88009a
:1018e000606c80000040a100606c8800606c80002b
:1018f0000030a100606c88004f04780000000600f2
:1019000000c0260001002000206f8800316f880091
:101910004efe070001042000606c800001006000a2
:10192000fdff3200606c80000060a100606c8800e8
:101930000000eb0082de2000e17b24006171780072
:101940000000e800e70f5000fcff3a0081e3a90027
:101950008de3a900606c80000010a100606c88001d
:10196000e922a800d0122000920f100001003600da
:101970000009eb0081de200021409000e14f500083
:10198000020036000040eb00a040980081de2000fd
:10199000a0d92000214190000248780031409000f9
:1019a000fb4f5000020036000040eb00b0409800b2
:1019b00081de200041409000ea4f500002003600d6
:1019c0000040eb00c040980082de2000d240900032
:1019d00030c6b30080cf5000020036000040eb005c
:1019e0005041980082de2000e240900030c6b300f3
:1019f00080cf5000020036000040eb0060419800ac
:101a00000000060000c0260001002000206f8800b2
:101a1000316f88000000eb00e27b240081de2000b3
:101a2000617178000000e800e70f5000fcff3a0009
:101a300027fe070001042000606c800001006000a8
:101a4000fdff3200606c80000060a100606c8800c7
:101a5000e922a8008de3a90081e3a900606c800061
:101a60000020a100606c8800606c80000040a10034
:101a7000606c8800606c80000030a100606c8800a1
:101a800000000600e8874700889fbe008a9fbe00ce
:101a90008c9fbe008e1f7800f0b79f000104780075
:101aa0000207780083bf9f00e8fd07000fb9970089
:101ab00002f0b900e0b79f00001420000046b80013
:101ac0008005eb008b4078008b0478000b057800d4
:101ad0002b0037000005eb0024003700606c80000d
:101ae0000068a30026003200606c80000060a10046
:101af000606c8800e07b24000081eb00900f1100f7
:101b000002003a000104e00020003200e87b2400db
:101b100038017800ffb097000a80400000004600be
:101b2000e0804e000414200004cab9000400400004
:101b3000e0804800083b0200000000008b05e80040
:101b40000a05e8008a0f570005003e008904e800f6
:101b50000fb99700890f5100deff36000005eb003a
:101b600000802400800f5400e9ff3a0081e3a800c0
:101b70008de3a8008fe3a80083e3a80011c0b300a1
:101b80006fb09700808f5500d4ff390081e3a90022
:101b90008de3a900606c80000010a100606c8800db
:101ba000e922a8004f0778004f06be004f05be008f
:101bb0004f04be008f00b10000000600889fbe00e9
:101bc0008a9fbe008c9fbe008005780001057800ca
:101bd0000281fb0003002000008f21000016b800e6
:101be00002212000030020000c00be00a60f02000e
:101bf000000000000004be004a48dd00c644de00cc
:101c0000890470004a44dd00022120000300200006
:101c10000c00be00c40f02000000000008044000d9
:101c200089844800e3844400286f8800396f880065
:101c300093032000820320008a0078000b007800c4
:101c400090ff07004f06be004f05be004f04be00c8
:101c50000000060002402a00d3002000226f880006
:101c6000336f8800330620000301780085ff0700ea
:041c7000000006006a
:020000040000fa
:10000800baf60000baf60000d43a0000b23a00008e
:10001800baf600003c3a0000baf60000baf6000052
:10002800baf60000baf60000baf6000086340000fe
:100038005c3a0000baf60000baf60000baf6000012
:10004800baf60000baf60000baf60000a8380000b8
:100058008a390000baf60000263a0000baf6000015
:10006800baf60000baf60000baf60000baf60000c8
:10007800baf60000baf60000baf60000baf60000b8
:10008800baf60000baf60000baf60000baf60000a8
:10009800baf60000baf600009c3700004a380000a3
:1000a8007a370000ea360000baf60000baf6000017
:1000b800baf60000baf60000b4390000baf600003b
:1000c800baf60000baf60000baf60000baf6000068
:1000d800baf60000baf60000baf60000baf6000058
:1000e800baf60000baf60000baf60000baf6000048
:1000f800baf60000baf60000baf60000baf6000038
:10010800baf60000baf60000baf60000baf6000027
:10011800baf60000baf60000baf60000baf6000017
:10012800baf600007438000056390000baf600002c
:10013800baf60000baf60000baf60000baf60000f7
:10014800baf60000baf60000baf60000baf60000e7
:10015800baf60000baf60000baf60000baf60000d7
:10016800baf60000baf60000baf60000baf60000c7
:10017800baf60000baf60000baf60000baf60000b7
:10018800baf60000baf60000baf60000baf60000a7
:10019800baf60000baf60000baf60000baf6000097
:1001a800baf60000baf60000baf60000baf6000087
:1001b800baf60000baf60000baf60000baf6000077
:1001c800baf60000baf60000baf60000baf6000067
:1001d800baf60000baf60000baf60000baf6000057
:1001e800baf60000baf60000baf60000baf6000047
:0801f800baf60000baf600009f
:020000040000fa
:10020800baf60000baf60000d43a0000b23a00008c
:10021800baf600003c3a0000baf60000baf6000050
:10022800baf60000baf60000baf6000086340000fc
:100238005c3a0000baf60000baf60000baf6000010
:10024800baf60000baf60000baf60000a8380000b6
:100258008a390000baf60000263a0000baf6000013
:10026800baf60000baf60000baf60000baf60000c6
:10027800baf60000baf60000baf60000baf60000b6
:10028800baf60000baf60000baf60000baf60000a6
:10029800baf60000baf600009c3700004a380000a1
:1002a8007a370000ea360000baf60000baf6000015
:1002b800baf60000baf60000b4390000baf6000039
:1002c800baf60000baf60000baf60000baf6000066
:1002d800baf60000baf60000baf60000baf6000056
:1002e800baf60000baf60000baf60000baf6000046
:1002f800baf60000baf60000baf60000baf6000036
:10030800baf60000baf60000baf60000baf6000025
:10031800baf60000baf60000baf60000baf6000015
:10032800baf600007438000056390000baf600002a
:10033800baf60000baf60000baf60000baf60000f5
:10034800baf60000baf60000baf60000baf60000e5
:10035800baf60000baf60000baf60000baf60000d5
:10036800baf60000baf60000baf60000baf60000c5
:10037800baf60000baf60000baf60000baf60000b5
:10038800baf60000baf60000baf60000baf60000a5
:10039800baf60000baf60000baf60000baf6000095
:1003a800baf60000baf60000baf60000baf6000085
:1003b800baf60000baf60000baf60000baf6000075
:1003c800baf60000baf60000baf60000baf6000065
:1003d800baf60000baf60000baf60000baf6000055
:1003e800baf60000baf60000baf60000baf6000045
:0803f800baf60000baf600009d
:020000040000fa
:020000040001f9
:101c74000106000001060000010400000506000042
:101c8400070b00000c1e0000201f0000c80000000d
:101c9400fa00000078050000780500008c0a0000b6
:101ca4008c0a00004100000096000000fe000000c5
:101cb4001e00000000000000ee020000ee02000022
:101cc4009001000090010000230000003200000099
:101cd40000000000140000000000000000000000ec
:101ce40000000000140000000000000000000000dc
:101cf40000000000140000000000000014000000b8
:101d040001000000000000001400000000000000ba
:101d14000000000014000000000000001400000097
:101d240014000000bc0200000f000000640000006a
:101d34000f000000bc0200000f000000640000005f
:101d44000f000000b00400000f000000b004000009
:101d54008c000000100e0000b00400000f00000012
:101d64000f000000b00400000f000000b0040000e9
:101d7400b0040000173b00001f0c000063000000cb
:101d84000001000001000000020100000405000041
:101d940006000000f4010000000000000000000044
:101da40000000000f40100000000000064000000d6
:101db40000000000580200000000000000000000c5
:101dc4003c0000003c000000520300000000000042
:101dd40000000000510300000100000000000000aa
:101de4000000000010170000401700006e170000ec
:101df40090170000a6170000ce170000f41700008b
:101e04002e1800006c180000b81800002a1a0000f0
:101e1400b61a0000bc020000000000000000000030
:101e240000000000bc02000000000000640000008c
:101e340000000000bc02000000000000c00300001d
:101e44008c00000058020000520300000000000053
:101e54000000000051030000010000000000000029
:101e640000000000841c0000a61c0000941d00005b
:101e7400aa1d0000c01d0000201e00003c1e000022
:101e8400621e0000841e000008000000090000001b
:101e94000a0000000d000000544500000e830000fd
:101ea400b84600001e150000e24700001e150000a1
:101eb400344800001e150000884800001e1500006c
:101ec400f86100001e150000b24800001e15000055
:101ed400d44800001e150000d44800001e15000060
:101ee400b64900001e150000d47500001e15000040
:101ef400224a00001e1500000c4b00001e150000b5
:101f0400044c0000d483000074500000c28400001c
:101f1400e05d00001e150000345e00001e15000088
:101f2400745e00001e150000586000001e150000bd
:101f34007c6000001e150000d86000003c85000095
:101f44004a6100008a850000b26100001486000026
:101f54003e6200001e1500002e640000d0860000c2
:101f6400906400001e150000f26500001e8700004a
:101f74009c66000066870000c06800001e15000013
:101f8400ce69000032880000426a00001e1500007d
:101f9400a46a00001e150000be6b00001e150000a0
:101fa400e06d000090880000666e00001e150000c1
:101fb400c06e00001e150000066f00001e15000014
:101fc400626f00001e150000c06f00001e150000a7
:101fd4006e700000d88800001e7100001e150000fd
:101fe400967200001e150000967400001e15000075
:101ff400787500001e150000841500007a29000081
:102004004415000062220000c62800006415000088
:102014001e150000281600001e1500001e150000e5
:102024003e29000044150000201500001e15000084
:1020340064150000262900001e1500003229000046
:102044001e1500001e1500001e15000020150000be
:102054001e1500001e1500001e1500001e150000b0
:102064001e1500001e1500001e1500001e150000a0
:10207400201500001e1500001e1500001e1500008e
:10208400201500001e1500001e1500001e1500007e
:102094001e150000201500001e1500001e1500006e
:1020a4001e1500001e1500001e1500001e15000060
:1020b4001e1500001e150000dc2800001e1500007f
:1020c4001e1500001e1500001e1500001e15000040
:1020d4001e1500001e1500001e150000201500002e
:1020e4001e1500001e1500001e1500001e15000020
:1020f4001e1500001e1500001e1500001e15000010
:10210400201500001e1500001e1500001e150000fd
:102114001e1500001e1500001e1500001e150000ef
:102124001e150000702700001e1500001e1500007b
:102134001e1500001e1500001e1500001e150000cf
:10214400141600001e15000058220000021600009c
:102154001e1500001e1500001e1500001e150000af
:102164001e1500001e1500001416000020150000a6
:102174001e150000021600001e15000020150000a8
:102184001e150000fa2800009e22000044150000dd
:102194002015000082220000641500001e150000b6
:1021a400c0220000201500001e1500000e230000b0
:1021b40044150000a8270000f62200006415000062
:1021c4001e150000d0150000a827000028160000e6
:1021d4002c230000ba240000482400005a230000e5
:1021e400a224000008240000ca2400009a2300004e
:1021f4003a1600001e1500002c280000f6270000e7
:102204001e150000042800001e150000e62700002b
:102214001e1500001e1500001e1500001e150000ee
:10222400982400001e1500001e1500001e15000055
:10223400942700001e1500001e1500001e15000046
:102244001e150000201500001e1500001e150000bc
:102254001e1500001e1500001e1500001e150000ae
:102264001e1500001e150000201500001e1500009c
:102274001e1500001e1500001e1500001e1500008e
:102284001e1500001e1500001e150000201500007c
:102294001e1500001e1500001e1500001e1500006e
:1022a4001e1500001e1500001e1500001e1500005e
:1022b4001e1500001e1500001e1500001e1500004e
:1022c4009c2900001e150000281600009a15000025
:1022d4004415000020150000ac1500006415000032
:1022e4001e150000d218000020150000281600005a
:1022f4001e150000181900002a1900001e15000000
:10230400061900001e150000561900002a190000c5
:10231400281600001e150000441600002a190000ab
:102324001e15000072160000de1600006019000081
:10233400a61600001e1500001e1500006a190000f4
:10234400cc1900001e150000741900001e150000b1
:102354007e1900001e15000028160000041a000053
:102364004415000020150000161a00006415000032
:102374001e150000d21a0000201500001e150000d2
:102384001e150000921a0000661a0000161b0000b9
:10239400a41a00001e1500007c1a0000661a000032
:1023a400281600001e150000f61a00002a19000065
:1023b4001e150000e01a00001e1500000c1b000092
:1023c4002a190000561b00001e150000da1b00002d
:1023d400601b00001e150000a01b00001e1500005d
:1023e400261b00001e1500001e1500001e1500000f
:1023f4001e150000141c00001e1500001e15000010
:102404001e150000401c0000141c000028160000cb
:102414001e15000088280000201500001e1500006d
:10242400942800001e150000a028000020150000bc
:102434001e1500005e1c00001e1500002015000083
:10244400701c00001e1500001e150000d01c0000aa
:10245400201500001e1500001e1500001e150000aa
:10246400201500001e1500001e1500001e1500009a
:10247400de1c0000201500001e1500001e150000c3
:102484001e150000221d00001e1500001e15000070
:102494001e150000041d0000661a00002816000026
:1024a4001e150000881d0000201500001e150000e8
:1024b4007c1d00001e150000662800002015000089
:1024c4001e150000421d00001e1500002a19000000
:1024d400541d00001e1500001e150000681d00009c
:1024e4002a190000881800008818000088180000c5
:1024f40020150000881800008818000088180000c3
:1025040088180000881800001e150000e01800005c
:102514004415000020150000f218000064150000a6
:102524001e1500009e1e0000201500001e15000050
:102534001e150000ac1e0000201500001e15000032
:10254400ce1e00001e1500001e1500001e15000002
:102554001e1500001e1500001e15000020150000a9
:102564001e1500001e1500001e1500001e1500009b
:102574002015000028160000f01e0000921f000025
:102584002a190000401f0000e21f00001e15000071
:10259400322000001e150000fa200000082100006f
:1025a40072210000e22000003c2100009221000082
:1025b4001e150000b22100001e1500001e150000ab
:1025c4001e1500001e150000ec2100001e15000061
:1025d4001e1500001e150000062200001e15000036
:1025e400242200001e1500001e1500002c220000ed
:1025f4001e1500001e1500001e1500003e220000de
:102604001e1500001e15000054290000c01500000e
:1026140020150000682900001e1500001e1500008a
:102624001e1500001e15000000000000d728000041
:102634000000000000000000000000000000000096
:1026440032000000000000006100000000000000f3
:10265400100000000000000037000000000000002f
:102664002700000000000000170000000000000028
:102674005601000087000000050100000000000072
:10268400ef000000000000000d000000000000004a
:102694000000000000000000000000000000000036
:1026a400a000000000000000000000000000000086
:1026b400a000000000000000000000000000000076
:1026c4000000000000000000000000000000000006
:1026d40000000000000000000000000000000000f6
:1026e40000000000000000000000000000000000e6
:1026f400000000000000000001000000d7280000d6
:102704000000000000000000641400000408000041
:102714000c10000020240000282c0000303400009d
:10272400383c00004044000050540000585c000055
:10273400607000007480000084880000641400004d
:1027440008010000090200000a0400000b05000053
:102754000c0c00000d0300000e0600000f0000002a
:1027640011110000100700001212000013130000e2
:1027740014140000151500001616000017170000a9
:1027840018180000d65c000034440000b54c00006a
:10279400375d0000fa7500005b7e00009c7e00003f
:1027a4009c7e00009c7e00007e7e00009b7e0000dc
:1027b400fc8600005eb70000dfe70000ffff0000ba
:1027c400ffff0000f65c0000f75c0000fa7d0000eb
:1027d4001a8600003daf0000ffcf0000ffcf0000cd
:1027e400ffc70000fec70000fec70000ffcf0000c7
:1027f400544c000054440000544c0000d55c0000cc
:10280400b87d00001ca70000dfc70000ffcf000058
:10281400ffcf0000ffc70000ffc70000b54c000059
:10282400b54c0000b5540000744c0000734c00001b
:10283400f55c00003a8e00007eb70000ffcf000078
:10284400ffcf0000ffcf0000576500005765000070
:1028540057650000f65c0000344c0000134400008f
:10286400b55c0000997500003eaf0000ffc7000092
:10287400ffcf0000f96d0000f9750000f975000044
:10288400d96d0000d7540000754c0000754c000051
:1028940095540000d97d00007eb70000ffc70000fa
:1028a4007b7e00007b7e00007b7e00007b7e000040
:1028b4003a760000f75c0000964c0000754c00006e
:1028c400b45400009b960000bfbf00007b7e000054
:1028d4007b7e00007b7e00007b7e00007b7e000010
:1028e4001a760000175d0000964c0000744c00003e
:1028f400b87500009fb700009b7e00009b7e00001f
:102904009b7e00009b7e00009b7e00009b7e00005f
:10291400f96d0000175d0000b6540000f55c00007e
:102924005fa700009c7e00009c7e00009c7e00004f
:102934009c7e00009c7e00009c7e00005b76000074
:102944009865000016550000d55c0000fe9e00004e
:102954009c7e00009c7e00007c7e00007c7e00004b
:102964007c7e00007b7e00005b7e0000d965000059
:102974005655000016650000dd9e00009b7e000099
:102984009b7e00009b7e00009c7e00009c7e0000dd
:102994009c7e00009c7e00003a760000b965000031
:1029a400586d0000de9e0000fc8e0000fc8e0000ce
:1029b400fc8e0000fc860000fc860000fc8e0000fb
:1029c400fc8e0000db8e00005b7e0000d9750000e9
:1029d400fe9600007eb700007eb700007eb70000c0
:1029e4007db700007db700009ebf00009ebf0000c1
:1029f4007dbf00001d9f0000bb8e00005d9f000096
:102a0400dfef0000dfef0000dfef0000dfef00008a
:102a1400dfef0000ffef0000ffe70000dfe700004a
:102a2400bec700005cb700009ebf0000ffff0000af
:102a3400ffff0000ffff0000ffff0000ffff00009a
:102a4400ffff0000ffff0000fff70000ffe70000aa
:102a5400ded70000ded70000ffff0000ffff00000c
:102a6400ffff0000ffff0000ffff0000ffff00006a
:102a7400ffff0000ffff0000ffe70000ffd700009a
:102a8400ffd700000001000002030000040500005d
:102a940006070000080900000a0b00001e0c0000d5
:102aa4000d0e00001e0f0000101100001213000094
:102ab400020100000001000002010000000100000a
:102ac40002010000020300000104000002010000f2
:102ad40005010000020100000202000000010000e4
:102ae4000504000008000000c4eb0000ff20000003
:102af400e1fb0000f1f20000f0ee0000e3ee000064
:102b040020ee0000f1e20000eee50000ede8000038
:102b1400ff200000f0e00000e1ee0000f2fb000006
:102b240020f1000020ef0000e5f70000fcfe0000ab
:102b340020e80000f1ef0000eeeb0000fce70000ed
:102b4400f3e90000f2e50000f0e50000e6e800002b
:102b5400ec20000022cf0000eeec0000eef90000b3
:102b6400fc2200000ac20000f5ee0000e420000090
:102b7400e8e7000020eb0000fee10000eee30000c7
:102b8400ee200000f0e00000e1ee0000f7e50000b8
:102b9400e3ee000020ec0000e5ed0000fe20000064
:102ba400efee000020ea0000edee0000efea000086
:102bb400e53a0000004f00007065000072610000fb
:102bc400746900006e6700002066000075720000e2
:102bd4006e610000636500002c2000007573000026
:102be400650a000022480000656c000070220000a5
:102bf40020770000686500006e65000076650000bf
:102c0400720a00006e6500006365000073730000c3
:102c140061720000792e00000a4500006e74000005
:102c24007279000020660000726f00006d200000c1
:102c3400616e0000792000006d6500006e75000073
:102c44000a620000792000006b650000793a0000f8
:102c540000ce0000f8e80000e1ea0000e000000017
:102c640045720000726f00007200000053500000b3
:102c7400492d0000eef80000e8e10000eae0000061
:102c840000530000504900003a2000004572000043
:102c9400726f0000720000005532000046450000cb
:102ca400525200002dee0000f8e80000e1ea0000b6
:102cb400e00000005532000046450000525200007a
:102cc4003a20000045720000726f0000720000009c
:102cd400553200004f450000525200002dee000016
:102ce400f8e80000e1ea0000e000000055320000ce
:102cf4004f450000525200003a2000004572000087
:102d0400726f00007200000055310000464500005b
:102d1400525200002dee0000f8e80000e1ea000045
:102d2400e00000005531000046450000525200000a
:102d34003a20000045720000726f0000720000002b
:102d4400553100004f450000525200002dee0000a6
:102d5400f8e80000e1ea0000e0000000553100005e
:102d64004f450000525200003a2000004572000016
:102d7400726f000072000000444d0000412d0000fd
:102d8400eef80000e8e10000eae000000044000082
:102d94004d4100003a20000045720000726f0000af
:102da4007200000053740000616300006b20000097
:102db40054720000617000002dee0000f8e800007d
:102dc400e1ea0000e00000005374000061630000c9
:102dd4006b20000054720000617000003a20000073
:102de40045720000726f0000720000004164000030
:102df40064720000657300007320000054720000c8
:102e0400617000002dee0000f8e80000e1ea000027
:102e1400e00000004164000064720000657300007b
:102e24007320000054720000617000003a2000001a
:102e340045720000726f000072000000cfe00000d5
:102e4400f0e00000ece50000f2f00000fb200000e0
:102e5400f0e50000e6e80000ece0000020c200001d
:102e6400e0ea0000f3f30000ec200000f3f10000be
:102e7400f2e00000ede00000e2eb0000e8e2000018
:102e8400e0fe0000f2f10000ff200000f2ee00007e
:102e9400ebfc0000eaee000020ea0000edee00008a
:102ea400efea0000e0ec0000e8200000222b000024
:102eb400222c0000222d0000222e000000560000cb
:102ec40061630000757500006d20000070610000f2
:102ed400726100006d65000074650000727300008b
:102ee4002069000073200000736500007420000056
:102ef400627900002042000075740000746f0000c5
:102f04006e730000206f00006e6c000079000000fa
:102f1400202000002020000020cf0000f0ee000060
:102f2400e4ee0000ebe60000e8f20000fc20000004
:102f34002d200000ceca0000202000002000000048
:102f4400202000002020000020200000436f00000b
:102f54006e740000696e000075650000202d00008d
:102f6400204f00004b200000202000002000000023
:102f74002020000020200000203f000028ef000057
:102f8400eeec0000eef90000fc290000202d00000a
:102f940020ce0000ca2000002020000020000000f5
:102fa4002020000020200000202000003f280000f6
:102fb400686500006c700000292000002d200000ce
:102fc400ceca0000202000002020000020000000c5
:102fd40020200000202000002020000020200000ed
